:1000000000800020BD010000459D0000FD9C000017
:10001000FD9C0000FD9C0000FD9C0000FD9C00007C
:10002000FD9C0000FD9C0000FD9C0000459D000023
:10003000459D0000FD9C0000C5930000C994000090
:10004000459D0000459D0000459D0000459D000028
:10005000459D0000459D0000459D0000459D000018
:10006000459D0000459D0000459D0000459D000008
:10007000459D0000459D0000459D0000459D0000F8
:10008000459D0000459D0000459D0000459D0000E8
:10009000459D0000459D0000459D0000459D0000D8
:1000A000017900000D790000459D0000459D00008C
:1000B000459D0000459D0000459D0000459D0000B8
:1000C000459D0000459D0000459D0000459D0000A8
:1000D000459D0000459D0000459D0000459D000098
:1000E000459D0000459D0000459D0000459D000088
:1000F000459D0000B1BD0000459D0000DDBE000033
:10010000459D00001DA70000459D0000459D000085
:10011000459D0000459D0000459D0000459D000057
:10012000459D0000459D0000459D0000459D000047
:10013000459D0000459D0000459D0000459D000037
:10014000459D0000459D0000459D0000459D000027
:10015000B5950000C9950000DD950000F1950000FF
:10016000459D000039AA0000459D0000459D000006
:10017000459D0000459D0000459D0000459D0000F7
:10018000459D0000459D0000459D0000459D0000E7
:10019000459D0000459D0000459D0000459D0000D7
:1001A000459D0000459D0000459D0000459D0000C7
:1001B000459D0000459D0000459D0000564B4CF2BA
:1001C000205210B51A804DF628121A8000BF00BFC9
:1001D00009F0BCFD514B4FF010621A60504A9A6012
:1001E000504ADA60504A136813F4807304D14F49BF
:1001F0000B604FF4A85313604D4B1A78110703D5C9
:100200001A7842F008021A704A4B4B492A221A7097
:100210004A4A4B4B8B4204D252F8040F43F8040B6A
:10022000F8E7484B484900228B4202D243F8042B9E
:10023000FAE74649464A002352F8230041F82300D2
:1002400001336F2BF8D1434B434A802103F8011B44
:100250009342FBD1414B3D4A1A60414B8A221A70AE
:10026000A3F5805324225A70A0221A709A7992071B
:10027000FCD59A79D406FCD43A4A937903F00C035E
:10028000082B384BF9D103221A7140225A719A79FE
:100290009006FCD5334A9179324B4906FBD5324A58
:1002A000324911600221516020221A709A7902F0BD
:1002B0000C020C2AFAD12E4B2E4A1A602E4B2F4AD2
:1002C0001A6000225A60072243F8042C2C4AC3F813
:1002D0000C2D62B60AF0EAF8144B1B68DA0705D554
:1002E000284809F0B7FE284B284A1A60284B1B788B
:1002F0005B0609D5244C254B22689A4204D121483B
:1003000009F0A8FE002323600DF0A2F809F024FDF7
:1003100009F052FCFEE700BF0E200540308004408B
:10032000823F04000100002B10D0034014D0034092
:1003300002D0074000E00740549AFF1F2C01010043
:100340004088FF1F549AFF1F44A1FF1F0082FF1F18
:100350000000000000E400E05FE400E008ED00E0E1
:100360000050064000400640448004400000030165
:1003700004800440C010050014E000E0FF76010096
:1003800000002020840F7A5E1CE00340A5C3945A2D
:1003900000F00740FFFFFFFFFFFFFFFFFFFFFFFF32
:1003A000FFFFFFFFFFFFFFFFFFFFFFFFFFFFFFFF5D
:1003B000FFFFFFFFFFFFFFFFFFFFFFFFFFFFFFFF4D
:1003C000FFFFFFFFFFFFFFFFFFFFFFFFFFFFFFFF3D
:1003D000FFFFFFFFFFFFFFFFFFFFFFFFFFFFFFFF2D
:1003E000FFFFFFFFFFFFFFFFFFFFFFFFFFFFFFFF1D
:1003F000FFFFFFFFFFFFFFFFFFFFFFFFFFFFFFFF0D
:10040000FFFFFFFFFFFFFFFFFFFFFFFFDEF9FFFF23
:1004100010B5054C237833B9044B13B10448AFF33E
:1004200000800123237010BD549AFF1F00000000BC
:1004300030010100084B10B51BB108490848AFF363
:1004400000800848036803B910BD074B002BFBD0A0
:10045000BDE81040184700BF00000000589AFF1F79
:1004600030010100549AFF1F0000000038B5044617
:10047000104621700A491D460CF0CCFD01464FF094
:100480007E500CF07BFE07490CF0C4FDE560606017
:100490002561656109F09AFFE061204638BD00BF23
:1004A000DB0FC9400024744938B50446104621705A
:1004B00009491D460CF0AEFD01464FF07E500CF090
:1004C0005DFE06490CF0A6FDE56060602561656192
:1004D00009F07CFFE06138BDDB0FC940002474499E
:1004E00038B503780446032B20D8DFE803F01A1848
:1004F0001002C16840690CF083FC0D490546606834
:100500000CF03CFE014628460CF038FE38BD084988
:1005100040680CF033FEE1680CF07CFD38BDC0682B
:1005200038BDC16840690CF06BFC38BD002038BD97
:100530000024744970B504460E4609F047FF05468D
:10054000E069281A0CF012FDE3682361E561666139
:10055000A061014660680CF011FE0146A0601048E1
:100560000CF00CFE0CF0E2F80BF082FD0CF0F4FB4A
:10057000054601464FF07E500CF042FC61690CF0DC
:1005800049FD2169064628460CF044FD01463046E7
:100590000CF038FCE0602046BDE87040FFF7A0BFDB
:1005A000000080BF08B50E2009F0E0F9114B1B8850
:1005B000012B19D0104B1B88984213DB40F6FF71BA
:1005C0008842D4BFC3EB0001C3EB0101C1EB013191
:1005D000C3F57F630F33282091FBF3F1BDE808409A
:1005E00009F04ABD0021F3E70146BDE808401420A8
:1005F00009F042BD669BFF1FF69AFF1F10B5044627
:1006000008F0B6FF204610BD70B44C88A04220D937
:1006100001230133DBB21CB2660031F8144084427E
:100620001D46F6D3A04211D005F10045013D965B71
:1006300031F8151032F81530401AF21A00FB02F0AA
:10064000641A90FBF4F4E01870BC7047905B70BCC7
:10065000704702260125E5E700280CDA064A4342E6
:1006600082FB0320DA17C2EB600000EB4000A3EB33
:100670008000C0F10C007047ABAAAA2A2DE9F04710
:100680000C2009F03FF90C2009F0F4FD95491420E5
:1006900009F000FE9449954806F038FE0221032037
:1006A00009F08EFE0221042009F08AFE02210520B5
:1006B00009F086FE0221062009F082FE01210A20AF
:1006C00009F07EFE0121092009F07AFE01210D20AA
:1006D00009F076FE0121282009F072FE0121142084
:1006E00009F06EFE02210B2009F06AFE01210C20A8
:1006F00009F066FE0C20002109F04EFE042009F0EE
:1007000051FE70B3052009F04DFE044680B300246D
:100710002046774D287004F045FB2B78EBB9204636
:1007200005F000FE734B74491B88744C0988744AA9
:100730002170A3F5AF7140F23A7303FB01F382FB22
:100740000312DB176F4D7048A3EB621332335A214B
:100750002B6007F085F990B9FEE7BDE8F04706F099
:10076000E5BC062009F01EFE0028CBD10124D0E70D
:10077000032009F017FEB0FA80F04009C9E7634A88
:1007800063481268DFF8D8A100230121FFF78CFE2F
:100790000B2009F007FE011E0CBF012300238AF87D
:1007A000003002D1112009F00BFEDFF87481594EA0
:1007B000594F5A4D0023C8F8003033603B604FF06A
:1007C000040914E009F0D2F833681844306009F0E5
:1007D000010080F0010003F081FA2B88002B14BF88
:1007E0004B20FA2009F014FEB9F1010919D00F20AD
:1007F0000AF000F83B6803440E203B6009F0B6F8AD
:10080000D8F800309AF800200344C8F800301520CA
:10081000002AD7D1112009F0EDFF33681844306069
:10082000D5E73B68D8F800203D493068DFF834E16F
:100830002D88002BB8BF0333002AB8BF03329210B3
:100840000A603849384A0988128800284FEAA30309
:10085000B8BF03303B608010344F30605E1A1944DB
:100860003E60CEF80010324F324E3349C2EB000EDC
:100870000244C7F800E032600B605DB94FF4FA70D3
:1008800003F03CFA03F026FA04F04AFD40F2DC5093
:1008900009F0BEFD294B012504201D6009F082FDF1
:1008A00010B9274B20701D70264B1B881C2B0FD0B6
:1008B000254A264B1078187005F03EFC03F006FA26
:1008C00045F6BF5222492348BDE8F04708F006BE6E
:1008D000214B18880028EBD0204BC0B2197805F0C6
:1008E00073FBE5E7001B3746801A06005C8FFF1F8D
:1008F000B89BFF1F689BFF1FAA9AFF1FD99BFF1F72
:10090000B5814E1BA089FF1F949BFF1FA889FF1F65
:10091000FC9AFF1FC49AFF1FB49AFF1FFC9BFF1F86
:10092000609BFF1F9C89FF1FA489FF1FB49BFF1FB3
:10093000309BFF1F9C9BFF1F489BFF1F9C9AFF1F24
:10094000229BFF1FF89AFF1F429BFF1F8A9BFF1FDE
:10095000A5050000349BFF1FA69AFF1FD49AFF1F16
:10096000F69BFF1FD49BFF1FF0B40E8886420DD26A
:1009700003F10043013B31F81350854202D9F0BC2A
:10098000FFF742BE32F81300F0BC70471088F0BC8D
:10099000704700BF094B1B880C2B09D8084A80B24E
:1009A00052F8232028B143F6FE73984203D9108CE5
:1009B0007047108870470349FFF726BE6A9BFF1FE8
:1009C00088E6000044E50000374A38491088384A74
:1009D000F8B5384B12881B68834248DB9342A8BFA6
:1009E000134698420B60C8BF002342DD101AB0F5D1
:1009F000804FAABF9B03C3EB8333013093FBF0F01E
:100A0000FFF7C8FF2C4B2D4F1C883B68C0F3C61561
:100A100005FB04F47F2CA8BF7F249D42064608D026
:100A2000274B1B88002B38D1264B1B88002B30D13D
:100A30003D60254D2B689E4205D0214B1B885A1FD7
:100A4000032A1DD92E60214D2B689C420ED0204BCD
:100A5000188848B11A4B1F4A1B88D35C834203D0C5
:100A6000C0B2E1B205F0B0FA2C60F8BDF8BD0346A3
:100A700008609A42D4BFC0EB0203C0EB0303B5E7A2
:100A8000144AD05C2030C0B206F07F0105F09CFA19
:100A9000D8E7284605F00CFBCAE70E4A2946D05C89
:100AA00005F092FAC0E700BFF69AFF1FEC9AFF1F0D
:100AB0000A9CFF1F909AFF1F9A9AFF1F7C9AFF1FA4
:100AC0008C9AFF1F7C9BFF1FC89AFF1F749AFF1F01
:100AD000889BFF1F2489FF1F2DE9F04F172089B045
:100AE00009F088FEAF4B1860162009F083FEAE4B6C
:100AF000AE4A1B8810600C2B00F03B81AC4BAD4A1A
:100B000019880093AC4B52F8214000221A70AB4B6D
:100B1000AB4D1B88AB4A2E88013B32F91370002E77
:100B20005CD0A94BA94A1B88A9491278013B31F92D
:100B30001380002A40F0DF80112009F05BFEA54BF6
:100B40000193D3F800A00646B24540F3DF80A24BE4
:100B5000DFF8A4921B88A14A012BD9F80030B2F823
:100B600000B09F4A02922046C8EB030800F09A8228
:100B70000CF0FCF9029A52F82B100CF04BFA0146DB
:100B800000200CF03DF90CF00BFCCAEB0802B0455C
:100B9000B8BFB0469042CAEB080880F2968200FBCC
:100BA0000888013298FBF2F08E4BDFF850820293F6
:100BB000D8F80030034403EBD3735B10C8F800305F
:100BC0002B88012B12D1884BDFF834B20393874B6B
:100BD000DBF8005004934FF0000A47E07D4B01938F
:100BE000DFF814927F4BDFF8148202937E4B03935D
:100BF0001D460F2009F0FEFD2B689842824641DA1F
:100C0000754A1288012A00F01D82744A05931288E1
:100C1000734D049220460CF0A9F9049ADFF8E0B174
:100C200055F82210DBF800500CF0F4F901460020D2
:100C30000CF0E6F80CF0B4FBEF1B059B5745A7EB57
:100C40000302B8BF5746FF1A9042BABF013200FBF9
:100C50000777474397FBF2F7D8F80020634B0493DC
:100C6000BB1803EBD3735B10C8F80030604B1B88D4
:100C7000013B032B00F2B082DFE813F06301A9010E
:100C8000C4008601594B04931B68984240F3C2810B
:100C9000514A1288012A00F0A682504A079311880F
:100CA0004F4A0691204605920CF060F9059A069984
:100CB000DFF84CB152F82110DBF800500CF0AAF923
:100CC0000CF06EFB079B2F445745A7EB0302A8BF10
:100CD0005746FF1AD8F800309042BABF00FB07779A
:100CE0000132474397FBF2F73B4403EBD3735B10AE
:100CF000C8F80030BAE7152008F038FE354B0193EC
:100D0000D3F800A00646B2453FF721AF354B02931A
:100D1000D3F800A0B24580F289812F4BDFF8D8903C
:100D20001B882E4A012BD9F80030B2F800B02C4AAB
:100D300003922046984400F070820CF017F9039A51
:100D400052F82B100CF066F90CF02AFBB045CAEBF8
:100D50000802A8BFB046CAEB08089042B6BF00FB25
:100D6000088800FB08F8013298FBF2F0DFF88C806D
:100D70001EE7204B1B78002B3FF4C0AE0C4B0D4AF6
:100D8000198800930C4B52F8210001221A700CF0C4
:100D9000EDF84FF07C510CF03DF90CF001FB0446EE
:100DA000B5E600BF849AFF1FF89AFF1F4C9BFF1FF8
:100DB0008E9BFF1F3889FF1FBE9AFF1F7489FF1F7C
:100DC0008A9AFF1F08E700007689FF1FF69BFF1F26
:100DD00020E70000309BFF1F069CFF1F3E9BFF1F6C
:100DE000E0E600009C9BFF1FB49BFF1FD49BFF1FEE
:100DF000AC89FF1FFA9BFF1FC49AFF1FA09AFF1F19
:100E0000B49AFF1F28460CF0B1F8B2490CF002F971
:100E1000054650460CF0AAF8AF490CF0FBF8014625
:100E200028460BF0EFFF0CF0BBFA0546CBF800505C
:100E3000D9F800000CF09AF8A6490CF0EBF8074638
:100E400030460CF093F8A4490CF0E4F8014638461B
:100E50000BF0D8FF0CF0A4FAC9F800009F4AA04B91
:100E6000168819889F4AA04B12681B889F4FC6EBB3
:100E7000050E3544039EC6F800E0461A084404995E
:100E80000D6001990E6002993E8808609A4280F2D6
:100E900089810025C3EB060E954974450F6880F2E1
:100EA0007681611C9F4205FB01F50EF1010E95FB59
:100EB000FEF5C0F2BE81BE42A8BF3E46F61A01FB57
:100EC00006F494FBFEF49A4200F33681BB42C0F272
:100ED0003381884C20680CF049F887490CF09AF867
:100EE00086490BF08FFF0CF05BFAA0F5FF531C3B1B
:100EF000082B98BF4FF40050D8F800301844002851
:100F00002060C0F24281B0F5804F80F252817C4B6C
:100F10001B781BB1B0F5005F40F05381794D2B7801
:100F2000002B40F05481784D20682B68714C98421A
:100F300004D080B205F026F923682B6009B0BDE823
:100F4000F08F28460CF012F870490CF063F8054653
:100F500050460CF00BF86E490CF05CF80146284640
:100F60000BF050FF0CF01CFA0546CBF80050D9F8F6
:100F700000000BF0FBFF65490CF04CF807463046CB
:100F80000BF0F4FF62495FE728460BF0EFFF5A4988
:100F90000CF040F8054650460BF0E8FF5D490CF0B8
:100FA00039F8014628460BF02DFF0CF0F9F90546FB
:100FB000CBF80050D9F800000BF0D8FF4E490CF0E8
:100FC00029F8074630460BF0D1FF52493CE7284646
:100FD0000BF0CCFF50490CF01DF8054650460BF0C5
:100FE000C5FF4E490CF016F8014628460BF00AFFE3
:100FF0000CF0D6F90546CBF80050D9F800000BF0FC
:10100000B5FF45490CF006F8074630460BF0AEFF39
:10101000424919E7D8F80030DFF810B103EBD37379
:101020005B10DBF80050C8F800301FE6DFF80081E5
:10103000DFF80091D8F8003003EBD3735B10C8F8E9
:101040000030BDE5364A06931188364A05912046A0
:101050000492DFF8D8B00BF089FF049A0599DBF809
:10106000005052F821100BF0D5FF0CF099F9EF1B4E
:10107000069B5745A7EB0302B8BF5746FF1AD8F89F
:1010800000309042BABF013200FB0777474397FB1D
:10109000F2F73B4403EBD373234A04925B10C8F886
:1010A0000030E3E50BF062FF029A52F82B100BF0D0
:1010B000B1FF0CF075F9CAEB0802B045B8BFB046F5
:1010C0008242CAEB08083FF76AAD00FB08F898FBBC
:1010D000F2F069E5CDCC4C3FCDCC4C3E9C89FF1F56
:1010E000A489FF1F849AFF1FF49BFF1F649BFF1FAF
:1010F0004C9BFF1F7089FF1F9A99193FCDCC4C451F
:101100008E9CFF1FA59AFF1F2089FF1F3333733F5B
:10111000CDCC4C3DCDCCCC3E6666663FCDCCCC3DF7
:101120003E9BFF1FE0E60000D49BFF1FB49AFF1F09
:10113000A09AFF1FC49AFF1F009B1B88002B3FF43F
:10114000C8AE2B1B002BB8BF5B42092B47DD05F552
:1011500000500130001B0BF009FF3B493B4C0BF0EA
:1011600059FF054620680BF001FF39490BF052FF8B
:10117000014628460BF046FE0CF012F9D8F8003074
:10118000184400282060BFF6BEAE002213E09F4244
:1011900005FB04F5B8BF002195FBFEF54BDA91FB8A
:1011A000FEF490E6B242D4BFC3EB0205C3EB0605E2
:1011B00070E643F6FF72274B22601B78002B3FF44A
:1011C000ADAE02F087FD244B01221A70ABE602F0AF
:1011D0007DFD00232B70A6E6D9F800003EE64FF413
:1011E00000501A4C88E61D491D4A069320460D887A
:1011F00005920BF0BBFE059ADFF868B052F8251097
:10120000DBF800500BF006FF014600200BF0F8FD64
:101210000CF0C6F82F44069B56E50BF0A7FE039A88
:1012200052F82B100BF0F6FE014600200BF0E8FD03
:101230008AE51E4642E6B742D4BFC3EB0701C3EBC3
:10124000060104FB01F1AAE7CDCCCC3E7089FF1F5B
:101250009A99193F8E9CFF1FA59AFF1F3E9BFF1F67
:10126000E0E60000B49AFF1F08B5244B1B88FBB1D1
:10127000234B1B78FBB1234B1B78E3B1224B1B782C
:10128000CBB1224B1B78B3B1214B22481A78C2B99B
:10129000214A22490088128809680244B1EB620F92
:1012A00009DD01221A706420BDE8084002F026BD65
:1012B000174A117801B908BD1370BDE8084004F061
:1012C0002BBF154A16490088128809680244B1EB01
:1012D000620FF0DD00221A7004F01EFF642002F09D
:1012E0000DFD642002F00AFD642002F007FD4FF4BA
:1012F0001670BDE8084009F08BB800BFB09AFF1F18
:10130000F09AFF1FAD9AFF1FAE9AFF1FAF9AFF1F03
:10131000989AFF1F649BFF1FF49BFF1F849AFF1F77
:101320004C9BFF1F2DE9F84FAB4C20680BF01EFEC5
:10133000AA490BF06FFE0546102009F05BFA0BF08E
:1013400015FEA7490BF066FE29460BF05BFD0CF07D
:1013500027F8A44B20601B88192B00F08C801A2BD7
:1013600000F0A4800126B1469F4D2B88002B2DD084
:1013700020689E4F3A88824233DD9D4A11780029C9
:1013800077D00024012B147000F09D80022B40F0D8
:101390003F81002E00F09D80964D2B68002B00F0C1
:1013A00098800420214604F00FFE934B2C6018888F
:1013B00000285ED0B9F1000F5BD0C0B2002104F06C
:1013C00003FE8E4B00221A60BDE8F88F8A4A12880D
:1013D000002ACDD1864B1978002972D01A70BDE849
:1013E000F88F834991F80080B8F1000F33D14FF0A6
:1013F000010E042B81F800E02DD1002E40F02C814D
:101400002B88022B01D0032B66D07B4B1888002839
:101410002FD0B9F1000F2CD023683C88784AA34222
:10142000128880F2D1800023141B7E2C734DD5BF0F
:10143000C3EB8313C3EBC3135B00013493FBF4F4DE
:101440002B680134A34203D0C0B2E1B204F0BCFD6A
:101450002C60BDE8F88F2B88012B67D0022BD2D1EE
:10146000002ED2D0DFF88CB1DFF894A1DBF8003089
:1014700087E0BDE8F88F634D634F2B784BB15E4A30
:10148000128832B13978994200F0D980D0B27F21E8
:1014900005E03A789A4246D0574B1878002104F07C
:1014A00093FD00262B783B70B1465DE7554B1B78CA
:1014B000002B0BBF012600264FF000094FF0010959
:1014C00052E7BDE8F88F26B14A4D2A68002A40F05D
:1014D000BB80494B18886BE74C4B1B88092B94D079
:1014E000002E92D023683D88454AAB42128880F294
:1014F000D9800023551B7E2DDFF8F8B0D5BFC3EB94
:101500008313C3EBC3135B00013593FBF5F5DBF8E5
:1015100000300135AB4203D0E9B24A2004F054FD5B
:10152000CBF8005071E70026B1461DE7002E3FF4CE
:101530006CAFDFF8CCA0BAF800309842D4BFC2EB51
:101540000008C2EB03089A1A7E2A40F3A280C8EB77
:10155000C81002F1010890FBF8F808F10108DFF863
:1015600094B0DBF80030434504D05FFA88F10120E5
:1015700004F02AFD2B88CBF80080022B7FF443AFC8
:1015800043462268B7F80080BAF80010424579DA7D
:101590000022C8EB0108B8F17E0FD3BFC2EB821264
:1015A000C2EBC21208F10108520092FBF8F808F1F0
:1015B0000108984504D05FFA88F1042004F004FD86
:1015C0002B88CBF800801EE79342D4BFC4EB030303
:1015D000C4EB020328E700BF509BFF1F9A99193FF5
:1015E000CDCCCC3EF89AFF1FBA9BFF1FC09BFF1FBC
:1015F000AC9AFF1FC09AFF1F789AFF1FE89AFF1F3F
:101600002E9BFF1FFA9BFF1F1E9BFF1F8C9AFF1F25
:10161000032B2CD12C4B1B88092B3FF45AAF002EE7
:101620003FF457AF294D2B68002B3FF452AF4A20AF
:10163000214604F0C9FC264B2C601888B8E6254DDD
:1016400000262B88B14694E61846214604F0BCFCDF
:101650001F4B2C601888ABE67F21402004F0B4FCBF
:101660002B88012B25D0022B7FF4CDAEFAE6042B7C
:101670007FF42FAF002E3FF42CAF2146402004F022
:10168000A3FC26E78A42D4BFC8EB0202C8EB0102E2
:101690007FE7C8EB88184FEA480898FBF2F808F192
:1016A00001085CE79342D4BFC5EB0303C5EB02031B
:1016B00020E720683A88DFF820A09042BAF800308E
:1016C000FFF641AF39E700BF8C9AFF1FC09AFF1F9A
:1016D000789AFF1FBA9BFF1F2E9BFF1F08B50F4B69
:1016E0001B88022B0FD0032B12D0042B03D00C4BE2
:1016F00001221A7008BD7F21092004F065FC084B07
:1017000001221A7008BD7F21412004F05DFCEEE744
:101710004021092004F058FCE9E700BF2C9BFF1F83
:10172000C49BFF1F38B51C4B1B881D2B26D01B4BA1
:101730001B88012B25D01A4A1A4B14881B681A4A99
:10174000A342128818DB9342D4BFC4EB0303C4EB5B
:101750000203141B7F2CC6BFDB010134C3EBC31390
:1017600093FBF4F4114D2B689C4203D0E1B20520A9
:1017700004F02AFC2C6038BD0023EAE70C4B1C88DF
:10178000F0E70C4B0C4A0D491B6812680C689B1A59
:101790001C1B84F30704E5E7F89AFF1F8A9AFF1FD2
:1017A000A09BFF1FD09BFF1FF29AFF1F909BFF1F64
:1017B000D49AFF1F489BFF1F3089FF1FC89BFF1F44
:1017C00010B50F4C23685BB90E4B1B88022B11D050
:1017D000033B012B09D90C4A00231370236010BD71
:1017E0000021052004F0F0FBEEE70021092004F0C1
:1017F000EBFBF0E70021412004F0E6FBEBE700BF44
:10180000909BFF1F2C9BFF1FC49BFF1F08B5274BFE
:101810001B78ABB1152008F0A9F8254A254B128892
:1018200018601D2A15D0244A1288EAB1012A25D051
:10183000224B1B78002B34D0BDE80840FFF7C0BF17
:10184000112008F0D7FF1A4A1A4B128818601D2A77
:10185000E9D11B4B1B78002BEAD0184B1B780BB33C
:10186000BDE80840FFF75EBF164A1288002ADFD0A5
:10187000154A1B6812889A42DADCEEE70F2008F05E
:10188000B9FF104B114A1B88106033B1104B114A3D
:101890001B6812689B1A9842DFDD084B1B78002BEF
:1018A000CAD108BDFFF71AFFDAE700BFF69BFF1F9A
:1018B000F89AFF1FD09BFF1F8A9AFF1FC49BFF1F30
:1018C000FA9BFF1F2C9BFF1FA09BFF1FC89BFF1FA6
:1018D000489BFF1F3089FF1F2DE9F04F87B003ADF4
:1018E0008E4F2C4606AE611BC9B28D4806F07CF8BF
:1018F0003B88834294BF0020012004F8010BA642DC
:10190000F1D18848884A9DF80C50884905709DF8A7
:101910000E00874E10709DF810209DF81430854FF2
:10192000854C0A709DF81210317000263B702670AD
:1019300063B9002940F0D380002A40F0D8807F4A64
:10194000002800F0DC800223237005E0002A40F02C
:101950008C800523794A2370794DDFF828B29DF8F1
:101960000DE09DF80F00DFF820A2DFF82092DFF8ED
:101970002082744F744E13709DF811109DF816203C
:101980009DF8133085F800E08BF800009DF815E015
:101990009DF817C089F80020012088F8003087F8EA
:1019A00000E08AF8001086F800C008F023FF674ABC
:1019B000674BD2F800E07045CCBF012200221A70BC
:1019C00057DD644B1988182953D80C39624B2D7890
:1019D0001A789BF800C09AF800A099F8003098F89F
:1019E0000080DFF8B0913F7836782478A2EB45028A
:1019F000AAEB8A0BCCEB02025A44C3EB837BC3EB0A
:101A00008B03134403EB4803B9F80020DFF88891F7
:101A10003B4406FB02334FF00C0B1BFB0433C9F8AD
:101A20000030BAF1000F06D02EB1042A0CBF0233E9
:101A30000433C9F80030494A494C12882488033AD3
:101A400002EB420203EB820222440C3A114495B1AC
:101A5000B8F1000F0FD0BCF1000F44D1BAF1000F64
:101A600051D1404A012414700EE006232370334AFA
:101A700072E70021AAE73B4A00241470BCF1000F72
:101A800000D027BB4FF0000C374A704582F800C0E9
:101A9000C4BF364A1360364A1368994213D0354B97
:101AA000354C18680190019820601B680293334CF4
:101AB000029B248811601B1AA34284BF304B19601B
:101AC00007B0BDE8F08F2C482A4B0068EDE7002DE9
:101AD000D8D1BAF1000FD5D14FF0010CD4E70423CF
:101AE0002370164A38E71F4A00241470CAE7134AC5
:101AF0001378002B3FF424AF032323702CE735B178
:101B00000123237028E7174A82F800C0BCE7137846
:101B1000012B8CBF23702B461EE700BF689BFF1F65
:101B2000949BFF1FAD9AFF1FAE9AFF1FAF9AFF1F36
:101B3000B09BFF1FB29AFF1F809AFF1F3C9BFF1FA5
:101B4000F79BFF1FF49AFF1F049CFF1FA089FF1F34
:101B5000FA9BFF1FF89AFF1F6C89FF1F209BFF1F36
:101B6000CE9BFF1F409BFF1F419BFF1F009CFF1F41
:101B7000949AFF1FF09CFF1FB89AFF1F089CFF1F3D
:101B8000CC9AFF1FF89BFF1FF99BFF1FF09AFF1FC6
:101B90007A9BFF1F5C9BFF1FF09BFF1F2DE9F04FFF
:101BA0003A4B1B788BB0002B6BD10E2007F0DEFE7A
:101BB0000BF0DCF901463648364C374DFEF7BAFCDF
:101BC0003348FEF78DFC0BF0EBFB80F30C0020603C
:101BD000FFF782FE2E68012E7AD0022E00F0A88236
:101BE000032E00F0B7832D4C23682D4A2D4E099308
:101BF000099B177830682C4C07210122181A11FB19
:101C000007229042236000F28E82284E32689A1A90
:101C10000D2A00F28182264E32689A1A132A00F2A7
:101C20007682244E32689A1A252A18D9224B1B88AC
:101C3000002B40F06581214B1B78002B40F0608128
:101C40001F4B1B881B3B9BB2022B04D81D4B1B78E0
:101C5000002B40F0588102F063F8236833601A4D7E
:101C60002A689B1A502B00F21182184B1B88012BFB
:101C700000F0298204F03CFA04F06AF80BB0BDE8E9
:101C8000F08F05F0DBF80BB0BDE8F08FB89BFF1FBD
:101C9000FC9AFF1F909AFF1F9C9AFF1FF09CFF1F4A
:101CA000D89BFF1FA89BFF1FD89AFF1F849BFF1F75
:101CB000549BFF1FE89BFF1FB09AFF1F989AFF1FBE
:101CC000F89AFF1FFA9BFF1F289BFF1F669BFF1FB1
:101CD000DFF82883A34AB8F800001378834204D0C1
:101CE000C3B21846137004F03FF9DFF80C939E4A14
:101CF000B9F800301178994204D09C4F3978002906
:101D000040F07E879A4A236812889A4C9A42C0F221
:101D1000FF80994A1278002A40F0FA80DFF8E0A2AA
:101D2000BAF8003023B9954B1B88002B00F01F85B3
:101D3000934A944B11881B88934A0B4412685B109A
:101D40009342924A126880F2C28400219342B4BF47
:101D500001230B4604910093ACBF4FF0010B8B465F
:101D600005910E2007F002FE894B8A4A1B6817680E
:101D700003930133A7F25232002B8446029240F3C0
:101D80005087802BA8BF8023834A84491278019111
:101D9000002A00F0C7800978914200F0C380B9F8AA
:101DA0000010DFF854E2994201F047816F49AEF824
:101DB00000307B4B4FF0010E81F800E01978DFF81E
:101DC00044E2019B8EF800101A70009B002B00F07B
:101DD0001B81BAF80030002B00F01681714B1B6894
:101DE0005A1C002A40F32187802A00F31D876E4E7B
:101DF0006E496F483688098800683144B0EB610F3E
:101E0000C1F2EF81A3F148020F2A02D8473BA8F89C
:101E100000300E2007F0AAFD6FF454731F44874270
:101E200002DC644B00221A70002008F0E3FC624AD6
:101E3000624B1168624E1B888842D4BF0022012287
:101E40003270002B00F03A845E4B1E78964240D0F0
:101E500088423EDD5C490E78002E00F0CB875B495E
:101E600091F800C0BCF1000F40F0C287584F0097B6
:101E7000584F59480297564F007887F800C0554F81
:101E80004FF0010E87F800C081F800E0002841F013
:101E9000668152490978002901F027805049039151
:101EA0000E460978002941F01D804E48494F0078C0
:101EB000397001210297317058B14548434900906B
:101EC000002008700099029F0870039901263E7057
:101ED00008701A70444B1B88A3F11B02012A40F2C0
:101EE0006A861D2B7FF480AE3E4F3B78002B41F07D
:101EF000E9803E4E3378002B40F06984337073E6FE
:101F0000FFF7B2F99CE62B68012B7FF4A4AEA4E6A0
:101F10002168374A069106983649106002220B6004
:101F20002A60FBE61E49DFF8DCE0097800293FF46F
:101F300048AF9EF8000081423FF443AF03984B281E
:101F400041F327801833802BB9F80000A8BF802305
:101F500098423FF436AF28480380044801230370B9
:101F60002FE700BF8A9BFF1FD99BFF1F229BFF1FEC
:101F7000F69AFF1FF09CFF1F989AFF1F1C9BFF1FE4
:101F8000649BFF1FF49BFF1F849AFF1F4C9BFF1F46
:101F9000009CFF1F609BFF1F409BFF1FDA9BFF1FE2
:101FA000419BFF1FF09BFF1FC09BFF1F2E9BFF1F2E
:101FB000509BFF1FEC9BFF1FA089FF1F8C9BFF1FE7
:101FC000D19AFF1FE49AFF1FF09AFF1FD09AFF1FBC
:101FD000449BFF1FA49AFF1F7A9BFF1FF79BFF1FC5
:101FE000D29AFF1FFA9BFF1FF89AFF1F1E9BFF1F2D
:101FF000709AFF1FDC9BFF1FAA9AFF1F429BFF1FC7
:10200000BC9BFF1FDB9BFF1F029B9C45BFF601AFE4
:10201000AC4B1B88002B3FF4FCAEBBF1000F7FF4F0
:10202000DDAEA94B1B881BB1059B002B7FF4D6AE00
:10203000049B002B3FF4EDAEA44B1A78002A7FF4EA
:10204000E8AEDFF8048398F8006001221A70002ED1
:1020500040F05A839E4B1B78002B01F004819D4B6E
:102060001B78002B01F015819B4B1B78002B7FF414
:10207000D0AE9A4B1B78002B3FF4CBAEB9F80030B2
:1020800097490A3BA9F800300A70C2E602F0D2FE76
:10209000944B1B7873B9944B1B785BB9934B1B78AB
:1020A00043B9934B1B782BB9924B1B7813B901F0B2
:1020B0000DFE01E001F016FE23682B608E4B1B889D
:1020C000012B7FF4D7AD8D4A8D4B11688D481A785E
:1020D000A1F118032A2101FB03F10160002A00F09D
:1020E000D782894A1368994200F3458380F24F836F
:1020F00086480068D0F17F0048BF0330801001306F
:102100001B1A994200F3438313601946C2E2FFF79A
:102110007DFB2368336084E5FEF7DEFCFFF702F900
:102120002368336077E5FEF74FFC236833606CE586
:10213000774A26681288B24204DB6E4B1B78002B6C
:1021400000F04083734C744823680793734B0799DE
:1021500000681B88091A994263D8002B61D0704B24
:10216000198800293FF440AD6E4B6F481B6800880A
:10217000B342B8BF33469A4241F32C806B4B1A608E
:10218000DFF8C88188F800105C4FFEF71DFC386846
:102190007F2840F32986664B7F3883FB0032C317C4
:1021A000C3EB620303EB4303A0EB83007330614B8B
:1021B00001931B883860002B40F031874B4B009314
:1021C0001B78002B00F05A845B4E3378002B00F014
:1021D0005584DFF87C91DFF858A14FF0000B0CE03C
:1021E00003F17300C0B298F8001003F015FF3378C4
:1021F0000BF1010B5B4540F341843B6859F8040F38
:102200001844A0F17F038AFB0321DA17C2EB6102B5
:1022100002EB42027F28A3EB8203E1DCFEF71CFA0B
:10222000E0E7404B40491B6808883D49B342B8BFCE
:1022300033469A4200F3AD823C4E09888342A8BFE0
:102240000346336000299BD19A42C8BF0B4640F336
:10225000A782801AB0F5804FAABF9B03C3EB8333DC
:10226000013093FBF0F0FEF795FBC0F3C6100AF0C7
:102270007DFE324B064618880AF078FE3049074644
:1022800030460AF0C7FE014638460AF0C3FE314622
:102290000AF0B8FD4FF07E5106460BF059F80028C1
:1022A00040F08D87274930460BF070F8002840F049
:1022B0004A8730460BF09AF8C0B2DFF8908088F871
:1022C000000061E71C9BFF1FBE9BFF1FEC9BFF1FD5
:1022D000F79BFF1FF89BFF1FF99BFF1FF09AFF1F43
:1022E000229BFF1FA49AFF1FD09AFF1F449BFF1F32
:1022F000D29AFF1F989AFF1F669BFF1FCC9AFF1F61
:10230000C49BFF1FA49BFF1FE09AFF1F909BFF1F12
:10231000F69AFF1FF09CFF1F709AFF1F809BFF1F04
:10232000589BFF1FDC9BFF1F0A9CFF1FEC9AFF1F9F
:10233000ABAAAA2A249BFF1F3489FF1F889AFF1F7C
:10234000CDCCCC3D0000FE42809AFF1FDC9AFF1FDF
:102350007489FF1FB94B26681988B14253DDB84B09
:102360001B78002B4FD1DFF8209399F800007F28CD
:1023700040F3A486A3F155337F3803F1004383FB78
:102380000032C317C3EB620303EB4303A0EB8300EC
:102390007330AC4B01931B88C0B289F80000002B4E
:1023A00040F0ED86A84B00931B78002B00F04D8584
:1023B000A64E3378002B00F04885A54FDFF89882B1
:1023C0004FF0000A0AE003F17300C0B203F04CFEC4
:1023D00033780AF1010A534540F3378557F8043F33
:1023E00099F800001844A0F17F0388FB0321DA1755
:1023F000C2EB610202EB42027F28A3EB8203E2DC24
:10240000FEF72AF9E1E7934F38687F2840F3CF8140
:10241000914B7F3883FB0032C317C3EB620303EB9E
:102420004303A0EB83007330DFF85C9299F800A0BF
:10243000824500F02682894B1B88002B43D1884AB5
:10244000884812680088914205DC8242D4BFC1EB03
:102450000203C1EB0003411AB1F5804FA6BF9B03F5
:102460000131C3EB833393FBF1F0FEF793FAC0F332
:10247000C6100AF07BFD7C4B064618880AF076FDF4
:102480007A49804630460AF0C5FD014640460AF0CA
:10249000C1FD31460AF0B6FC4FF07E5106460AF007
:1024A00057FF002840F06886714930460AF06EFFF9
:1024B000002840F0378630460AF098FFC0B2DFF8B7
:1024C000CC8188F80000BAF17F0F40F3888462481D
:1024D000AAF17F0A80FB0A304FEAEA73C3EB60007F
:1024E00000EB4000AAEB80007330574B00931B7841
:1024F000C0B289F80000002B40F0E8835D4B0393E5
:102500001B78002B40F0B5855B4B02931B78002BAA
:1025100040F058864B4B0193029B1B78002B3AD01E
:10252000564B1B88182B17D099F800201344A3F1A1
:1025300018007F2840F3F985474A973B82FB032127
:10254000DA17C2EB610202EB4202A3EB820303F152
:102550007300C0B203F088FD494A4A4B127833F841
:102560001230182B17D099F800201344A3F118004B
:102570007F2840F3E485384A973B82FB0321DA1732
:10258000C2EB610202EB4202A3EB820303F1730090
:10259000C0B203F069FD009B1B78002B00F0B584EE
:1025A000019B284E1988002900F05C8538687F2837
:1025B00040F35783284B7F3883FB0032C317C3EBAC
:1025C000620303EB4303A0EB830073303860002900
:1025D00040F0F084009B1B78002B00F05D811B4EC7
:1025E0003378002B00F05881DFF864A0DFF89C807E
:1025F0004FF0000B0CE003F17300C0B298F800102C
:1026000003F00AFD33780BF1010B5B4540F3448185
:102610003B685AF8040F104A1844A0F17F0382FB6C
:102620000321DA17C2EB610202EB42027F28A3EB1F
:102630008203E0DCFEF710F8DFE700BFF69AFF1F29
:10264000989AFF1F249BFF1F449BFF1F3489FF1F85
:102650007489FF1FCC9AFF1FABAAAA2A589BFF1FA1
:10266000EC9AFF1F0A9CFF1F889AFF1FCDCCCC3D20
:102670000000FE42D29AFF1FA49AFF1FC29BFF1FB9
:10268000CC9BFF1FE09BFF1F7E9BFF1FDC9AFF1F61
:10269000A84B1960A84B1B68A92202FB03F3002B6F
:1026A000BCBF03F57F533F339B13543B194481F365
:1026B0000C01282007F0E0FCFFF7DCBA9F4EA04891
:1026C000A049A14A337003700B70137002E4934267
:1026D0004FF0000B6EDA0123CDF800B0CDF814B046
:1026E0000493FFF73EBB994B1B78002B7FF491AB13
:1026F000039B974A243B83F34703D9B25B201360C3
:1027000003F062FC98F80060032E30D1DFF890826D
:1027100098F80030002B40F03F868E4F3B78002B1E
:1027200040F02D86894E3378002B40F01B868A4B73
:102730001B78002B40F00986884A1380884B1B7851
:10274000002B40F0F585874B7F221A8098F80030E7
:102750006BB93B785BB933784BB9834A7F2107204B
:10276000138003F031FC7F210B2003F02DFC7F4B05
:102770001F68FFF74EBB7E480068D0F17F0048BF5E
:10278000033003EBA00301339942BFF6BDAC1160E7
:1027900080E7784B09881A6000297FF4F1AC134672
:1027A0009842D4BFC2EB0003C2EB030351E5FDF72F
:1027B00053FF39E60123CDF810B0CDF800B00593F2
:1027C000FFF7CFBA01232B606B4CFFF70DBA6B4BB1
:1027D0006A20198803F07CFD3B783370FFF704BA58
:1027E000564B1B78002B3AD0654B1B88182B17D003
:1027F00099F800201344A3F118007F2840F3F684D1
:10280000604A973B82FB0321DA17C2EB610202EBBD
:102810004202A3EB820303F17300C0B203F024FC75
:10282000594A5A4B127833F81230182B17D099F8AE
:1028300000201344A3F118007F2840F3DB84514AA1
:10284000973B82FB0321DA17C2EB610202EB4202E3
:10285000A3EB820303F17300C0B203F005FC019BFC
:102860001B88002B00F09584354B1B78002B40F023
:102870008A84474B3F4A198826680020012310604C
:102880002B60B1423C4CBFF6AFA92268414B089285
:10289000089A1A60FFF7A8B9039B1B78002B00F079
:1028A00083803B68A3F10C007F2840F3FA8335480E
:1028B0008B3B80FB0320DA17C2EB600000EB40008B
:1028C000A3EB800303F17300DFF8D080C0B298F867
:1028D000001003F0A1FB009B1B78002B64D02E4E50
:1028E0003378002B60D0DFF8BCA04FF0000B0BE07A
:1028F00003F17300C0B298F8001003F08DFB337839
:102900000BF1010B5B454FDD3B685AF8040F1D4A84
:102910001844A0F18B0382FB0321DA17C2EB61029A
:102920000C3802EB42027F28A3EB8203E0DCFDF7C8
:1029300093FEDFE7E09AFF1F7089FF1FA49AFF1F35
:10294000D09AFF1F449BFF1FD29AFF1FF09AFF1FD0
:10295000989BFF1FF99BFF1FF89BFF1F7C9BFF1F8E
:102960007A9BFF1F589BFF1F8C9AFF1F609BFF1FC6
:10297000909BFF1FEC9AFF1FF09CFF1FD49AFF1F34
:10298000C29BFF1FABAAAA2ACC9BFF1FE09BFF1F85
:10299000F69AFF1F989CFF1F3489FF1FDC9AFF1FC8
:1029A000F79BFF1F7489FF1F029B1B78002B3AD0F7
:1029B000AD4B1A88182A18D03B681344A3F11800AD
:1029C0007F2840F3B683A94A973B82FB0321DA179D
:1029D000C2EB610202EB4202A3EB820303F173003C
:1029E000A34BC0B2197803F017FBA2490B78022B56
:1029F00000F253830133DBB20B701A469E4830F865
:102A00001260182E40F090820422032B03F101067D
:102A1000F3B208BF002330F81360182E40F0838211
:102A2000013AF2D10B70019B1B88002B00F0CB8286
:102A3000009B1B783BB9039B1B7823B9029B1B7837
:102A4000002B00F0E0838D4B1B78002B00F0D6802C
:102A50008B490B78082B00F2D1808A483A680068CD
:102A6000894E0133DBB25F1E101A46F827000B7047
:102A7000864B2668198889F8002002E77F4B1B786F
:102A8000002B40F0C1823B68814A1278002A45D071
:102A9000A3F10C007F2840F30A83744A8B3B82FB2E
:102AA0000321DA17C2EB610202EB4202A3EB8203BD
:102AB00003F17300C0B298F8001003F0ADFA009B68
:102AC0001B7853B36E4E33783BB3DFF8FC91DFF8DD
:102AD0009CA14FF0000B0BE003F17300C0B298F81B
:102AE000001003F099FA33780BF1010B5B4514DD0C
:102AF0003B6859F8040F1844A0F18B038AFB0321AB
:102B0000DA17C2EB61020C3802EB42027F28A3EB1A
:102B10008203E1DCFDF7A0FDE0E73B685D4A127847
:102B2000002A3DD0504A1288182A18D01344A3F125
:102B300018007F2840F30D834C4A973B82FB03210A
:102B4000DA17C2EB610202EB4202A3EB820303F14C
:102B50007300C0B298F8001003F05EFA3B68454974
:102B60000A78022A00F2A6820132D2B20A70164610
:102B7000414830F816E0BEF1180F40F0F08104260D
:102B8000032A02F1010E5FFA8EF208BF002230F82C
:102B900012E0BEF1180F40F0E181013EF0D10A7061
:102BA000019A1288002A00F041823B4903220B70EF
:102BB0002A60FFF719B8394F3B78002B3FF499A9E9
:102BC000374E307801F0FCF8364B1B78002B00F0C4
:102BD000918233887E2B00F28D82334A0133108834
:102BE00099B23180002800F09582C9B2C0B22F4E50
:102BF00003F0EAF93B783370FEF7F6BF3A6837E73F
:102C0000DBB21846137003F0BDF9294B1B491A4675
:102C10001F4B184600230B703B7013700370FFF7B7
:102C200071B80123FFF7B0B880262249224B234A0E
:102C300009881B8812680B44B2EB630FBFF6E9A842
:102C4000164B1B78002B40F0FE81B9F800301C4A6F
:102C5000B3423FF4DEA81B4B168001221A70FFF727
:102C6000D8B8FDF7F9FCB1E4C29BFF1FABAAAA2AB2
:102C7000DC9AFF1FCC9BFF1FE09BFF1FD09AFF1F1A
:102C80003489FF1FAC9BFF1F7889FF1FF69AFF1F37
:102C9000D29AFF1FA49AFF1F7E9BFF1FFA9BFF1F64
:102CA000D49AFF1FF49AFF1FA69AFF1F1E9BFF1FB7
:102CB000449BFF1F2E9BFF1FC09BFF1F509BFF1FAE
:102CC000AA9AFF1F229BFF1F7489FF1FC14B01930C
:102CD0001B88002B40F06C83BF4B0393BF4B0293C8
:102CE000BF4E33786BB3DFF81483DFF8F8A24FF0F0
:102CF000000B09E003F17300C0B203F0B5F93378BB
:102D00000BF1010B5B451CDD58F8043F99F80000FE
:102D10001844A0F17F038AFB0321DA17C2EB61029A
:102D200002EB42027F28A3EB8203E3DCFDF794FC75
:102D3000E2E7AA4B029303F097F9009B1B78002B64
:102D4000CED1039B1B78002B3FF4E6AB99F8003003
:102D5000A3F10C007F2840F3A781A2488B3B80FBA6
:102D60000320DA17C2EB600000EB4000A3EB800306
:102D700003F17300C0B203F077F9009B1B78002BBE
:102D800000F08081964E3378002B00F06582DFF8EA
:102D90006C82DFF850A24FF0000B0AE003F17300E1
:102DA000C0B203F061F933780BF1010B5B457FF79B
:102DB000B3AB58F8043F99F800001844A0F18B0316
:102DC0008AFB0321DA17C2EB61020C3802EB4202E4
:102DD0007F28A3EB8203E1DCFDF73EFCE0E75046F1
:102DE000FDF73AFCFFF781BBFDF736FCFFF7DFB9D3
:102DF000002008707C49087840B17C49009109782E
:102E0000002900F0A981009F0021397078490978D4
:102E100000297FF443A8002E67D1002865D1754EA4
:102E2000724F96F800E06C4E03966C4E02966A4E16
:102E300071493070694E0097087038703070BEF17B
:102E4000000F7FF43DA8FFF744B8634B1B78002BBD
:102E50003FF4C6AC99F80030A3F10C007F2840F392
:102E6000C281604A8B3B82FB0321DA17C2EB61020D
:102E700002EB4202A3EB820303F17300C0B203F042
:102E8000F3F8009B1B78002B3FF4AAAC544E337828
:102E9000002B3FF4A5AC594FDFF848814FF0000AF2
:102EA0000AE003F17300C0B203F0DEF833780AF1F0
:102EB000010A53457FF794AC57F8043F99F8000096
:102EC0001844A0F18B0388FB0321DA17C2EB6102DF
:102ED0000C3802EB42027F28A3EB8203E1DCFDF712
:102EE000BBFBE0E703980021017042490978002903
:102EF0003EF4EFAF394902910978002900F088814A
:102F0000029800210170FEF7E4BF039B1B78002BA1
:102F10007FF446AB029B1B78002B7FF441AB019BF7
:102F20001988FFF743BB0B703B681E44A6F11800DD
:102F30007F2840F301812B4B973E83FB0632F3172A
:102F4000C3EB620303EB4303A6EB830606F17300B6
:102F50002B4BC0B2197803F05FF864E50A70734434
:102F6000A3F118007F2840F3F1801E4A973B82FBB3
:102F70000321DA17C2EB610202EB4202A3EB8203E8
:102F800003F17300C0B298F8001003F045F83B68F5
:102F900006E6243B002BB9F8000040F32F8198424D
:102FA0003EF40FAF9BB21748A9F80030012303701D
:102FB000FEF707BFDFF84880C0B298F8001003F0B2
:102FC0002BF8FFF707BB0E4B3878197803F024F87D
:102FD0002EE500BF249BFF1FD29AFF1FA49AFF1F5C
:102FE0003489FF1FABAAAA2A7A9BFF1F449BFF1FAD
:102FF000F79BFF1FFA9BFF1FD09AFF1F7489FF1FCB
:10300000DC9AFF1F229BFF1F7F21402002F0DCFF84
:10301000B349B44A3B680B600021117034E5C0B27B
:1030200098F8001002F0F8FFFFF7C8B8D8B298F887
:10303000001002F0F1FF3B68B7E5AB4BDFF8ECE2C4
:103040001978FEF7BEBE4B2E40F3A9801836802EAD
:10305000B9F80030A54AA8BF8026B3427FF4FBAD83
:10306000FEF7D7BE99F8000002F0FEFF3188FFF7A7
:103070009DBA9F4B01931B88002B7FF45AAE9D4B4A
:10308000029363E6029B1B78002B7FF449AA039B03
:103090001B78002B7FF484AA41E7002213460A70B4
:1030A000ACE4FDF7D9FA0FE4FDF7D6FA62E6FDF7D6
:1030B000D3FAFFE4002216460A7059E5FDF7CCFA70
:1030C000FFF767B98C4E307800F07AFE8B4B1B7897
:1030D0001BB133887E2B40F2A780894B1B7823B12C
:1030E0003388854A002B40F0AB80864E3B783370A6
:1030F000FEF77ABD824B1B78002BF6D033887E4AD0
:10310000002BF2D08049013B088899B21180002839
:103110007FF46BADC8B27B4E02F0CAFF3B783370D0
:10312000FEF762BD7F20FFF7CAB9FDF795FAFFF7FA
:1031300010BAFDF791FA53E4FDF78EFA08E7FDF7B0
:103140008BFAFFF725BA7F20FFF7B7B8FDF784FAAF
:1031500018E7FDF781FAFCE4664F6C4902974FF0DF
:10316000000C81F800C0009F02994FF0010E87F813
:1031700000E081F800C049E60120FFF7A0B902F0A5
:1031800073FFFFF70FB90021402002F01DFFFFF78A
:1031900070BB99F8000002F067FFFFF765BB243EA3
:1031A000002EB9F800303ADDB3423EF432AEB6B28A
:1031B000574BA9F8006001221A70FEF72ABE0120C1
:1031C000FFF77BB84A4B01931B88002B7FF4B3AD0C
:1031D000FFF7A2B94F4A8342A8BF03461360FEF728
:1031E000CFBF16462CE5FDF737FA47E6FDF734FA70
:1031F000FFF713BBFDF730FAFFF72EBB01283EF4B3
:10320000E0AD0123CFE699F8000002F02DFF1AE4AB
:103210004148009041483D490390FEF751BE012BC3
:103220003EF4F7AD0126C3E701339BB23380D9B238
:103230000520344E02F0C8FE3B783370FEF7D4BC54
:10324000013B9BB2D9B205202E4E138002F0BCFE8A
:103250003B783370FEF7C8BC029B1B78002B7FF4D1
:103260005FA9FFF79DB92E4B1B782BB32D4B1B7815
:10327000002B7EF4CEAD2C4B1B78002B3EF4C9AD59
:10328000B9F8003022490A33A9F800300A70FEF775
:10329000C0BD244B1B78002B7EF4BBAD224B1B78AA
:1032A000002B3EF4B6ADB9F800301949013BA9F83E
:1032B00000300A70FEF7ADBD1A4B1B78002B7FF46F
:1032C00012AA194B1B78002B3EF4A3ADB9F80030BD
:1032D0000F490133A9F800300A70FEF79ABD00BF0C
:1032E000AC9BFF1F3489FF1F419BFF1FAA9AFF1F42
:1032F000249BFF1FA49AFF1FD49AFF1FF49AFF1F5D
:103300007A9BFF1F1E9BFF1FA69AFF1FD09AFF1FCD
:10331000229BFF1FEC9AFF1F449BFF1FD29AFF1FA7
:10332000F89BFF1FF99BFF1FF09AFF1FDB9BFF1FFE
:10333000224B00227F2107201A8002F045FE7F21C8
:103340000B2002F041FEFFF701BA1D4B01227F2145
:1033500007201A8002F038FE7F210B2002F034FE95
:10336000FFF7ECB9174B04227F2107201A8002F0E7
:103370002BFE00210B2002F027FEFFF7D8B9114BDE
:1033800002227F2107201A8002F01EFE7F210B20DF
:1033900002F01AFEFFF7C6B90A4B002107201E8073
:1033A00002F012FE7F210B2002F00EFEFFF7B5B9EE
:1033B000054B0393054B0293BDE400BF589BFF1FD1
:1033C0007C9BFF1F8C9AFF1FD29AFF1FA49AFF1F9E
:1033D00038B506F067FB0B4804F09EFA00234FF067
:1033E0007E5201210848FDF741F8084B084A094977
:1033F000802400251C7118461D60BDE838400AF085
:1034000015B800BF949BFF1FFC9AFF1F349BFF1F42
:103410001C89FF1FFD05000043682A20198802F05F
:1034200057BF00BF10B5044622206368198802F018
:103430004FFFE36824201988BDE8104002F048BF20
:1034400010B504460A206368198802F041FFE3685A
:103450000C201988BDE8104002F03ABF10B50446B0
:1034600006206368198802F033FFE3680820198892
:10347000BDE8104002F02CBF10B50446022063687E
:10348000198802F025FFE36804201988BDE8104080
:1034900002F01EBF70B50E4C84B012250422012329
:1034A00006460390029320468DE824001423102141
:1034B00005F036FC06220923029303960195204667
:1034C00000921423102105F02BFC04B070BD00BF46
:1034D000249CFF1F2DE9F041224D82B0012602B24B
:1034E00084B20092284601967823192105F05EFBEC
:1034F00004F10C0212B28DE844002846A719782383
:10350000192104F1020805F051FB3FB20FFA88F8C7
:1035100019233A46284619460196CDF8008005F051
:1035200045FB78233A4628461946CDF80080019697
:1035300004F10A070B3405F039FB3FB224B27823BB
:103540003A46284619468DE8500005F02FFB19230E
:1035500000943A4601962846194605F027FB02B02A
:10356000BDE8F081249CFF1F2DE9F0411E4682B08A
:103570001446002A6AD0099B4D4A00EBC305012C72
:103580006F8929896868A7EB010382FB03E21A446B
:103590004FEAE373C3EBA21302887BD0042C38D12B
:1035A00012FA83F3994203DC9F423946A8BF1946B9
:1035B000089A0180B6F90030BDF920803D48971D7A
:1035C0004FF0000E3FB2194642460097CDF804E096
:1035D00005F0ECFA29896A896B68521A1B885C2A03
:1035E000A3EB010359DD03EB43030132C3EB4313A8
:1035F00093FBF2F303F11B0213B201203280194650
:103600004246019000972B4805F0D0FA2A4B002241
:103610001A702A4B022CB3F9001045D0082C31D176
:1036200000221A8091422DD0089AB6F90030214824
:103630000632012412B2009219460194BDF92020ED
:1036400005F0B4FA204602B0BDE8F0811C4D1D4AD9
:103650002B681268CB1A93420F4617D9164A338843
:1036600011781448012918BF01241470089A0632F1
:103670001BB212B28DE814001946BDF9202005F0E6
:1036800095FA2F60012002B0BDE8F081204602B01B
:10369000BDE8F0819BB2D31A84E75C2101FB03F300
:1036A00093FBF2F21B32A7E74A1C12B21A80B9E769
:1036B000C94216B2249CFF1F9D9CFF1F169CFF1F32
:1036C000989CFF1FD4ED000030B583B000230C465A
:1036D00005B2009326225B231C210C4804F0B6FFA0
:1036E000294601232622094804F0C0FA002C24B2FE
:1036F00005DB214601232622044804F0B7FA044AD8
:10370000044B15801C8003B030BD00BF249CFF1FFC
:10371000AE89FF1FB089FF1F70B5944C237882B02B
:103720001BB1934B4FF6FF721A80924BB3F90030E6
:10373000C3B9914A8E4B1068B3F9002080F30C0096
:103740005B2303FB00F000131C3082425AD04FF081
:10375000FF31FFF7B9FF894804F0DCFF0023237035
:1037600002B070BD012B32D0022B6AD0032B4FD098
:10377000042BF3D1272200258DE8240076231C2179
:103780007E487F4E05F012FA17E0B0F5AF7FA8BF74
:103790004FF4AF70323803FB00F386FB0321DB17D5
:1037A000C3EB61111C3109B201231D442722734868
:1037B00004F05CFA0C2D00F08180E9B2714804F04D
:1037C00013F931284FF05B03DFDC1C21ECE76E4B73
:1037D0001A68B2F52F7F32DB41F25C239342A8BF17
:1037E0001346A3F52F735B22684802FB03F380FBAB
:1037F0000320DB17C3EBA0201C305D4BB3F9003076
:103800008342A4D1624BB3F9003001339FD1A5E7C5
:10381000604B1B68B3F5FA7F11DBB3F57A6FA8BF75
:103820004FF47A63A3F5FA725B485B2303FB02F360
:1038300080FB0320DB17C3EB20201C30DDE71C20BE
:10384000DBE7564B1B68B3F5FA7F33DBB3F57A6FD2
:10385000A8BF4FF47A63A3F5FA724F485B2303FBCA
:1038600002F380FB0320DB17C3EB20201C304C4B02
:103870001B68B3F5FA7F1FDBB3F57A6FA8BF4FF46F
:103880007A63A3F5FA7244495B2303FB02F381FBDD
:103890000321DB17C3EB21211C31354BB3F9003079
:1038A00083427FF456AF3A4BB3F900308B427FF43A
:1038B00050AF53E71C20DAE71C21EEE7012006F0A9
:1038C00099FF6FF495733238364A03FB00F082FBA0
:1038D0000023C017C0EB632303F5AF73312B3ADD30
:1038E000B3F5AF7FA8BF4FF4AF735B22323B244DDB
:1038F00002FB03F385FB0325DB17C3EB65151C35C2
:10390000002006F077FF6FF495733238254A03FBE9
:1039100000F082FB0023C017C0EB632303F5AF73F5
:10392000312B1ADDB3F5AF7FA8BF4FF4AF735B2225
:10393000323B134902FB03F381FB0321DB17C3EB8B
:1039400061111C310A4BB3F90030AB4207D0284655
:10395000FFF7BAFEFFE61C25D2E71C21F2E70C4B6D
:10396000B3F900308B42F2D1F5E600BF0C9CFF1F8B
:10397000AE89FF1F129CFF1F909AFF1F249CFF1F00
:103980004B48371B949BFF1FD09BFF1FD3058541DE
:10399000B089FF1F509BFF1F011FB812849AFF1FA1
:1039A0004C9BFF1F67BBCF462DE9F04FDFF8EC8241
:1039B000B74CB8F900604D7854F8264087B082467D
:1039C000039305B10D78DFF8FCB2002A34D19BF8DF
:1039D00000308BBBAF4EB6F90000002800F0CE805F
:1039E000012800F02481012032232A46019000930F
:1039F0005146A94B2046FFF7B7FD00250746B6F90B
:103A00000030022B40F3F48000233380B8F90030FB
:103A1000A24A002BC0F2F880042BC4BF00231380FD
:103A2000039B002B40F0F680002D0CBF38464FF072
:103A3000FF3007B0BDE8F08F964EE36822689848E3
:103A400004930027059237808BF8007004F056FD30
:103A50001120FFF73FFD4FF0010919232821CDF870
:103A600004900091242219468D4805F09FF8782390
:103A700028212422CDF8049000918948194605F0A8
:103A800095F84946864805F027FC0222192184480A
:103A900005F01EFCDDF8149048460AF091FA4946FC
:103AA00002467F4805F0AEFD7D4805F0C1FD394670
:103AB00014227B4805F00CFC03227A49784805F073
:103AC000A1FD774805F0B4FD39462322744805F07E
:103AD000FFFB03227449724805F094FD704805F01D
:103AE000A7FD049B002B72D10123704A1846137066
:103AF000FFF7D0FC208963896768191A5C293A8826
:103B00005BDC131A5C2202FB03F292FBF1F31B3322
:103B1000674A6348138001271BB21A2219468DE8B1
:103B20008400142205F042F8049BDBB1218A638AE9
:103B3000E768581A5C283A886FDD521A02EB420295
:103B4000C2EB4212431C92FBF3F31B33524A54481C
:103B50001380012738221BB28DE8840019463222D7
:103B600005F024F8534A544BB6F9000001211170B6
:103B70004FF6FF721A8000287FF432AFDFF84891C9
:103B80004E4AD9F800301268C3EB0A0393424CD96D
:103B9000464B1A78012A18BF012018700127FFF739
:103BA00079FCC9F800A0012D4ED0042D59D0022D6A
:103BB00060D0082D64D0002521E7121A02EB4202E2
:103BC000C2EB42124B1C92FBF3F31B33A0E72F20F6
:103BD000FFF780FC39463222314805F079FB032299
:103BE00037492F4805F00EFD2D4805F021FD7BE7F4
:103BF0007FF40CAFE368002B3FF406AFB8F9003058
:103C0000264A002BBFF608AF04231380039B002B2A
:103C10003FF40AAFFFF780FD06E7511A5C2202FB72
:103C200001F292FBF0F31B3390E70746BBE7002756
:103C300014238DE888002A4651461D4B2046FFF785
:103C400093FC3D460746DAE6B8F800308BF80050A2
:103C50000133A8F80030636983B1002520469847F6
:103C6000CDE6B8F800300122013BA8F800308BF80F
:103C70000020F0E7012333800025C7E61D46BEE69D
:103C80006369002232804FF0FF35002BE6D1BDE69C
:103C9000B489FF1F169CFF1F109CFF1F129CFF1F63
:103CA000249CFF1F98E700009CE700009D9CFF1FDD
:103CB0000E9CFF1F0C9CFF1FAE89FF1FD4ED000060
:103CC000A0E70000149CFF1F989CFF1F01210D20FE
:103CD00006F062BB00210D2006F05EBB01460D2000
:103CE00006F05ABB08B50D2006F05CFBB0FA80F177
:103CF00049090D20BDE8084006F04EBB10B5002173
:103D000044080D2006F048FB204606F081FB0D20FC
:103D1000012106F041FB2046BDE8104006F078BBCB
:103D200008B5214A214B12881868824234DA204BA8
:103D30001B88991A8342A8BF0346B1F5F87FA3EB0D
:103D4000020321DAC3EB031303EB431393FBF1F1FB
:103D500005310A2006F090F9164B1978F1B1164B8F
:103D600016491B6883F30703C3EB031303EB4313E9
:103D700081FB03211944DB17C3EBA1110531092095
:103D8000BDE8084006F078B9C3EB43131B010131CD
:103D900093FBF1F10531DCE70021DAE70920BDE80A
:103DA000084006F069B900BFF69AFF1FEC9AFF1FA2
:103DB0000A9CFF1FC49BFF1F909BFF1F09040281E9
:103DC0007F2838B5A8BF7F200D4D4FF4FA7303FB51
:103DD00000F485FB04232344E117C1EBA3110A205F
:103DE00006F04AF9A4F578400C3885FB003101440F
:103DF000C017A0EBA111BDE83840092006F03CB97E
:103E000009040281024B4E20198802F061BA00BFFA
:103E1000249BFF1F024B4420198802F059BA00BFAF
:103E2000C29BFF1F024B1020198802F051BA00BF3D
:103E3000429BFF1F024B2C20198802F049BA00BF99
:103E40006A9BFF1F024B1E20198802F041BA00BF77
:103E50003E9BFF1FC3680E20198802F039BA00BFCD
:103E6000024B2820198802F033BA00BF209BFF1FA5
:103E7000024B6220198802F02BBA00BF5C9BFF1F27
:103E8000024B6420198802F023BA00BF669BFF1F13
:103E9000024B5A20198802F01BBA00BF9A9AFF1FE2
:103EA000024B1620198802F013BA00BF589BFF1F5F
:103EB000024B2E20198802F00BBA00BF809BFF1F17
:103EC000024B3020198802F003BA00BF889AFF1F06
:103ED000024B1820198802F0FBB900BF2C9BFF1F72
:103EE000024B1A20198802F0F3B900BF8E9BFF1F06
:103EF000024B1C20198802F0EBB900BFBA9BFF1FD0
:103F0000024B6620198802F0E3B900BF789AFF1FC0
:103F1000024B2020198802F0DBB900BF089CFF1F6C
:103F2000024B3220198802F0D3B900BFF89AFF1F64
:103F3000024B6820198802F0CBB900BFA69AFF1F78
:103F4000024B5220198802F0C3B900BFAC89FF1F91
:103F5000024B5020198802F0BBB900BF7489FF1FC3
:103F6000024B5420198802F0B3B900BF9C89FF1F8F
:103F7000024B5C20198802F0ABB900BF7689FF1FA5
:103F8000024B5E20198802F0A3B900BFA489FF1F6D
:103F9000024B6020198802F09BB900BF8A9AFF1F6C
:103FA000024B5620198802F093B900BF069CFF1FF0
:103FB00038B5094D4624204602F0A4F935F8021B15
:103FC00000B28842204601D002F082F90234A4B245
:103FD0004E2CF0D138BD00BFE09BFF1F064B074AB7
:103FE00010B41C88064B0846002C14BF1146194615
:103FF000042210BC0AF0A2B8BC9BFF1FC8EE000050
:10400000CCEE0000064B074A10B41C88064B08464D
:10401000002C14BF11461946042210BC0AF08EB8B9
:104020001C9BFF1FC8EE0000CCEE0000064B074AA9
:1040300010B41C88064B0846002C14BF11461946C4
:10404000042210BC0AF07AB8B09AFF1FC8EE000034
:10405000CCEE0000064B074A10B41C88064B0846FD
:10406000002C14BF11461946042210BC0AF066B891
:104070008C9BFF1FC8EE0000CCEE0000064B074AE9
:1040800010B41C88064B0846002C14BF1146194674
:10409000042210BC0AF052B8BE9BFF1FC8EE0000FD
:1040A000CCEE0000064B074A10B41C88064B0846AD
:1040B000002C14BF11461946042210BC0AF03EB869
:1040C000FC9BFF1FC8EE0000CCEE0000064B074A29
:1040D00010B41C88064B0846002C14BF1146194624
:1040E000042210BC0AF02AB87C9BFF1FC8EE000017
:1040F000CCEE000070B5284E05460FCE86B06C465B
:104100000FC496E8030044F8040B2320218005F037
:104110002DFC40F6B833984230DC204B40F6F502D7
:1041200019889B78ADF80D1090428DF80F302DDD79
:1041300000EB40001A4B1B491B4E00EB0010C2174E
:1041400083FB0043C2EB632381FB0314D917C1EB4C
:10415000A40101EB810186FB0040C2EB6030A3EBC0
:104160004103303030338DF811008DF8133069463B
:104170002846162209F0E2FF06B070BD0B4B1A88E4
:104180009B78ADF80D208DF80F30D1E7084B1868FB
:10419000CDF81100EBE700BFE0EE0000D0EE00002C
:1041A000976A3E2B676666668BAA3045DCEE000098
:1041B000D4EE0000F8B5174C174E2278174D33781F
:1041C0002F888E46003218BF012201467046FFF745
:1041D000EBFB002398423370237015DB14BF0120E2
:1041E00000202B889F420ED040F23A72A3F5AF73A5
:1041F0000B490C4C02FB03F381FB0312DB17A3EB0F
:10420000621332332360F8BD0749012218460A7051
:104210002270E6E7608BFF1FBA9CFF1F689BFF1FA1
:10422000B5814E1BA089FF1F1C9CFF1F014B1878F6
:1042300001F0E6BFB09CFF1F014B187801F0FABFF8
:10424000E48CFF1F134BB3F9003030B583EAE374FD
:10425000A4EBE374002BA0B218DB012300E01346AB
:1042600003EB830252009442F9DA0B4D90FBF3F218
:1042700085FB03E403FB1200DB173032D3EBA4030E
:1042800080B201F8012BF1D10B7030BD2D230B70E2
:104290000131E2E7E48CFF1F67666666144BB3F9F1
:1042A000003070B583EAE375A5EBE375002BACB283
:1042B0001ADB012300E0034603EB83004000854244
:1042C000F9DA0C4E94FBF3F086FB03E503FB104494
:1042D000DB173030D3EBA503A4B201F8010BF1D109
:1042E00005480B70106070BD2D230B700131E0E7A5
:1042F0009A9AFF1F67666666F8EE0000134BB3F9E3
:10430000003030B583EAE374A4EBE374002BA0B271
:1043100018DB012300E0134603EB830252009442B2
:10432000F9DA0B4D90FBF3F285FB03E403FB12007B
:10433000DB173032D3EBA40380B201F8012BF1D1AB
:104340000B7030BD2D230B700131E2E7AC89FF1FEC
:1043500067666666134BB3F9003030B583EAE374E1
:10436000A4EBE374002BA0B218DB012300E013469A
:1043700003EB830252009442F9DA0B4D90FBF3F207
:1043800085FB03E403FB1200DB173032D3EBA403FD
:1043900080B201F8012BF1D10B7030BD2D230B70D1
:1043A0000131E2E77489FF1F67666666134BB3F954
:1043B000003030B583EAE374A4EBE374002BA0B2C1
:1043C00018DB012300E0134603EB83025200944202
:1043D000F9DA0B4D90FBF3F285FB03E403FB1200CB
:1043E000DB173032D3EBA40380B201F8012BF1D1FB
:1043F0000B7030BD2D230B700131E2E79C89FF1F4C
:1044000067666666134BB3F9003030B583EAE37430
:10441000A4EBE374002BA0B218DB012300E01346E9
:1044200003EB830252009442F9DA0B4D90FBF3F256
:1044300085FB03E403FB1200DB173032D3EBA4034C
:1044400080B201F8012BF1D10B7030BD2D230B7020
:104450000131E2E77689FF1F67666666134BB3F9A1
:10446000003030B583EAE374A4EBE374002BA0B210
:1044700018DB012300E0134603EB83025200944251
:10448000F9DA0B4D90FBF3F285FB03E403FB12001A
:10449000DB173032D3EBA40380B201F8012BF1D14A
:1044A0000B7030BD2D230B700131E2E7A489FF1F93
:1044B00067666666054B1B881BB9054B1868086064
:1044C0007047044B18680860704700BF249BFF1FAB
:1044D00000EF0000FCEE0000164B1B880BB31BB274
:1044E00030B583EAE374A4EBE374002BA0B21CDBC9
:1044F000012300E0134603EB830252009442F9DAF1
:104500000D4D90FBF3F285FB03E403FB1200DB1778
:104510003032D3EBA40380B201F8012BF1D10B7040
:1045200030BD064B1868086070472D230B700131B1
:10453000DEE700BF3E9BFF1F67666666CCEE0000AD
:10454000164B1B880BB31BB230B583EAE374A4EBA4
:10455000E374002BA0B21CDB012300E0134603EB45
:10456000830252009442F9DA0D4D90FBF3F285FB81
:1045700003E403FB1200DB173032D3EBA40380B259
:1045800001F8012BF1D10B7030BD064B18680860A3
:1045900070472D230B700131DEE700BF889BFF1FA2
:1045A00067666666CCEE0000164B1B880BB31BB229
:1045B00030B583EAE374A4EBE374002BA0B21CDBF8
:1045C000012300E0134603EB830252009442F9DA20
:1045D0000D4D90FBF3F285FB03E403FB1200DB17A8
:1045E0003032D3EBA40380B201F8012BF1D10B7070
:1045F00030BD064B1868086070472D230B700131E1
:10460000DEE700BF589BFF1F6766666604EF000089
:10461000174B1B881BB31BB270B583EAE375A5EB80
:10462000E375002BACB21EDB012300E0034603EB75
:10463000830040008542F9DA0E4E94FBF3F086FBCE
:1046400003E503FB1044DB173030D3EBA503A4B222
:1046500001F8010BF1D108480B70106070BD074BD9
:104660001868086070472D230B700131DCE700BF2C
:10467000809BFF1F67666666D8EE0000CCEE0000E8
:10468000164B1B880BB31BB230B583EAE374A4EB63
:10469000E374002BA0B21CDB012300E0134603EB04
:1046A000830252009442F9DA0D4D90FBF3F285FB40
:1046B00003E403FB1200DB173032D3EBA40380B218
:1046C00001F8012BF1D10B7030BD064B1868086062
:1046D00070472D230B700131DEE700BF889AFF1F62
:1046E00067666666CCEE0000164B1B880BB31BB2E8
:1046F00030B583EAE374A4EBE374002BA0B21CDBB7
:10470000012300E0134603EB830252009442F9DADE
:104710000D4D90FBF3F285FB03E403FB1200DB1766
:104720003032D3EBA40380B201F8012BF1D10B702E
:1047300030BD064B1868086070472D230B7001319F
:10474000DEE700BF789AFF1F67666666CCEE000062
:10475000174B1B881BB31BB270B583EAE375A5EB3F
:10476000E375002BACB21EDB012300E0034603EB34
:10477000830040008542F9DA0E4E94FBF3F086FB8D
:1047800003E503FB1044DB173030D3EBA503A4B2E1
:1047900001F8010BF1D108480B70106070BD074B98
:1047A0001868086070472D230B700131DCE700BFEB
:1047B000089CFF1F6766666608EF0000CCEE0000ED
:1047C000074B1B88022B06D0012B0CBF054B064B59
:1047D000186808607047054B18680860704700BF8C
:1047E0008A9AFF1F10EF000014EF00000CEF00008A
:1047F000054B1B881BB1054B186808607047044BBC
:1048000018680860704700BF069CFF1F1CEF00007F
:1048100018EF000038B5FDF75FF80D4B1B7833B982
:104820000C4B1020198801F053FD012038BD0A4DB2
:104830000A4C2B782288B3FA83F382F008025B09D2
:10484000114642202B70228001F042FD002038BD2D
:10485000FA9BFF1F429BFF1FD89BFF1FBC9AFF1FA5
:10486000184B1A8852B3184A128830B50A80B3F927
:104870000030002B83EAE374A4EBE374BCBF2D2368
:104880008B70A0B2ACBF02310331012300E01346AC
:1048900003EB830252009442F9DA0C4D90FBF3F2E1
:1048A00085FB03E403FB1200DB173032D3EBA403D8
:1048B00080B201F8012BF1D10B7030BD044B1868A8
:1048C000086070478E9BFF1F20EF000067666666DA
:1048D000CCEE000010B40A4B0A4C0A4693E80300E1
:1048E00083B0238802AC04E9030004EB8303104681
:1048F00053F8081C052203B010BC09F01FBC00BF10
:1049000028E80000669BFF1FF0B40C4D0C4F0E46CC
:104910000FCD8CB001AC0FC40FCD0FC495E80700CC
:104920003B8884E807000CAA02EB8303304653F867
:104930002C1C04220CB0F0BC09F000BC30E80000D4
:104940008C9AFF1FF0B40A4D0A4F0E460FCD86B069
:1049500001AC0FC42A683B88226006AA02EB8303DD
:10496000304653F8141C042206B0F0BC09F0E6BB34
:104970005CE800002C9BFF1FF0B40A4D0A4F0E4666
:104980000FCD86B001AC0FC42A683B88226006AA0E
:1049900002EB8303304653F8141C0C2206B0F0BC23
:1049A00009F0CCBB70E80000BA9BFF1F164B1B88B8
:1049B0000BB31BB283EAE370A0EBE370002B30B5BE
:1049C00084B21DDB012300E0134603EB8302520097
:1049D0009042F9DA0D4894FBF3F280FB03E503FB08
:1049E0001244DB173032D3EBA503A4B201F8012B3C
:1049F000F1D10B7030BD08460422054909F09EBB79
:104A00002D230B700131DDE7A69AFF1F67666666EE
:104A100024EF000070B53C4D2B780646002B35D1B5
:104A20001C4673780BB9204670BDFCF755FF374A1A
:104A3000374B3848127831781B78007802EB430303
:104A40004A1E03EB80030E2AEDD801A050F822F095
:104A5000B94A0000DB4A0000274A0000B94A0000BA
:104A6000274A0000274A0000274A0000A74A000002
:104A7000274A0000274A0000274A0000274A000072
:104A8000274A0000274A0000A34A0000AE2122481E
:104A900003F0E4FA204803F031FD00232B700124D9
:104AA000BFE705F0C7FFAF211B4803F0D7FA1B4A49
:104AB000012313702B70B6E783B9194803880429C2
:104AC0004FF6FF7103F1FF320CBF01230B46134475
:104AD00003F07F03013303800FE073B1013B114A00
:104AE00032F813304BB10E4E0F481049104A338044
:104AF0000123002606700B701370084A022101235F
:104B000011702B70204670BD608BFF1F7A9BFF1FBA
:104B1000F49AFF1F049CFF1F249CFF1F1C9CFF1F77
:104B2000AA9AFF1F6C9BFF1FD99BFF1F229BFF1F91
:104B3000909CFF1F10B5064B064C1A882046012199
:104B400001F0B4FB21884220BDE8104001F0C0BB59
:104B5000BC9BFF1FBC9AFF1F10B5064B064C1A8862
:104B60002046022101F0A2FB21884220BDE810402E
:104B700001F0AEBB1C9BFF1FBC9AFF1F10B5064B7C
:104B8000064C1A882046042101F090FB218842201F
:104B9000BDE8104001F09CBBB09AFF1FBC9AFF1FFC
:104BA00010B5064B064C1A882046052101F07EFB05
:104BB00021884220BDE8104001F08ABB8C9BFF1F7A
:104BC000BC9AFF1F10B5064B064C1A8820460621DA
:104BD00001F06CFB21884220BDE8104001F078BB59
:104BE000BE9BFF1FBC9AFF1F10B5064B064C1A88D0
:104BF0002046002101F05AFB21884220BDE81040E8
:104C000001F066BBFC9BFF1FBC9AFF1F08B512207A
:104C100001F078FB054B1988884206D0122001F07C
:104C200057FBBDE8084001F06BBA08BD8C9AFF1F26
:104C300008B5582001F066FB054B1988884206D05C
:104C4000582001F045FBBDE8084001F059BA08BD05
:104C5000889BFF1F08B5142001F054FB054B1988F1
:104C6000884206D0142001F033FBBDE8084001F073
:104C700047BA08BD7C9BFF1FF0B480EAE075A5EB46
:104C8000E0750028ACB21FDB1DBF2B230B704E1C40
:104C90000E46012300E0134603EB830252009542C7
:104CA000F9DA0B4F94FBF3F287FB030503FB124485
:104CB000DB173032D3EBA503A4B206F8012BF1D1F8
:104CC00033700846F0BC70472D230B704E1CE0E794
:104CD00067666666144B18880C2811D0192813D003
:104CE0001A2815D01B2817D01C2819D01D2803D02E
:104CF0000C3800B2FFF7C0BF0C4A1068086070475C
:104D00000B4A1068086070470A4A106808607047CC
:104D1000094A106808607047084A106808607047C0
:104D2000074A106808607047F89AFF1F40EF0000BC
:104D30002CEF000030EF000034EF000038EF0000EF
:104D40003CEF0000034B1888A0EB8000400000B24D
:104D5000FFF792BFB09CFF1F024BB3F90000FFF7B3
:104D60008BBF00BF5C9BFF1F024B1888033800B24B
:104D7000FFF782BF209BFF1F024B18880C3800B240
:104D8000FFF77ABFCE9BFF1F024B1888183800B27E
:104D9000FFF772BFC29BFF1FC3681888183800B2A4
:104DA000FFF76ABF30B5134C85B001252B463C2276
:104DB00002212046009503F0C7F9204603F09EFB30
:104DC00000224021802320460191009311460A4B86
:104DD000029504F041F8204603F09CFC074808497E
:104DE000084A0023036083800B608B8013609380EC
:104DF00005B030BD249CFF1FD8E80000889CFF1F31
:104E0000B49CFF1FA09CFF1F10B500EBC00000F179
:104E10000F02D2B293B284B09C1E981C3D23039122
:104E20008DE819003921024803F07AFF04B010BD63
:104E3000249CFF1F014B01221A707047BA9CFF1F70
:104E4000F0B585B05E4C5F4B02935F4A019204233C
:104E5000009320465D4B5E4F5E4E5F4D40228021A9
:104E600002F07AFF20465D4C5D4A5E4908F0DEFAAA
:104E7000A7615D485D4FE7615D4F87615D495E4FAA
:104E8000C7615E4F8F615E4A5E4FCF615E4F976133
:104E90005E4B5F4FD7615F4F9F615F4FDF615F4F39
:104EA000B7615F4FF7615F4FAF615F4C5F4FEF617D
:104EB0005F4FA7615F48604FE761604F876160495E
:104EC000604FC761604F614A8F61614FCF61614F31
:104ED000614B9761614FD761614F624E9F61624F35
:104EE000DF61624F624DB761624FF761624F634CA1
:104EF000AF61634FEF61634F6348A761634FE76141
:104F0000634F64498761644FC761644F8F61644A2E
:104F1000644FCF61644F9761644B654FD761654FB4
:104F20009F61654E654FDF61654FB761654D664FA7
:104F3000F761664FAF61664C664FEF61664FA761E0
:104F40006648674FE761674F87616749674FC76189
:104F5000674F8F61674A684FCF61684F9761684BB1
:104F6000684FD761684F9F61684E694FDF61694F35
:104F7000694DB761694FF761694F6A4CAF616A4F1C
:104F80006A486B49EF616B4F6B4DA761E5616B4FF1
:104F90006B4D6C4CDFF8D0E16B4A6C4B8761C5619F
:104FA0008C61C1F81CE06A4E6A4F6B4D6B4C6C48CB
:104FB0006C499761D5619C61D861B16005B0F0BD65
:104FC000249CFF1FA0860100801A06005C8FFF1F33
:104FD000794D00009C8CFF1F348AFF1FC08CFF1F7F
:104FE0001C89FF1FB17D00003C8BFF1F553E000058
:104FF000694D0000EC89FF1F613E0000DD3F0000AD
:10500000548DFF1F354B0000054000008C8BFF1FA7
:10501000594B00002D4000007D4B00005540000022
:10502000A14B0000594D0000F48AFF1F713E0000A3
:105030007D4000006C8EFF1FC54B0000D54800006E
:10504000D88EFF1F813E0000A5400000108AFF1F80
:10505000E94B0000454D0000E88CFF1F2D42000089
:1050600045420000048EFF1F39420000094900003C
:10507000EC8BFF1F0D4C000041450000AC8AFF1F68
:10508000314C00009D420000648AFF1F913E0000E9
:10509000CD400000208FFF1F554C0000A9450000A7
:1050A000108CFF1FA13E000011460000888AFF1FE0
:1050B000B13E000081460000B08BFF1FC13E0000E2
:1050C00045490000188BFF1FD13E000061480000D9
:1050D000308DFF1FE13E000079490000908EFF1FD8
:1050E000F13E0000E9460000588CFF1F013F000020
:1050F00051470000288EFF1F113F0000D54C0000D3
:10510000B48EFF1F213F0000AD490000D08AFF1F71
:10511000313F0000FD420000348CFF1F413F000082
:1051200055430000C889FF1F513F0000BC8DFF1F81
:10513000E08DFF1FAD430000613F0000054400000B
:10514000713F00005D440000FC8EFF1F0C8DFF1FAF
:10515000588AFF1FC1470000913F0000F14700003F
:10516000A13F0000D9540000813F00002DE9F04F1D
:105170002F4DDFF8CCB0DFF8C4A0DFF8C8900FCD1A
:1051800091B003AC0FC40FCD0FC40FCD0FC42B686B
:1051900023600025A8462F462E4600E09846BAF820
:1051A000003024495BF8232028461123FBF7DCFB61
:1051B00000EBC00400EB840089FB00340444C017FA
:1051C000C0EB6434C4F13C00C6F13C0207F141017C
:1051D000012600B208F1410300901BB2019612B201
:1051E00009B2154803F0E2FC08EB060305F21115BD
:1051F0003C2B2646ADB24746D0D134226B210E4817
:1052000004F066F800210C4804F066F80B4B1B888C
:1052100010AA02EB830353F8344C204608F0D0FE6A
:1052200002460548214611B0BDE8F04F04F0EAB946
:1052300098E8000044E50000249CFF1F6A9BFF1FC4
:1052400088E60000090002802DE9F043804685B021
:10525000002956D10121304804F03EF82F4998F832
:10526000062098F8083011F80290994522DA4FEAA2
:1052700089064D460C24D8F80C3027489B595F68A6
:1052800022B2002104F024F8384608F099FE39468D
:105290000246214804F0B6F91F4804F0C9F998F80D
:1052A000083001350934AB42A4B206F1040601DD31
:1052B000422CE0D1B9F1000F13D109F1060999454B
:1052C0000CDA3C2301213B220391029300930192CB
:1052D00039233F223A21104803F022FD05B0BDE8F2
:1052E000F0830F2301213B2203910293009301924B
:1052F00039230C223A21084803F012FD98F80830AF
:10530000DBE700213423009301913F230C22024864
:1053100003F01AFC9EE700BF249CFF1FB49CFF1FF4
:1053200010B5104C0121204603F0DCFF204601217E
:1053300003F0D2FF20463422552103F0C9FF204656
:105340000222094904F05EF920460522074904F0CB
:1053500059F9204604F06CF92046BDE8104003F0EE
:10536000D9B900BF249CFF1F44EF000048EF0000A4
:1053700070B50D46064608F023FE00EB40008400A1
:10538000002D36D0284608F01BFE00EB4000400000
:1053900023185B1003F16001091A282209B217488B
:1053A000C3F1600403F094FF0121144803F094FF5B
:1053B000284608F005FE29460246104804F022F966
:1053C0000E4804F035F902210C4803F085FF21B2A4
:1053D00021220A4803F07CFF304608F0F1FD3146F7
:1053E0000246064804F00EF90448BDE8704004F097
:1053F0001FB96410C4F16004E5E700BF249CFF1FDF
:10540000214B70B5B3F9003083EAE374A4EBE37485
:10541000002B82B0A1B22FDB68466D46012300E06D
:10542000134603EB830252009442F9DA174E91FBC4
:10543000F3F286FB03E403FB1211DB173032D3EBEC
:10544000A40389B205F8012BF1D119462B70FFF79F
:105450008FFF0F4B1B786BB101210E4803F03CFF0F
:10546000332274210B4803F033FF01220A49094813
:1054700004F0C8F802B070BD2D238DF800300DF196
:1054800001056846CAE700BF429BFF1F6766666664
:10549000D89BFF1F249CFF1F48F2000010B50D4B46
:1054A0001B5C51F82340237884B013B1012004B071
:1054B00010BD04AA01A942F8103D2046A3699847EF
:1054C000A38A9B07F2D401A80099FFF751FF01209E
:1054D00004B010BD889CFF1FF8B51F4D287840B957
:1054E0001E4B1B68994203D31D4A012313702B7076
:1054F000F8BD0C4600261B48184F02F0FFFF04F6CB
:10550000B833324617483B6031212E7003F0E0FE7D
:105510000121144803F0E6FE3146124803F0DCFE98
:10552000052211490F4804F06DF80E4804F080F888
:105530000C2210210B4803F0CBFE0B220B4909482B
:1055400004F060F805220A49064804F05BF80548B3
:1055500004F06EF80120F8BD608BFF1F849CFF1FD4
:105560001C9CFF1F249CFF1F50EF000058EF000001
:1055700048EF000010B5424C424882B002F0BEFF36
:105580002378C3B906213F4803F0A6FE2378012BF8
:1055900037D90A22022B11463A486BD003F098FE05
:1055A00039490322374804F02DF8364802B0BDE8E7
:1055B000104004F03DB8354B1A7801210523002A2C
:1055C00035D10191009311462E4803F03FFB304B3B
:1055D0001A78002A36D00523012201920093002276
:1055E0000A21284803F0B0FA2A4B1A78002A35D14C
:1055F00001210523019100931421224803F026FB89
:10560000C0E7254C2388092B32D9632B8CBF0A2194
:105610001F210A221B4803F05BFE2188194804F071
:1056200057F8184802B0BDE8104004F001B8002255
:10563000019100931146134803F086FA144B1A782F
:10564000002AC8D105230121019100930A210D48A8
:1056500003F0FCFA0F4B1A78002AC9D00122052367
:105660000192009300221421064803F06DFA89E7A5
:105670003021CEE703F02CFE0322084992E700BF59
:10568000909CFF1F249CFF1F68EF00007A9BFF1F68
:10569000F49AFF1F049CFF1FAA9AFF1F64EF0000EB
:1056A0002DE9F041754C2278002A05460F4614BFBB
:1056B0004FF001084FF000084ED1714E3368CB1AFD
:1056C000B3F5FA6F04D86B78A3B94046BDE8F08112
:1056D0006C4B6D486D49DFF8D0E11A7001230370FF
:1056E0000988237026208EF8002000F0F1FD6B78E9
:1056F000002BEAD03760FCF7EFF8654A654B664946
:10570000127828781B78097802EB4303421E03EBDA
:1057100081030E2AD9D801A151F822F00D580000BA
:10572000D9570000CB5600000D580000CB560000A2
:10573000CB560000CB560000C1570000CB560000EE
:1057400073570000CB560000CB560000CB5600002C
:10575000CB5600006F570000AF215048484E02F072
:105760007DFCFFF707FF002337602370ABE705F0F0
:1057700061F94A4802F0C2FE0221484803F0ACFD3C
:105780000F222321454803F0A3FD05224449434845
:1057900003F038FF414803F04BFF1E2223213F480E
:1057A00003F096FD05223F493C4803F02BFF3B48A0
:1057B00003F03EFF394802F0ADFF00F0ADFC84E796
:1057C000394D2B78012B50D9304B2620198800F009
:1057D0007FFD00232B7078E7002B3FF476AF013B71
:1057E000324A32F81330002B3FF46FAF274C304869
:1057F00025492D4A23804FF001080023037081F8CA
:10580000008082F80080FFF7B5FE5EE793B1013BB0
:10581000264A32F8131019B31C4B254D1A4C224A54
:1058200019800026012326202E702370137000F0AB
:105830004FFD15E0154C1E4922880B7004284FF6C9
:10584000FF7002F1FF310CBF012202460A440E4EE6
:10585000154D02F07F0201320121228031702B7040
:10586000FFF788FE4FF001082FE70649064A01239B
:105870000020087013702370A6E700BF608BFF1F25
:10588000AC9CFF1F1C9CFF1F229BFF1FAA9AFF1F9F
:105890007A9BFF1FF49AFF1F049CFF1F249CFF1F8D
:1058A0006CEF000074EF0000909CFF1F6C9BFF1FCB
:1058B000D99BFF1F2DE9F04F05468BB00F46AD4831
:1058C0000121164603F00EFDAA8812F0010440F0F3
:1058D000B080DFF8CC8298F80030002B7DD1AB7916
:1058E000A54AD15CA1B9DFF8BCA279781AF8039077
:1058F00041B339780139072900F2B780DFE811F0A8
:10590000F1005401B5006C01B500B500B500E90027
:105910007C78002C00F0CA800139EC68387854F8A3
:105920002170FC68411EB4F80080072900F2A780AE
:10593000DFE811F074015901A5006C01A500A50074
:10594000A5009F00DFF854A2DAF80020B21AB2F5E1
:10595000967F75D9894A107801281ABF01201070E6
:105960001170874A18BF0146D05CC0EB0900C0B275
:10597000FFF74AFA0124CAF80060AB889B0770D58C
:105980007B78002B6DD0FBF7A7FF7E4B7E4A7F48CC
:105990001B78127839780078022515FB02330A2922
:1059A00003EB800300F04E810C295AD1002B58D014
:1059B00003F11900764E774A013B0021400080B286
:1059C00026F813100123157088F8003000F080FCD1
:1059D000714B032220461A702FE0664802F08EFDBC
:1059E0000121644803F078FC62482246214603F016
:1059F0006FFCAB88580725D42C68204608F0E0FAE5
:105A0000214602465B4803F0FDFD5A4803F010FEB4
:105A1000092201238DE80C0000217F23554803F063
:105A2000C5F800212846FFF70FFC002388F8003056
:105A300055E7AB683146384698470BB0BDE8F08F64
:105A40000846FAE72B6804A8984704A808F0B8FAB3
:105A500004A90246474803F0D5FD464803F0E8FD97
:105A6000D6E720460BB0BDE8F08F00240AF803907B
:105A700083E70021D1543846FB699847FC68A4F8B5
:105A80000080002725223C238DE884004121182234
:105A9000384803F059F8E968A879FFF7FFFC374A5E
:105AA0003E4B17701E600BB0BDE8F08F3B490A6893
:105AB000B21AB2F5967FD4D9304F0E603E78012EDF
:105AC00000F0B480E968184601233B70FFF7E6FC5C
:105AD000B3E7304AE9791170012288F800200024E8
:105AE000C4E72A7A013A4A45BFDD09F10104E4B26C
:105AF000A145BAD0224E16F803B0CBEB0900C0B2D4
:105B00000021FFF781F92B7A052BD9461BD9CBEB66
:105B10000402042A40F3AE80A4F1040BBBF1000F91
:105B2000C0F2B080063B5B45A8BF5B465FFA83F9D5
:105B3000AA791348B15C994205D000F8029001217E
:105B40002846FFF781FBC9EB0400C0B201210B4ED0
:105B5000FFF75AF900213423019100930548317071
:105B600040230B223F21A14602F0EEFF0124AB7936
:105B70007CE700BF249CFF1FA09CFF1F9D9CFF1F74
:105B8000B49CFF1F7A9BFF1FF49AFF1F049CFF1F0A
:105B90006C9BFF1F1C9CFF1F909CFF1F989CFF1F6E
:105BA000608BFF1F889CFF1F0FFA89F1E868604C2B
:105BB00050F821602168049134785E4904980860A7
:105BC000002C71D0012C7FF450AF5B4A317A88F8F9
:105BD00000401170002449E7B9F1000F50D009F1DD
:105BE000FF34E4B284E7B98A01F0040189B20029E4
:105BF0003FF440AF3B6A03929847039A00283FF472
:105C00003DAFAB79FC680021D15438E77B8A43452E
:105C10003CD908F101081FFA88F830E73B8A434570
:105C20003BD208F1FF381FFA88F828E725238DE8D2
:105C3000180042483C703C231822412102F084FFA6
:105C40003046FAE6002B3FF40CAF3D4A3D4E11883A
:105C5000394A03F11900013B400080B226F81310C5
:105C6000012388F80030157000F032FB364B2046D7
:105C70001D70E2E6002A3FF755AF04F1FF3B4DE708
:105C80004C46F3E64FF000094B4651E7BB8ADA0772
:105C90007FF5F5AEB7F81080F1E6BB8AD9077FF53E
:105CA000EEAEB7F81280EAE62849C85CC0EB0900FE
:105CB00009F1010EC0B201214FF0340B02F803E0EC
:105CC000FFF7A2F8B6681D48019440230B223F213C
:105CD0000124CDF800B002F037FF40230B223F2112
:105CE0001648CDF800B0019402F0B0FF21461348E9
:105CF00003F0F2FA304608F063F9A0EB800000F1FF
:105D00005F0109B20F220D4803F0E2FA304608F0B5
:105D100057F931460246094803F074FC074803F07E
:105D200087FCE968A879FFF7B9FBAB799EE600BF6D
:105D3000F09CFF1F989CFF1F1C9CFF1F249CFF1FB3
:105D4000AA9AFF1F6C9BFF1F909CFF1FB49CFF1F14
:105D50002DE9F047DFF808926D4B99F800601B6859
:105D6000DFF800A282B0003601934FF0030018BFA5
:105D70000126019F9AF8008004F014FB05460420D8
:105D800004F010FB0446052004F00CFB800040EA00
:105D90004404062004F006FB2C4364B25D4944EA47
:105DA000C0000A7880F00F03DBB29A425A4A3CD016
:105DB0001760002259480B7003788DF800808DF829
:105DC000012053B3564A12684EF66021BA1A8A422D
:105DD00019D8022B59D0012B5FD0062B48D0032BAA
:105DE00063D0042B69D0052B77D0072B7DD0082BEF
:105DF00000F08380092B68D016B14A4802F08AFC73
:105E000002B0BDE8F087484A484C002301212370C6
:105E100003701360938089F800103A46694644483D
:105E2000FFF748FD3043C6B2E6E71268BA1A1E2AE9
:105E30006BD99AF80020934222D0394C3D488AF819
:105E40000030012B276082EA030207609846B1D038
:105E5000042BAFD137480068381AB0F5C87FA9D9EC
:105E6000354C2068381A3228A4D927601A46A1E791
:105E70003A4669463148FFF71DFD3043C6B2BBE7DD
:105E8000012B4FF00002E3D1E4E73A4669462C4883
:105E9000FFF710FD3043C6B2AEE73A4669462948DF
:105EA000FFF708FD3043C6B2A6E73A4669462648E2
:105EB000FFF700FD3043C6B29EE73A4669462348E5
:105EC000FFF7F8FC3043C6B296E73A4669462048E9
:105ED000FFF7F0FC3043C6B28EE73A4669461D48EC
:105EE000FFF7E8FC3043C6B286E73A4669461A48EF
:105EF000FFF7E0FC3043C6B27EE73A4669461748F2
:105F0000FFF7D8FC3043C6B276E7002252E700BF65
:105F1000F09CFF1F9C9CFF1F189CFF1F1C9CFF1FD9
:105F2000949CFF1F249CFF1FA09CFF1F8E9CFF1FA3
:105F3000ACEE0000A89CFF1F209CFF1FE8ED0000B6
:105F4000F8ED0000D8ED000098ED000020EE000014
:105F500004EE0000B8EE000054EE0000588AFF1F67
:105F6000608BFF1F8F9CFF1F28B11028044BA8BF18
:105F7000102018607047024B01201860704700BF66
:105F8000BC9CFF1F38B50F4D2B78013B01381B021D
:105F9000C4B203F47063200443F4404343F00C03A1
:105FA00000F4FE00184305F065FB2868013860F036
:105FB0003F00C0B204F08CFB2046BDE8384004F03E
:105FC00087BB00BFBC9CFF1F70B5124D2B78013BF7
:105FD0001B0203F47063064643F4304308063204A0
:105FE00000F0FE4043F00B03034302F4FE001843AD
:105FF0000C4605F03FFB2868013860F04F00C0B246
:1060000004F066FB304604F063FB2046BDE87040B8
:1060100004F05EBBBC9CFF1F70B5124D2B78013B9A
:106020001B0203F47063064643F41043080632046F
:1060300000F0FE4043F00903034302F4FE0018435E
:106040000C4605F017FB2868013860F06F00C0B2FD
:1060500004F03EFB304604F03BFB2046BDE87040B8
:1060600004F036BBBC9CFF1F38B5104D2B78013BAC
:106070001B0203F47063044643F41043000443F02E
:10608000090300F4FE00184305F0F4FA286801380B
:1060900060F06F00C0B204F01BFB204604F018FB58
:1060A0000020BDE8384004F013BB00BFBC9CFF1FBC
:1060B00038B50E4D2B78013B1B0203F47063044688
:1060C00043F45043000443F00D0300F4FE00184372
:1060D00005F0D0FA2868013860F02F00C0B204F053
:1060E000F7FA2046BDE8384004F0F2BABC9CFF1F26
:1060F00008B5002005F088FB0028FAD108BD00BFD4
:1061000008B564210720FFF75FFF7F210B20BDE862
:106110000840FFF759BF00BF10B500217B20FFF7F3
:1061200053FF0024E0B2FFF79FFF0134022004F088
:106130006FF9802CF6D110BD10B504464FF44060C5
:1061400004F076FA04F0CEFA2CB1102C044BA8BF60
:1061500010241C6010BD024B01241C6010BD00BF48
:10616000BC9CFF1F10B5044641F0E00004F0B0FAFB
:1061700004F07F0004F0ACFAC4F3C610BDE8104090
:1061800004F0A6BA38B5134D2B78044641F6FF72D9
:10619000A0F50050824203F1FF33A8BF02461B0264
:1061A00002F5005203F47063100443F4604343F0BB
:1061B0000E0300F4FE005204184302F0FE421043A6
:1061C00005F058FA296801392046C9B2BDE83840BF
:1061D000FFF7C8BFBC9CFF1F38B504460D46F02032
:1061E00004F076FA35B1254414F8010B04F070FA86
:1061F000AC42F9D1F720BDE8384004F069BA00BFDD
:1062000000B50B4B83B00246998818680090032AAA
:10621000ADF8041002D903B05DF804FB684606210E
:106220008DF80520FFF7D8FF03B05DF804FB00BF31
:10623000A0F2000000B50B4B024683B018689988A5
:106240000090131F4C2BADF8041002D903B05DF879
:1062500004FB684606218DF80520FFF7BDFF03B05B
:106260005DF804FBA8F20000030203F4FE43C0F350
:10627000C6101843704700BF03784078DB0103F471
:106280007E5300F07F001843704700BF82B002AA1F
:10629000114642F8040D002012F8013B03F07F0381
:1062A000914243EA0020F7D102B07047003210B4A7
:1062B00003884FF0010404FA01F418BF012202FA26
:1062C00001F123EA04020A43028010BC704700BFB8
:1062D00070B5CEB20C46054603F02CFC864203D0C6
:1062E0003146284603F040FC0135284603F022FCE5
:1062F000240A844205D021462846BDE8704003F0B8
:1063000033BC70BD38B5054603F014FC4FF00004F3
:1063100060F30704681C03F00DFC60F30F24A0B2C7
:1063200038BD00BFF8B504460020FFF7EBFF002C96
:1063300000F0FD804FF4AF610220FFF7C9FF042099
:106340004FF47A61FFF7C4FF0B2004F02BF800280C
:1063500040F0B4844FF496610620FFF7B9FF4FF484
:10636000FA610820FFF7B4FF4FF4AF610A20FFF78E
:10637000AFFF40F6FC010C20FFF7AAFF4FF4966137
:106380002220FFF7A5FF4FF416612420FFF7A0FF9E
:106390007D212A20FFF79CFF0C210E20FFF798FF9C
:1063A00001211020FFF794FF02211220FFF790FF38
:1063B00000211420FFF78CFF00211620FFF788FF33
:1063C00002211820FFF784FF01211A20FFF780FF28
:1063D00002211C20FFF77CFF04211E20FFF778FF1D
:1063E00014212020FFF774FF01212620FFF770FF02
:1063F00003212820FFF76CFF04212C20FFF768FF02
:106400000F212E20FFF764FF00213020FFF760FFEF
:106410000C213220FFF75CFF00213420FFF758FFEA
:1064200000213620FFF754FF00213820FFF750FFEE
:1064300000213A20FFF74CFF00213C20FFF748FFE6
:1064400000213E20FFF744FF00214020FFF740FFDE
:1064500000214220FFF73CFF1F214420FFF738FFB7
:1064600013214620FFF734FF0E214820FFF730FFAD
:1064700011214A20FFF72CFF0A214C20FFF728FFAB
:1064800000214E20FFF724FF06215020FFF720FFB8
:1064900002215220FFF71CFF0C215420FFF718FFA8
:1064A00000215620FFF714FF00215820FFF710FFAE
:1064B00001215A20FFF70CFF03215C20FFF708FFA2
:1064C0000A215E20FFF704FF00216020FFF700FF94
:1064D00004216220FFF7FCFE01216420FFF7F8FE93
:1064E00000216620FFF7F4FE0B216820FFF7F0FE85
:1064F0007F216A20FFF7ECFE00216C20FFF7E8FE09
:1065000000216E20FFF7E4FE22210020FFF7E0FECD
:106510000220FFF7F7FEB0F5805F034616D34FF475
:10652000AF610220FFF7D4FE4FF4AF630EE04FF6E9
:10653000FF7398423FF4FEAE222840F0CB83022046
:10654000FFF7E0FEB0F5805F0346E8D2D24A0420B0
:106550001380FFF7D7FEB0F5805F034680F0CF824F
:10656000CE4A06201380FFF7CDFEA0F52F739BB215
:10657000B3F57A6F024606D940F628210620FFF7C8
:10658000A7FE40F62822C64B08201A80FFF7BAFE65
:10659000A0F52F739BB2B3F57A6F024606D940F689
:1065A000E4410820FFF794FE40F6E442BD4B0A2088
:1065B0001A80FFF7A7FEA0F5FA739BB240F6AC5124
:1065C0008B42024606D94FF4AF610A20FFF780FEE6
:1065D0004FF4AF62B44B0C201A80FFF793FEA0F586
:1065E000FA739BB240F6AC518B42024606D940F694
:1065F000FC010C20FFF76CFE40F6FC02AB4B0E20BA
:106600001A80FFF77FFE1828034600F26682A84A28
:1066100010201380FFF776FE431E9BB20F2B02461D
:1066200004D901211020FFF753FE0122A14B1220B3
:106630001A80FFF767FE0A28034600F248829E4A46
:1066400014201380FFF75EFE0128034604D90021C1
:106650001420FFF73DFE0023984A16201380FFF711
:1066600051FE7F28034600F22C82954A18201380A1
:10667000FFF748FE0428034600F21D82914A1A20C3
:106680001380FFF73FFE0C28034600F282828E4AF9
:106690001C201380FFF736FE0428034600F27382A5
:1066A0008A4A1E201380FFF72DFE0928034600F2B8
:1066B0006482874A20201380FFF724FE4628034681
:1066C00000F25582834A22201380FFF71BFEA0F5BB
:1066D000FA739BB240F6AC518B42024606D94FF496
:1066E00096612220FFF7F4FD4FF496627A4B242046
:1066F0001A80FFF707FEA0F5FA739BB240F6AC5183
:106700008B42024606D94FF416612420FFF7E0FDC4
:106710004FF41662714B26201A80FFF7F3FD7F2895
:10672000034600F21E826E4A28201380FFF7EAFD1E
:106730000628034600F20F826A4A2A201380FFF7D8
:10674000E1FDA0F132039BB2B3F5967F024604D976
:106750007D212A20FFF7BCFD7D22634B2C201A806F
:10676000FFF7D0FD0C28034600F2EF815F4A2E2090
:106770001380FFF7C7FD1E28034600F2E0815C4A44
:1067800030201380FFF7BEFD0928034600F29082F7
:10679000584A32201380FFF7B5FD1D28034600F24A
:1067A0005282554A34201380FFF7ACFD7F28034600
:1067B00000F24382514C36202380FFF7A3FD7F284F
:1067C000034600F2348238206380FFF79BFD7F2868
:1067D000034600F226823A20A380FFF793FD7F282C
:1067E000034600F218823C20E380FFF78BFD7F28F0
:1067F000034600F20A823E202381FFF783FD7F28B3
:10680000034600F2FC8140206381FFF77BFD7F2877
:10681000034600F2EE814220A381FFF773FD384D5D
:1068200028804420FFF76EFD3028034600F2DB810C
:10683000344A46201380FFF765FD3028034600F2F6
:10684000CC81314C48202380FFF75CFD3028034683
:1068500000F2BD814A206380FFF754FD30280346D3
:1068600000F2AF814C20A380FFF74CFD3028034697
:1068700000F2A1814E20E380FFF744FD012803468A
:1068800004D900214E20FFF723FD00231F4A50208A
:106890001380FFF737FD3BE0F69AFF1F0A9CFF1FAE
:1068A000A09BFF1FF29AFF1FF49BFF1F649BFF1F1B
:1068B000CE9BFF1F429BFF1F8C9AFF1F7C9BFF1FDD
:1068C000589BFF1F2C9BFF1F8E9BFF1FBA9BFF1F18
:1068D0003E9BFF1F089CFF1FC09BFF1F2E9BFF1F9F
:1068E000AA9AFF1F209BFF1F689BFF1F6A9BFF1F29
:1068F000809BFF1F889AFF1FF89AFF1F6C9BFF1F4A
:10690000BC9AFF1FC29BFF1FE09BFF1F249BFF1F22
:10691000431E9BB20B2B024604D906215020FFF7E1
:10692000D7FC0622CB4B52201A80FFF7EBFC042841
:10693000034600F23A81C84A54201380FFF7E2FC74
:10694000431E9BB21D2B024604D90C215420FFF795
:10695000BFFC0C22C14B56201A80FFF7D3FC012844
:10696000034604D900215620FFF7B2FC0023BC4A9D
:1069700058201380FFF7C6FC7F28034600F20F81E2
:10698000B84A5A201380FFF7BDFC431E9BB2092B67
:10699000024604D901215A20FFF79AFC0122B24B8A
:1069A0005C201A80FFF7AEFC431E9BB2102B024600
:1069B00004D903215C20FFF78BFC0322AB4B5E2044
:1069C0001A80FFF79FFC431E9BB21D2B024604D981
:1069D0000A215E20FFF77CFC0A22A54B60201A806A
:1069E000FFF790FC022803467DD8A24A642013805A
:1069F000FFF788FC0128034604D901216420FFF732
:106A000067FC01239C4A62201380FFF77BFCC31EB6
:106A10009BB2012B024604D904216220FFF758FCE7
:106A20000422964B66201A80FFF76CFC7F280346F1
:106A30007FD8934A68201380FFF764FC7F280346C1
:106A400071D8904A6A201380FFF75CFC7F280346C8
:106A500063D88D4A6C201380FFF754FC042803464A
:106A600055D88A4A6E201380FFF74CFC192840D86D
:106A70002B88DFF838E2864F864A874D874E884C50
:106A8000884903F0010CAEF800C0C3F3400EA7F82C
:106A900000E0C3F380071780C3F3C007824A2F705A
:106AA000C3F30017C3F34015C3F380133780258069
:106AB0000B801080F8BD02211820FFF709FC02238B
:106AC000DCE500211620FFF703FC0023CDE50221C1
:106AD0001220FFF7FDFB0223B1E50C210E20FFF78A
:106AE000F7FB0C2393E500216020FFF7F1FB002367
:106AF0007BE76E200021FFF7EBFB0020B8E74FF4A7
:106B00007A610420FFF7E4FB4FF47A6328E5002163
:106B10006C20FFF7DDFB0023A3E77F216A20FFF74E
:106B2000D7FB7F2395E70B216820FFF7D1FB0B23D1
:106B300087E700216620FFF7CBFB002379E70F21D1
:106B40002E20FFF7C5FB0F2319E604212C20FFF7A9
:106B5000BFFB04230AE603212820FFF7B9FB032328
:106B6000EAE501212620FFF7B3FB0123DBE5142131
:106B70002020FFF7ADFB1423A4E504211E20FFF71E
:106B8000A7FB042395E502211C20FFF7A1FB0223AC
:106B900086E501211A20FFF79BFB012377E5002101
:106BA0005820FFF795FB0023EAE602215220FFF769
:106BB0008FFB0223BFE60A214C20FFF789FB0A2343
:106BC00058E611214A20FFF783FB11234AE60E21E4
:106BD0004820FFF77DFB0E233CE613214620FFF7FC
:106BE00077FB13232DE61F214420FFF771FB1F23A2
:106BF0001EE600214020FFF76BFB00230BE600217F
:106C00003E20FFF765FB0023FDE500213C20FFF758
:106C10005FFB0023EFE500213A20FFF759FB00233B
:106C2000E1E500213820FFF753FB0023D3E50021E5
:106C30003620FFF74DFB0023C5E500213420FFF788
:106C400047FB0023B6E50C213220FFF741FB0C2364
:106C5000A7E500BF7489FF1FAC89FF1F9C89FF1F38
:106C6000069CFF1F889BFF1F9A9AFF1F7689FF1FB4
:106C7000A489FF1F8A9AFF1F669BFF1F5C9BFF1F53
:106C8000789AFF1FA69AFF1FD49AFF1F5A9BFF1FD7
:106C9000BC9BFF1F1C9BFF1FD89BFF1FB09AFF1FB1
:106CA0008C9BFF1FBE9BFF1FA89AFF1FFC9BFF1F13
:106CB00000213020FFF70CFB002369E540F6282176
:106CC0000620FFF705FB40F6E4410820FFF700FB34
:106CD000FFF74ABB17287FF62DAB19287FF69CAB30
:106CE0001B287FF6B9AB1C283FF4CEAB1E287FF6DD
:106CF000D3AB1F283FF4D8AB20283FF4F1AB2128B9
:106D00007FF402ACFFF7F8BBF8B5812006F0C8FBB2
:106D1000204B214A054603CB1368C5F803001A0C23
:106D20007020C5F807102B80AA70FFF79DFA2E4639
:106D3000002426F80B0FA0B2FFF7E4FAFFF794FA4D
:106D40000234702C26F8020FF5D16C1E05F17C067A
:106D50004FF0FF3014F8013F082758400F4B40F325
:106D600000017A1E0B4012F0FF0783EA5000F5D1B4
:106D7000B442EFD1C043FFF789FA3A46C5F87D0027
:106D80008121284604F0C4FC2846BDE8F84006F0FE
:106D90008FBB00BFB4F20000B0F200002083B8ED5A
:106DA000F0B50E4B0E4C054693E8070085B02468FD
:106DB0002E88AD7801AB83E80700270C1846002227
:106DC0000B21ADF804408DF80670ADF80C608DF81D
:106DD0000E5004F09DFC05B0F0BD00BFC0F20000F5
:106DE000B0F20000F0B5124B124D1E68124F0FCDDD
:106DF00087B06C460FC495E8030044F8040B38686C
:106E00003B79CDF80D00320C222021808DF8022034
:106E10008DF81130ADF80060FFF726FA0022ADF8CA
:106E20000B001221684604F073FC07B0F0BD00BFF0
:106E3000B0F20000CCF2000048EF0000002004F0A7
:106E4000E3BC00BF02F02EBE70B5124C82B000252C
:106E500040230646294620460093019580232022A0
:106E600001F072FE20222946204602F031FA204627
:106E7000012102F037FA304607F0A2F83146024607
:106E8000204602F0BFFB204602B0BDE8704001F092
:106E900041BC00BF249CFF1FF0B5802983B075D989
:106EA0000546441E00F17C064FF0FF3014F8012F18
:106EB00008275040404A40F300017B1E0A4013F06F
:106EC000FF0782EA5000F5D1B442EFD1C043FFF78B
:106ED000DDF90146D5F87D000190019A914202D07A
:106EE000B2F17F2F0BD105F10B00FFF7C5F9702828
:106EF0000BD03248FFF7A8FF002003B0F0BD3048A8
:106F0000FFF7A2FF384603B0F0BD05F10D00FFF713
:106F1000B3F9222840D1002440F6AC5613E00428EF
:106F20001AD0062821D008281FD00A2828D00C28DB
:106F300022D1A1F5FA7292B2B24201D8FFF7C8F994
:106F40000234702C0ED004F10D002844FFF794F9A0
:106F5000022C0146A0B2E2D1B1F5805FEED302343B
:106F6000702CF0D1012003B0F0BDA1F52F7292B2C8
:106F7000B2F57A6FE4D8E1E7222801D0242811D1B4
:106F8000A1F5FA7292B2B242DAD8D7E70D48FFF70C
:106F90005BFF002003B0F0BD0B48FFF755FF00205A
:106FA00003B0F0BD2A28C9D1A1F1320292B2B2F5E4
:106FB000967FC5D8C2E700BF2083B8ED10F300006C
:106FC000FCF20000E4F2000024F3000003290CD9D5
:106FD00070B5461C82B005460C46304603222A494D
:106FE00007F05CF810B102B070BD70470B2C05D9EA
:106FF00005222649281D07F051F840B12448FFF723
:1070000023FF244802B0BDE87040FFF7C9BE05F178
:107010000901032201A807F091F801A803221E49E3
:1070200007F03CF8D8B103221C4901A807F036F854
:1070300008B301A803221A4907F030F8B0B919487B
:10704000FFF702FFA11E89B23046FFF725FF002897
:10705000C9D0154802B0BDE87040FFF7F5BE13482F
:10706000FFF7F2FEFFF750FE1148F3E71148FFF774
:10707000EBFE1148C6E71148FFF7E6FE02B0BDE897
:107080007040FFF7AFBE00BFB0F2000050EF00004D
:107090003CF3000050F3000054F300007CF30000C8
:1070A00094F3000098F30000ACF3000058F30000E4
:1070B0006CF30000C0F30000D4F3000080F3000084
:1070C0002DE9F043174D2B6883B081460F4690465B
:1070D000F3B1154E34880A1992B21846114632801F
:1070E00006F05CFD28603A464946204402F06CFDFB
:1070F000B8F1000F09D031882868FFF767FF2868CA
:1071000006F0D6F900232B60338003B0BDE8F0838E
:10711000054E01930846318006F0C2F9019B2860B4
:107120001C46E0E7C49CFF1FC09CFF1F10B51F4C0E
:107130004FF4FA70FCF7E2FD204601F0DFF900227F
:107140001146204602F0C4F82046012102F0CAF898
:107150002046002102F0C0F80B221549204602F01B
:1071600051FA204602F064FA0F221249204602F03A
:1071700049FA204602F05CFA0F490722204602F045
:1071800041FA204602F054FA204601F0C3FA0B4BB4
:107190000B4A1A604FF4FA70FCF7B0FDFFF722FEBD
:1071A0000848BDE81040FFF74FBE00BF249CFF1FFA
:1071B000D8F30000E4F30000F4F300007C9EFF1F0E
:1071C000C1700000FCF300000020704790F83920E7
:1071D00090F83800101A704790F8383090F839203D
:1071E0009A4205D95A1C034480F83820187E70470B
:1071F0004FF0FF30704700BF90F8383090F83920DA
:107200009A4286BF1B18187E4FF0FF30704700BFB0
:10721000704700BF38B50546B0F85E0090B195F8EC
:107220005D301446C3F1210294420CD805F13B00B5
:107230001844224602F0C8FC95F85D30234485F8D6
:107240005D30204638BD012014462871EEE700BFAE
:10725000B0F85E306BB190F85D30202B07D8C218C3
:10726000013380F85D30012082F83B107047012324
:1072700003710020704700BF0023426980F8383056
:1072800080F8393080F85C3080F85D3080F85E300E
:1072900080F85F3006CA30B40D68046943662A433B
:1072A00083660A60A370426990F8613016491468D9
:1072B00013441D7A5B7B01EBC5051B026D6803F46B
:1072C000E06343F064032B6090F8623013449D7CCC
:1072D000DB7D01EBC5011B02496803F4E06343F069
:1072E00064030B6021685368194205D003692722A3
:1072F0005A70036904229A71036920225A71036942
:1073000080229A7030BC704730FF000043690CCB7C
:1073100012681A420CD0094B99420AD9084B99427B
:10732000036994BF1A220D225A70036904229A71CC
:107330007047036927225A70F7E700BF7F1A0600DB
:107340003F420F0010B50269D378DBB2D90604467C
:107350003DD510215806D17038D503F0040303F051
:10736000FF02002B51D03D49626E00230B7084F860
:107370005D30002A5BD0904794F85D30002B56D0EA
:107380002369D0229A70236994F83B201A712369EB
:10739000012284F85C200222DA7010BD304B84F8A0
:1073A00060009C424AD02F4B9C4252D094F8391036
:1073B00013791F29DBB207D82848007820B160185C
:1073C000013184F8391003760223D37010BD5906B9
:1073D000C3D4917801F0100101F0FF000029DDD045
:1073E00013F001031ED194F85C1094F85D008842FC
:1073F00081BF4B1C091984F85C3091F83B30137144
:107400002369D0229A702269DEE7236984F8392043
:10741000C0229A702369114A197901211170022240
:10742000DA7010BDC023937022691379CCE7012272
:10743000002384F85D2084F83B30A1E7626994F86A
:107440006130094913440322187A02F043FD22698E
:10745000ACE7626994F861300449F3E7C89CFF1F08
:107460005C8FFF1FC88FFF1FCD740000D974000010
:107470000369DB7803F0200373B190F860300133C7
:10748000DBB2012B80F860301AD9426990F8613084
:107490001344187A02F09ABD70B5426903F0FF05F3
:1074A00090F8613013440446187A02F08FFDA36E01
:1074B0005BB184F8385094F83900BDE87040184743
:1074C00090F85F30002BE0D0704770BD0148FFF7A7
:1074D000CFBF00BF5C8FFF1F0148FFF7C9BF00BFD0
:1074E000C88FFF1F2DE9F047374FDFF8E0903B686A
:1074F000026982B006460093DDF800800021A025D5
:10750000D3789B065BD53B680193019BC8EB0303D3
:107510000F2BF5D949B1102BF2D0002090703369B0
:1075200080229A7002B0BDE8F087726996F86130E7
:1075300013440521187A02F043FF726996F861300E
:107540001344012193F812A0504602F039FF092498
:107550000021504602F020FF2B46013BFDD10121C6
:10756000504602F019FF2B46013BFDD1013CEFD103
:10757000706996F8611001444FF4A0720C7A4B7B4D
:1075800009EBC4011B02496803F4E06343F06403A0
:107590000B6096F862300344997CDB7D09EBC101F6
:1075A0001B02496803F4E06343F064030B60013A93
:1075B000FDD13269D3789B064FF00101A3D401209D
:1075C00002B0BDE8F08700BFF09CFF1F30FF000055
:1075D000F0B503691222DA700269937803F0200390
:1075E00085B004460D46002B5ED0B42393703C4911
:1075F00022690B680093009E05E00B680193019BD4
:107600009B1B042B42D8D37803F0200303F0FF0028
:10761000002BF2D094F85D30002B31D04FF0000EEB
:107620004FF0020C04EB0E0393F83B3013710B6820
:107630000393039F206907E09B060DD50B68029317
:10764000029BDB1B052B28D8C378DBB203F00202B8
:1076500002F0FF06002AEFD080F803C02669F37815
:10766000DBB2DF0632462DD49F062BD5DB0731D4A3
:107670000EF1010E94F85D305FFA8EFE7345D1D89D
:1076800000201DBB002384F85E3004E09070236965
:1076900080229A70042005B0F0BD86702369802294
:1076A00004209A7005B0F0BD03F0FF06FFF71AFF43
:1076B00010B9042005B0F0BD236984F85F60B022E2
:1076C0009A7094E78023B3700420DAE72669802358
:1076D000B370D7E7BEF1000F0CBF02200320F6E71E
:1076E000F09CFF1F2DE9F04106690025122780F864
:1076F000385080F83950F770D0F810C09CF802E08C
:107700000EF0200E88B00446884615461E46BEF18F
:10771000000F49D0B4238CF80230784B21691A68E5
:107720000092DDF800E006E01A6801920198CEEBC5
:107730000000042830D8C87800F0200000F0FF07CF
:107740000028F1D04FEA480242F00102D2B20A7199
:107750001A680292DDF808E0206906E01A680392D0
:107760000399CEEB010105292AD8C17801F0020165
:1077700001F0FF070029F1D04FF0020C80F803C0A0
:107780002269D17811F0110722D12DBB002E0CBF38
:10779000A0238023937003E08F70236980229A7066
:1077A000384608B0BDE8F0810EF0FF07FFF79AFEFB
:1077B0000028F5D0236984F85F70B0229A70ACE796
:1077C00087702369802238469A7008B0BDE8F0813E
:1077D000802393700027E3E7012D75D0A0219170DD
:1077E00021690A79BE4667464FF0A80C1A680492D0
:1077F000049805E01A680592059A121A052A4AD8D3
:10780000CA7802F0020202F0FF08002AF2D0CF701C
:107810002169CA78D2B212F0100F08465AD19206E6
:1078200058D5013DEDB2012D49D0BEF11F0F3BD916
:107830000A79012DDAD11A680692069D05E01A68C8
:107840000792079A521B052A46D8C27802F0020214
:1078500002F0FF01002AF2D00223C3702269D3781C
:10786000DBB2D9063AD49B0634D5B023BEF11F0F44
:1078700093703FD8226904EB0E0312791A760EF149
:10788000010E5FFA8EFE16B1236980229A7084F889
:1078900039E0774684E781F80280236980229A7074
:1078A000774684F839E07BE704EB0E0291F8048018
:1078B00082F818800EF1010E5FFA8EFEB9E781F8AA
:1078C00002C021690846B0E7A82191702069BE4630
:1078D0000279B0E7774663E78170DEE71021A023E5
:1078E000D170013BFDD12269937803F0F70377460D
:1078F000937055E723691B79C5E700BFF09CFF1F14
:107900000148FFF71FBD00BF5C8FFF1F0148FFF755
:1079100019BD00BFC88FFF1F704700BF38B5144C9A
:10792000037801225B000546204684F83B3084F84A
:107930005E2084F85D20FFF78BFC20460021FFF7D6
:1079400047FE0B4C2978012320461A46FFF7CAFE52
:107950000128F6D194F8383094F839209A4205D9A4
:10796000E218013384F83830107E38BDFF2038BD6E
:107970005C8FFF1F38B51B4C037801225B00054666
:10798000204684F83B3084F85E2084F85D20FFF7C1
:107990005FFC20460021FFF71BFE124C2978204691
:1079A00001230222FFF79EFE0228F6D194F8382028
:1079B00094F839108A420FD2531CDBB2A0189942B6
:1079C00084F83830007E0AD9234402321B7E84F8C2
:1079D000382040EA032038BD4FF6FF7038BD40F430
:1079E0007F4038BD5C8FFF1F0C2901D900207047F4
:1079F0000231490001F0FE01FFF7BCBF70B50C4C2D
:107A00000378164601255B00204684F83B3084F855
:107A10005E5084F85D50FFF71BFC31462046FFF7AF
:107A200017FC29462046BDE87040FFF7D1BD00BFD6
:107A30005C8FFF1FF8B505460F46164641242146C8
:107A40003A462846FFF7DAFF611C0234C9B23246D3
:107A50002846E4B2FFF7D2FF592CF0D1F8BD00BFA1
:107A600038B504460D463548FFF706FC63228021F1
:107A700020462570FFF7C2FF012002F0C9FC204616
:107A800000225E21FFF7BAFF20465D21FFF746FF87
:107A9000242801D0002038BD204606220C21FFF703
:107AA000C9FF204601222B21FFF7A8FF2046012213
:107AB0002C21FFF7A3FF20460E222D21FFF79EFF6A
:107AC000204600222E21FFF799FF204601222F2178
:107AD000FFF794FF204605223021FFF78FFF204655
:107AE00001223121FFF78AFF204600223221FFF7D1
:107AF00085FF204600223321FFF780FF2046002229
:107B00003421FFF77BFF204600223521FFF776FF67
:107B1000204600225B21FFF771FF204610225C21E6
:107B2000FFF76CFF204620225D21FFF767FF20460C
:107B30008F225E21FFF762FF012038BD5C8FFF1F9F
:107B400010B4047F4160022CC26002D010BC01F06E
:107B5000D7BB836810BC184790E80C00F0B41C68D1
:107B600059682568164F174E29432160164D17494D
:107B70001760D66015611160417A154A5C180A31A8
:107B800094F8244053F8215002EBC40149680D6079
:107B9000017A5C1803EB8101247ECD6902EBC401FC
:107BA00049680D60817A581803EB810390F8300022
:107BB000596B02EBC002F0BC53681960704700BFFC
:107BC00001401F00011000380110007800001F80E4
:107BD00030FF0000704700BFF0B50C1EBDF8146008
:107BE00034DBB0F906701919B942C4BF3B1B1BB294
:107BF000002BA6461CDD002A1146B8BFD11D02F09D
:107C00000705CC10826A012007FB04E1A840012E81
:107C10000A44C0B21ED00CD3022E09D1013B12FA85
:107C200083F3013A12F8011F41409A421170F9D1D1
:107C3000F0BDC043013B12FA83F3C0B2013A12F81F
:107C4000011F014093421170F9D1F0BD23441BB2D2
:107C50000024C6E7013B12FA83F3013A12F8011F30
:107C600001439A421170F9D1F0BD00BFF8B50D1E65
:107C70000EDB14461F46064601F03AFBA84207DD1C
:107C8000002C05DB304601F037FBA04201DCF8BDDB
:107C9000F8BD304601F02AFB022853D003284BD010
:107CA000012806D16540F3886C406540013B5D1BAF
:107CB0002DB2012F03D02AD3022F14D0F8BD002CEF
:107CC0002246B6F90630B06AB8BFE21D42F3CF02D1
:107CD00002FB035504F00704435D012101FA04F49B
:107CE0001C434455F8BD002C2246B6F90630B06A54
:107CF000B8BFE21D42F3CF0202FB035504F00704B4
:107D0000435D012101FA04F45C404455F8BD002CA8
:107D10002246B6F90630B06AB8BFE21D42F3CF0280
:107D200002FB035504F00704435D012101FA04F44A
:107D300023EA04044455F8BD3389013B591B254609
:107D40000CB2B6E7F18832890139013A4D1B141B98
:107D50002DB224B2ADE700BF2DE9F041079E9DF999
:107D60001880089D04461F4600F0C0FF0D4B0E48CA
:107D70000E4984F83380FF22002F08BF1F4684F885
:107D80002F20002384F8302084F8312084F832201A
:107D90002060A665E565676261652362A36220468F
:107DA000BDE8F0815C8FFF1F88F4000001100138EE
:107DB00010B50446806A034B236008B105F078FBD8
:107DC000204610BD88F40000F8B5436ADBB190F896
:107DD0002C200125AA4083F83B2083F85E5083F8CD
:107DE0005D500446406A03680E461B6800219847B0
:107DF000606A036831461B6898472946606ABDE897
:107E0000F840FFF7E5BBC26BC56C1368046A23EA50
:107E1000050313604CB122684FF00043D3625163F5
:107E2000D36A002BFCDA936BF8BD836B466B082595
:107E3000802410E03768426C3A4332601F68826CDD
:107E40003A431A601A68876C013D22EA07024FEA3A
:107E500054041A6007D02142ECD13268476C22EA00
:107E600007023260EAE7F8BD70B50446406A0D4685
:107E700000282BD0A16DFFF749FA002D20460CBF3A
:107E8000A621A721FFF7A0FF606A20B1E16DBDE840
:107E90007040FFF73BBA216C226D0868236A0243E9
:107EA0000A6093B1DA7A82B1D00703D5224A996980
:107EB0001160DA7A910703D5204AD9691160DA7A1C
:107EC000520702D51E4A1B6A136070BD236A002B3D
:107ED0002BD0D97A626DE1B172B6D97ACE0706D5C8
:107EE0001848D9680668314099610160D97A8807D5
:107EF00006D51548196906683140D9610160D97AFB
:107F00004E0705D51148596906683140196201606C
:107F100062B61B68D968914207D00D4818600D49B8
:107F2000DA6042F0804018611960226C216D13689C
:107F300023EA01031360A0E700E100E004E100E0B0
:107F400008E100E080E100E084E100E088E100E099
:107F500001403F0000003F80436A2DE9F0410546A3
:107F60000E469046002B3ED090F82C100124A140E4
:107F700083F83B1083F85E4083F85D40406A0368F5
:107F800000211B6808F1FF379847FFB2B8F1000FD6
:107F900023D03744A046013E686A16F8011F0368E3
:107FA0001B6898470134B742E4B216D0202CF3D1B5
:107FB0000121686AFFF70CFB95F82C206B6A5200D0
:107FC00083F83B2083F85E8083F85D80686A0368ED
:107FD00000211B6898470124DEE7686A0121BDE89B
:107FE000F041FFF7F5BAC26BC16C136823EA0103D5
:107FF00006EB080413604FF00048A6420ED02B6A2F
:1080000016F801EB63B11A68C2F82C80C2F834E0AC
:10801000D36A002BFCDAA642936BF0D1BDE8F08165
:10802000AB6BD5F834C008208021DCF800206F6CE1
:108030001EEA010F14BF3A43BA43CCF800201A6875
:10804000AF6C3A431A601A68AF6C013822EA070233
:108050004FEA51011A60E8D1CFE700BF70B504467E
:10806000406A0D46002828D0A16DFFF74FF9204641
:108070002946FFF7A9FE606A20B1E16DBDE87040B6
:10808000FFF744B9216C226D0868236A02430A6035
:1080900093B1DA7A82B1D00703D5234A9969116086
:1080A000DA7A910703D5214AD9691160DA7A520741
:1080B00002D51F4A1B6A136070BD236A002B2BD0A8
:1080C000D97A626DE1B172B6D97ACE0706D5194870
:1080D000D9680668314099610160D97A880706D568
:1080E0001548196906683140D9610160D97A4E078F
:1080F00005D512485969066831401962016062B6B7
:108100001B68D968914207D00D4818600D49DA60A4
:1081100042F0804018611960226C216D136823EAD7
:1081200001031360A3E700BF00E100E004E100E009
:1081300008E100E080E100E084E100E088E100E0A7
:1081400001403F0000003F802DE9F041044686B029
:10815000806A9DF830801E460F461546B4F90830F7
:10816000002800F04281DA1D48BF03F10E02B4F985
:108170000630D21003FB02F2002105F0BDFCB4F979
:108180000820202A00F39280B4F90610A34B0120A6
:10819000203A733902EBD27201EBD1714FF0200E0D
:1081A000029073208DE8014042F34F0241F34F01EA
:1081B000204600F051FE606A84F82D70002800F01F
:1081C0004D81002D40F08A80B4F90830202B14BF77
:1081D0003D253C2584F82C50B8F1000F40F08580F7
:1081E00006B394F93300002818DBC0B2012102F075
:1081F000E7F8012194F8330002F0CEF8012002F0F4
:1082000007F9002194F8330002F0C6F80A2002F0C2
:10821000FFF8012194F8330002F0BEF8606A0028EC
:1082200000F08280A16DFFF771F804227C4920469E
:10823000FFF792FE217A0139C9B22046FFF7C4FD4B
:10824000784904222046FFF787FE94F92D30012B50
:1082500014BF142110212046FFF7B6FD04227249F5
:108260002046FFF779FEB4F90630802B00F09280AB
:10827000602B00F0A680D9212046FFF7A5FD94F9D8
:108280002D30012B14BFF12122212046FFF79CFD48
:10829000204606226549FFF75FFE606A50B3E16D34
:1082A000FFF734F8012006B0BDE8F081B4F90610FC
:1082B0005F4B0120403A52394FF0400E029002EBE2
:1082C000D272522001EBD1718DE8014042F34F028E
:1082D00041F34F01204600F0BFFD6CE76DB284F81A
:1082E0002C50B8F1000F3FF47BAFFEF7C5FF002E16
:1082F00094D076E7216C226D0868236A02430A60F5
:1083000073B1DA7A62B1D00703D54A4A996911602C
:10831000DA7A91077CD4520702D5474A1B6A136068
:10832000012006B0BDE8F081236A002B2BD0D97A5A
:10833000626DE1B172B6D97ACF0706D53F48D968E8
:108340000568294099610160D97A8E0706D53C48B5
:10835000196905682940D9610160D97A4D0705D5A9
:1083600038485969056829401962016062B61B687E
:10837000D968914207D0344818603449DA6042F035
:10838000804018611960226C216D136823EA010393
:1083900013604AE7B4F90830202B00F08680402BA8
:1083A0007FF469AF2A4920460322FFF7D5FD94F9EF
:1083B0002D30012B14BFCF219F212046FFF704FD54
:1083C00059E7B4F90830102B7FF455AF2149204606
:1083D0000322FFF7C1FD94F92D30012B14BFAF210B
:1083E00010212046FFF7F0FC45E7DA1D48BF03F1F6
:1083F0000E02B4F90630D21003FB02F210460592C9
:1084000005F04EF8A06200283FF44DAF059AB3E6A0
:10841000114AD9691160DA7A7DE700BFE0F4000003
:10842000C0F60000C4F60000C8F60000CCF600005C
:10843000D4F6000000E100E008E100E080E100E0A7
:1084400084E100E088E100E001403F0000003F805F
:10845000DCF4000094F9000004E100E0012194F84C
:108460003100244F01F0ACFF94F83200012101F0FB
:10847000A7FF94F9312094F9323057F83220E263A3
:1084800057F83330206A23640125E56425651A68AE
:108490002A431A6078B1B8F1000F3FF428AFFFF714
:1084A0005BFB002E3FF4BAAE9BE604221249204645
:1084B000FFF752FDDFE6294694F82F0001F080FF18
:1084C000294694F8300001F07BFF94F92F2094F9AD
:1084D000303057F83220626357F833306564A56452
:1084E0001A68A36322F001021A60002E3FF496AED0
:1084F00077E600BF30FF0000D8F40000B0F9082094
:10850000D31D48BF02F10E03B0F90620806ADB10CC
:1085100002FB03F2002105F0EFBA00BFF0B500291D
:10852000BDF814502EDBB0F90660B1422ADA002AF9
:1085300059DBB0F9087014461C44BC42C4BFBB1AD6
:108540001BB2002B1EDDD2B2D408D0F828E016FBF7
:10855000041112F00702DBB20EEB010421D0C2F1CC
:108560000807FAB2374F9342BF5C0CD2C3EB020C40
:10857000FF2646FA0CF6012D07EA06073FD005D381
:10858000022D36D0F0BD012D39D030D21EF8016059
:1085900026EA07070EF801709342F3D3B0F90610EC
:1085A0000C449A1AD2B2072A10D9022D36D0002DC7
:1085B00014BFFF26002613462670083BB0F90610AC
:1085C000DBB2072B0C44F7D802F00702002AD9D0FF
:1085D0001D4B012D9B5C1DD017D3022DD2D12278CB
:1085E00053402370F0BD13441BB20022A1E7022DBB
:1085F00025D11EF8016077400EF80170CCE71EF817
:10860000016037430EF80170C6E7227822EA0303BF
:108610002370F0BD227813432370F0BD11462378F8
:10862000DB4323700839B0F90630C9B207291C446E
:10863000F5D812F00702A5D0034B9B5CCFE734447A
:10864000AFE700BF78F4000068F4000070B4C47DA8
:10865000BDF80C50022C18D0032C1FD0012C0BD0CD
:10866000002A03DBB0F90840944201DC70BC70477B
:10867000039570BCFFF7B0BAC4880395013CA41AF7
:108680000A4621B270BCFFF749BF0689C488013E83
:10869000641AB21AE41A12B221B2E1E7048903950E
:1086A000E41A641A114622B270BCFFF737BF00BF4C
:1086B00070B4C57DBDF80C60022D1AD0032D12D008
:1086C000012D03D0039670BCFFF728BFC488E41ABD
:1086D000A41A0A4621B2002A03DBB0F908409442EA
:1086E00013DC70BC70470489013C641A114622B245
:1086F000F1E7C48805890396013CAD1AED1A621AA8
:1087000011B22AB270BCFFF709BF039670BCFFF725
:1087100063BA00BF2DE9F8430446406A002863D0DD
:10872000A16DFEF7F3FD052274492046FFF714FC06
:10873000A1790139C9B22046FFF746FBB4F90820F8
:10874000E588A66AD31D48BF02F10E03DB10626AFA
:1087500015FB03F51FFA85F8002A7BD094F82C301E
:108760000125AB4082F83B3082F85E5082F85D50C4
:10877000606A036840211B6808F1FF379847BFB261
:10878000B8F1000F23D03744A846013E606A16F8BE
:10879000011F03681B6898470135B742EDB216D038
:1087A000202DF3D10121606AFEF712FF94F82C20EE
:1087B000636A520083F83B2083F85E8083F85D8013
:1087C000606A036840211B6898470125DEE70121A4
:1087D000606AFEF7FDFE606A002800F08D80E16DA2
:1087E000BDE8F843FEF792BD236A002B2BD0D97A5F
:1087F000626DE1B172B6D97ACE0706D54048D96824
:108800000568294099610160D97A8D0706D53D48F0
:10881000196905682940D9610160D97A480705D5E9
:1088200039485969056829401962016062B61B68B8
:10883000D968914207D0354818603549DA6042F06E
:10884000804018611960226C216D136823EA0103CE
:10885000136068E7E26BE36C1168276A0B4306EB71
:10886000080913604FF0004E4E450DD016F801CBAD
:108870002FB33A68C2F82CE0C2F834C0D36A002B98
:10888000FCDA4E45936BF1D1226C236D11680B43DA
:10889000136097B1FB7A83B1D90703D51D4BBA6931
:1088A0001A60FB7A9A0703D51B4BFA691A60FB7AA8
:1088B0005B0702D5194B3A6A1A60BDE8F883A36BCF
:1088C000D4F8348008208021D8F80020656C1CEA98
:1088D000010F14BF2A43AA43C8F800201A68A56CE8
:1088E0002A431A601A68A56C013822EA05024FEA89
:1088F00051011A60E8D1B7E7276AC5E770F40000B4
:1089000080E100E084E100E088E100E001403F0018
:1089100000003F8000E100E004E100E008E100E049
:108920002DE9F04F85B09946BDF93870BDF83CA0EF
:10893000BB1AC1EB090B002BB8BF5B42BBF1000FA8
:10894000B8BFCBF1000B5B450D4616460093804641
:1089500048DC4D453A4633464CDC194613460A4638
:10896000C5EB09019B1A89B2002B0CB2B8BF5B4260
:1089700004EBD474BE42ACBF4FF0FF3201224D4530
:10898000039102924FEA640429DC9BB201930DE04B
:10899000D8F80070BF69B847019BE41AA3B21CB2B3
:1089A0000135002C2DB211DBA94518DB009B5B457E
:1089B0002A46534631464046EADCD8F80020534662
:1089C0009769294632464046B847E5E7029A164479
:1089D000039AA94502EB030436B224B2E6DA05B0E5
:1089E000BDE8F08F4A462B46B94635464D451746F9
:1089F0001E46B2DD304629463E464D46074689466C
:108A0000AEE700BF10B404682469A44610BC6047F8
:108A100030B40468BDF808500295A46BA44630BC7D
:108A2000604700BF30B40468BDF808500295E46B9D
:108A3000A44630BC604700BF70B40468BDF90C6048
:108A4000BDF8105003960495246CA44670BC604792
:108A5000704700BF10B582B0B0F90C2001910168D9
:108A6000009200220C6CB0F90A301146A04702B007
:108A700010BD00BF704700BF01F003010129C1759F
:108A800006D0032904D0C2880389428183817047BC
:108A90000289C38842818381704700BF2DE9F0417C
:108AA0000568134E6F6986B0B7420446BDF8308042
:108AB00010D1013B13441BB20093CDF804800B4648
:108AC000AD6A2046A8472368DB6AB3420AD106B0E4
:108AD000BDE8F081059304920391B84703A9256886
:108AE0000EC9E6E7204606B0BDE8F041184700BFD2
:108AF000518A00002DE9F0410568124E6F6986B079
:108B0000B7420446BDF830800FD1013BCDF8048058
:108B10000B4400921BB2AD6A2046A8472368DB6A6B
:108B2000B3420AD106B0BDE8F081059304920391E7
:108B3000B84703A925680EC9E7E7204606B0BDE897
:108B4000F0411847518A00002DE9F04F0568DFF821
:108B500058B06F6985B05F450646BDF93890BDF8DD
:108B60003CA00C46904615D11F19BC420CDACDF83A
:108B700000A0214601342D6A4B464246304624B2BD
:108B8000A847BC423568F2DBEB6A5B4507D105B00C
:108B9000BDE8F08F0393B8473568039BE4E73046A0
:108BA00005B0BDE8F04F1847518A00002DE9F043A9
:108BB00087B099420546BDF93840BDF83C6025D0E4
:108BC000A24212D00768DFF88080D7F81490C14520
:108BD00032D18DE850002846BC6AA0472B68DB6A7A
:108BE000434524D107B0BDE8F083994202DD084631
:108BF0001946034628680E96C46B01335B1A1BB2F4
:108C00002846A44607B0BDE8F0436047A24202DD13
:108C1000134622461C4628680E96631C846B9B1ADA
:108C20001BB22846A44607B0BDE8F043604728467B
:108C300007B0BDE8F0431847059304920391C84775
:108C400003A92F680EC9C4E7518A00002DE9F04F2F
:108C5000D0F800E0DFF89090DEF814B083B0CB4598
:108C60000446BDF93080BDF834A00D4617461E46B7
:108C700031D1CDF800A0DEF824B0294633463A467B
:108C80002046D8472368CDF800A008F1FF323A44C7
:108C9000D3F824B0294612B233462046D847236879
:108CA000CDF800A02946D3F820B03A4643462046E6
:108CB000D8472068CDF800A0711E29444346056AB4
:108CC00009B23A462046A8472368DB6A4B4506D1DD
:108CD00003B0BDE8F08FD847D4F800E0C9E72046DC
:108CE00003B0BDE8F04F1847518A0000F0B40024EB
:108CF00001264FF6FF75094F07600471C475C481E2
:108D000004824476C4618675067685824582C18078
:108D1000028141818281F0BC704700BFA0F9000050
:108D20002DE9F04F85B00668BDF84450BDF9388094
:108D3000CDF8008004460195D6F848B00392BDF9FD
:108D40003C60BDF9407089469A46D8472368019532
:108D5000009742465146D3F8488020463346C047E4
:108D60002068039B0E930F95856C4B463A4631461F
:108D70002046AC4605B0BDE8F04F60472DE9F04F06
:108D800087B01746BDF9404000912546E91D05937F
:108D900044BF2B4603F10E010268BDF848605369D9
:108DA0000294C91003912B49BDF9444001968B42AE
:108DB000824645D1002C3CDD029B3C445E1EB6B28F
:108DC0004FF0000923B2049301364D46029B002B5D
:108DD00028DD059B002403EB090806E0EDB22B0615
:108DE00004F1010411D4A6421CD0A1B211F0070F66
:108DF00023B24FEA4505F1D1002BB8BF0733DB1092
:108E0000013418F803502B06EDD5009BD2F818B0AA
:108E100019443A4609B2019B5046D847A642DAF8AF
:108E20000020E2D1039B01379944049B3FB2BB422F
:108E3000CCD1D36A074A934206D107B0BDE8F08F80
:108E40009847DAF80020B5E7504607B0BDE8F04F84
:108E5000184700BF518A000070B4BDF90C60BDF91D
:108E60001050BDF8144003960495059470BCFFF7AC
:108E700085BF00BF2DE9F04F93B090460591C169C1
:108E80001090BDF870000790BDF874909DF878A020
:108E90000493002900F0CD800A7A0AC98946049912
:108EA0008A1AD2B203EBC203BAF1010FDA780B923D
:108EB00093F905201E8893F802B00F9293F90640AB
:108EC00079D913B2099323B20C93109B1A68A94B5A
:108ED0001193194653698B4240F0A6800B9B002BDF
:108EE00055D01FFA88F300210D93C8462344DDF8BE
:108EF000409006910E930F460C46BBF1000F3FD0F9
:108F0000BDF818100C9B03971FFA8AF0CB1813FBBF
:108F100000F304900E9801440D98034409B21BB26B
:108F20000A910893002505E00135EBB264009B45EA
:108F3000E4B222D9039B2B44590703D1731C18F8C0
:108F400006409EB22306EFD5099BBDF81000E91834
:108F500011FB00F10598BAF1010F0FFA8AF30144F1
:108F60001CD0079801900093D26909B21746484671
:108F7000089AB847D9F80020D6E7039F5F44FFB2AC
:108F8000069B0B9901330693DBB29942B5D8D36A9D
:108F9000119A934243D113B0BDE8F08F0F9B19187B
:108FA00093690A9A29441F4609B2079B4846B84765
:108FB000D9F80020B8E700230C93099385E70A9AB3
:108FC0000D9B0132013B52B213F0FF030A920D9345
:108FD0006FD1DDF81890079BDDF83C80DDF820A00C
:108FE0004B4517D0BAF1010F00F0C8800B9A109DC5
:108FF000CDF804900BEB8B014FEACB030A440093AE
:109000001146DEF81C405346424609B22846A047A6
:10901000D5F800E0DEF82C30119A9342BBD01098BE
:1090200013B0BDE8F04F1847109D284698472A68AE
:1090300054E7109A0598B2F90A308342ABDDB2F9D1
:109040000C304345A7DD062313FB0A03002BA2DDEA
:1090500008EBCA03002B9EDD537E2BB9049BAF2B7C
:1090600002D90133DBB20493109BD3F800E0414BEB
:1090700011931A46DEF81430934240F08E801FFAA6
:1090800088F30E9308339BB2BDF814200593052393
:109090000D9300230A93CDF83C800FFA8AF3DDF894
:1090A0004080CDF818900B921FFA8AFBCDF820A0D3
:1090B00099460A9ABDF810000B9C0E9D052319468F
:1090C00011FB00232C481146C75C039702FB0B429F
:1090D00014FA81F312B21BB209920C932C462E465D
:1090E0001CE0089B0999012B2AB24B4640462DD023
:1090F000079F0197CDF80090DEF81CA0D047D8F864
:1091000000E0039B5B0801340393059BA4B25D441C
:109110005E44A342ADB2B6B23FF451AF039BD80751
:10912000DFD4079B069A9342EBD0089B012B16D005
:10913000069B0193CDF80090DEF81CA009994B46E0
:1091400032B24046D047D8F800E0DAE7DEF818A09F
:10915000079B0C9922B2D047D8F800E0D1E7DEF89F
:1091600018A00C991346404622B2D047D8F800E028
:10917000C7E700BF518A0000F0F900000B99109D6D
:10918000CDF800900531DEF8204009B242460823B0
:109190002846A047D5F800E03CE7109C20469847B9
:1091A000D4F800E06BE700BFF0B5C36985B00446B2
:1091B0002BB30A2968D00D294AD01A7A914247D395
:1091C000587A884244D35D688A1A05EBC205AA78AA
:1091D000002A50D0E87800284DD0207E00283AD0D0
:1091E00095F905E0B4F90E00A67DB4F90A70724451
:1091F00006FB0202BA4262DCB4F9102030E00A2910
:1092000056D00D2924D0027E002A4BD0B0F90E0092
:10921000A57DB4F90A60062212FB0502B2423EDDCA
:10922000228AE38102EBC50212B218462282A78A83
:10923000668A02950B468DE8C00001462046FFF77E
:1092400019FEA37DE28903EB430302EB4303E381B1
:10925000012005B0F0BDA67DB4F90E00B4F91020D0
:10926000B4F814E0678A02960B468DE88040014608
:109270002046FFF7FFFD2979E389A27D012001FB4C
:109280000233E38105B0F0BD0022C2819A7A817D6C
:10929000038A01FB02330382012005B0F0BDB4F95B
:1092A0001020C4E7857DB4F91020B0F90E00BEE7A8
:1092B000028A817DC38102EBC1030382C8E70020DB
:1092C000E0819B7A228A03FB062212B22282C7E740
:1092D000C1810282704700BF002908BF012181754A
:1092E000704700BF81824182704700BFC07D7047D8
:1092F000B0F90A00704700BFB0F90C00704700BF1A
:1093000010B4EFF3108272B6437F33B9017F0129A5
:1093100007D003290FD00123437702B962B610BCEE
:109320007047124C2168A1B1114943610B688361F8
:1093300008605861EFE70F4C216881B10E49436125
:109340000B688361086058610C4B4FF080511960C5
:10935000E1E7074B4161816120601860DBE7064B64
:109360004161816120601860EEE700BFDC9CFF1F57
:10937000D89CFF1FCC9CFF1FD09CFF1F04ED00E07A
:1093800070B5EFF3108272B60C4C206880B10C4EB1
:1093900000254369236073B19D6102B962B64577C8
:1093A00083689847EFF3108272B620680028F0D1E6
:1093B00002B962B670BD3360EFE700BFCC9CFF1FFF
:1093C000D09CFF1FFFF7DCBF184A30B41468002C94
:1093D00027D0036821688B420ED2CB1A002184600B
:1093E000C1602360E06010600223037530BC7047E9
:1093F00011688B42144608D3A2685B1A0360002AE6
:10940000F6D18260C460A060EEE7D268C26084607A
:10941000E060C568CB1A0222A8602360027530BCE8
:1094200070478460C4601060DEE700BFD49CFF1FFB
:10943000F8B5224E34682CB32368002B3AD1204F64
:109440001D4604E03468ECB12368002B32D1A368D8
:1094500003B1DD6020693360036825751B68BB427A
:1094600021D1037F4560022BC46020D0FFF748FF65
:109470006368002BE6D023602046FFF7A5FF346821
:10948000002CE1D1EFF3108372B60E4A0021106870
:10949000116003B962B628B18468FFF795FF2046D2
:1094A0000028F9D1F8BD224600219847E0E78368FB
:1094B0009847DDE7013B2360E4E700BFD49CFF1F32
:1094C000417B0000E49CFF1F024A136801331360D4
:1094D000FFF7AEBFF09CFF1F704700BF0368F0B4FA
:1094E000FBB1002501249D60DC601B4C1A601C440C
:1094F000241104F144056A11032692009E60174F5F
:109500000679174B47F8241002F1604202F56142D8
:1095100005F01F05012000FA05F5E6541560F0BCC2
:109520007047104C236843F40003236000BF0E4BC8
:109530000E4DA4F58734A4F59E7401261E602346C3
:1095400004609C68002CD0D01033AB420360F8D18B
:10955000002303601846E2E7008FFCBF3490FF1F32
:1095600044E400E03C80044000700340407103404C
:109570000168A9B10B4BF0B40B441B110A4E0B4F01
:109580000B4D46F8237003F1440202F01F0401233F
:109590005211A340002445F822308C600460F0BCD6
:1095A000704700BF008FFCBF3490FF1FD9940000AC
:1095B00080E100E0024A034B012111601B6818475B
:1095C0000C7103403490FF1F024A034B01211160CC
:1095D0005B6818471C7103403490FF1F024A034B1D
:1095E000012111609B6818472C7103403490FF1FC4
:1095F000024A034B01211160DB6818473C710340AC
:109600003490FF1FF8B50E4671B17AB10746144683
:1096100000253B6816F8011B1B6838469847013C3B
:109620000544F6D12846F8BD0846F8BD1046F8BDF9
:1096300000B5064A036812885B6883B001A9ADF8DB
:1096400004200222984703B05DF804FBF0FE0000FE
:10965000F0B507468BB0002A33D0012A08BF0A2292
:1096600051B3212400E0F4B2B1FBF2F502FB151175
:10967000C8B2092900F1300198BFC8B20AA988BF51
:109680003730214488BFC0B201F8240C661E294639
:10969000002DE8D133B1013CE4B20AAB23442D22C2
:1096A00003F8242C3B6801AA11195B683846C4F101
:1096B000220298470BB0F0BD30228DF825202124DE
:1096C000E8E70368C9B21B6898470BB0F0BD00BF5C
:1096D0000029BABF49422D2300230A22FFF7B8BF51
:1096E000374A384913681B06FCD40B6813F0800313
:1096F000F8D172B634490A78002A5FD0334A344828
:10970000F0B4344C176806682568D4680C303E44C1
:10971000143200681268304F35442C44204402440F
:10972000C2F34E022D4E2E482E4D2F4C42F40042D5
:109730003A60376806682D682C4A24680C303E442D
:10974000006812682A4F35442C4420440244C2F376
:109750004E02284E2848294D294C42F400423A60D6
:10976000376806682D68274A24680C303E44006834
:109770001268254F35442C4420440244C2F34E0263
:10978000224E2348234D244C42F400423A6037686D
:1097900006682D68214A24680C303E44006812682F
:1097A00035442C4420440244C2F34E021C4842F487
:1097B000004202600B7062B6F0BC704762B6704740
:1097C00024B0034024B00B40E99CFF1F38B0034095
:1097D0003CB0034040B003402CB0034058B00340BD
:1097E0005CB0034060B0034064B003406CB0034021
:1097F00030B0034038B00B403CB00B4040B00B40A1
:1098000044B00B404CB00B402CB00B4058B00B4058
:109810005CB00B4060B00B4064B00B406CB00B40D0
:1098200030B00B4030B42948294A2A4B2A4D6024D5
:10983000E121047011701B78284C082B30D00A2BC2
:109840002748284937D00C2B0CBF35223D22122344
:109850002A60236002600B60234B24491B78244A52
:10986000BBB101230B601360224B23491B78234AB1
:10987000012B26D9042B0FD9082B1ED9102B94BFEE
:10988000862387230B6013601D4B01221A7030BCA6
:1098900070470B601360E7E784230B601360F3E706
:1098A00000F58E200F490830012213232A6023601F
:1098B00002600B60D0E73922F7E785230B60136065
:1098C000E2E780230B601360DEE700BF0040074043
:1098D000014007404490FF1F08B003400CB0034014
:1098E00008B00B400CB00B40EC9CFF1F20B00340B5
:1098F00020B00B404590FF1F24B0034024B00B4024
:10990000E99CFF1F0C2830B417D91023984228BFB8
:1099100018461C46104A114D1178181A8C422870AE
:1099200018D00F4913700B7823B10E490E4A00234B
:109930000B60136030BCFFF775BF0A2802D90C23F7
:109940001C46E7E7082802D90A231C46E2E7082359
:109950001C46DFE730BC70474490FF1FE89CFF1FA8
:10996000E99CFF1F24B0034024B00B4028282FD8C7
:10997000334B2DE9F0411E5CFF2E2BD0314B1B7871
:10998000002B2AD132062CD472B62F4D2F4C2F46E5
:10999000012326602B7062B672B623681B060CD4B6
:1099A0003B781BB9F4E72B78002BF1D062B602F0BC
:1099B0009BF972B623681806F5D5254B1B68002263
:1099C0002A7062B6234A107843FA00F0BDE8F081AD
:1099D000002070470020BDE8F081FFF781FE3206CD
:1099E000D2D572B61C4DDFF87C801C4C06F04007C7
:1099F000FFB206F03F06D8F80030DFB123F01003C5
:109A0000C8F8003001232660134A2B7062B672B684
:109A1000236819060CD413781BB9ECE72B78002BBC
:109A2000E9D062B602F060F972B623681B06F5D57C
:109A30000B4BC3E743F01003C8F80030E2E700BF68
:109A4000F4FE0000E99CFF1FEB9CFF1F00B00340E9
:109A500010B00340E89CFF1FEA9CFF1F00B00B40C2
:109A600010B00B400CB00B400A4A0B49136843F48A
:109A7000805313600B7843B9084BC0221A70084B0F
:109A800080F30C0000B218807047044B80221A70DB
:109A9000F5E700BF2C800440EC9CFF1F21C00C4068
:109AA00000C00C40F0B51B4B1B4E596818689A68F3
:109AB000DB6885B06C460FC4337899071DD5174A0B
:109AC000174C1378174913F0700318BF1370164A18
:109AD000164B8027177000263320032226706D4610
:109AE00008701A7072B6043C45F001052046A8477C
:109AF00062B6237813F0700309D10D4B064901E0DB
:109B0000013B02D00A78D207FAD505B0F0BD237028
:109B100005B0F0BD20FF000001000240000002403F
:109B2000040002400B000240070002400A0002400D
:109B3000410D0300B0F5006F0AD210B5094B1B7838
:109B4000DB07044606D504F1A0500078C0B210BD72
:109B500000207047FFF7A6FF04F1A0500078C0B2C4
:109B600010BD00BF01000240B0F5006F17D238B53C
:109B70000F4B1B78DA070D46044611D504F1A050AF
:109B80000378AB420AD00B4A137813F0700318BF66
:109B90001370074A05701378DB07FCD538BD704792
:109BA000FFF780FF04F1A0500378AB42EBD1F5E75B
:109BB000010002400000024008B5F6F75FFDF7F72C
:109BC000EDFF02F091F8FAE7844641EA000313F052
:109BD00003036DD1403A41D351F8043B40F8043BB4
:109BE00051F8043B40F8043B51F8043B40F8043B77
:109BF00051F8043B40F8043B51F8043B40F8043B67
:109C000051F8043B40F8043B51F8043B40F8043B56
:109C100051F8043B40F8043B51F8043B40F8043B46
:109C200051F8043B40F8043B51F8043B40F8043B36
:109C300051F8043B40F8043B51F8043B40F8043B26
:109C400051F8043B40F8043B51F8043B40F8043B16
:109C500051F8043B40F8043B403ABDD2303211D3B6
:109C600051F8043B40F8043B51F8043B40F8043BF6
:109C700051F8043B40F8043B51F8043B40F8043BE6
:109C8000103AEDD20C3205D351F8043B40F8043BB6
:109C9000043AF9D2043208D0D2071CBF11F8013BB4
:109CA00000F8013B01D30B8803806046704700BF7A
:109CB000082A13D38B078DD010F003038AD0C3F189
:109CC0000403D21ADB071CBF11F8013B00F8013B6B
:109CD00080D331F8023B20F8023B7BE7043AD9D32A
:109CE000013A11F8013B00F8013BF9D20B780370FF
:109CF0004B7843708B7883706046704708B5104C82
:109D000008E0236859050DD423681A050FD4236889
:109D1000DB0411D423685803F3D500F08DFE2368CB
:109D20005905F1D502F044F823681A05EFD502F081
:109D3000D5F82368DB04EDD500F0F0FCEAE700BFBE
:109D40003480044008B5FFF7D9FF00BF014B102253
:109D50001A80704700200540704700BF094908B5C8
:109D60000B6830B16A461844A2F58052904202D284
:109D70000860184608BD03F065FB0C2303604FF034
:109D8000FF3008BD4890FF1FFEE700BFEFF31380D0
:109D900070B9EFF310836BB9EFF305825AB94FF442
:109DA0008070EFF311832BB1984228BF184670479B
:109DB0004FF0FF3070470F2A01D81846F1E7014BEA
:109DC000D05CEEE7F0E300E0F0B44D1E2E46002438
:109DD00000E00134B0FBF2F302FB1300092800F1AC
:109DE00030078ABF3730F8B2C0B206F8010F184604
:109DF000002BEED10A1953704CB1107815F8016F91
:109E000028700133E01A834202F80169F5DB084645
:109E1000F0BC7047704700BF10B40F4B53F83020B0
:109E200092F880422CB1012369B182F8803010BCD5
:109E3000704703EBC0035B681A6841B922F0020265
:109E40001A6010BC704782F8003110BC704742F0B5
:109E500003021A6010BC704730FF00001C4A02EB7E
:109E6000C00301295B6811D004291BD052F83000CF
:109E7000002280F8802229B1022920D0032922D093
:109E80001A6070474FF480721A60704752F83000C1
:109E90004FF4A27280F880121A601A6822F0200231
:109EA0001A60704752F830104FF4A272012081F806
:109EB00080021A601A6842F020021A60704740F26D
:109EC00003121A6070474FF481721A60704700BF26
:109ED00030FF0000212848D8F8B5042A44D8DFE82C
:109EE00002F0484B4E0345004FF410262B4B03EB7A
:109EF000C0030D465C68216811F4E06148D0284B2E
:109F0000284A2949C3F89C2104F140422748C3F854
:109F1000A411A2F59221264FC3F8A0017C2925485F
:109F2000C3F8A871C3F8AC012CD9A2F594237C2BFB
:109F30002AD9A2F596237C2B28D9A2F598237C2B2D
:109F400029D9A2F59A227C2A27D81B4872B6236801
:109F500023F4702343F08072C4F38401164323601A
:109F600040F82150266062B6F8BD70474FF43026A5
:109F7000BCE74FF40026B9E74FF44026B6E74FF4AC
:109F80002026B3E70D48E1E70D48DFE70D48DDE7A0
:109F9000FFF764FFB3E70C48D8E7F8BD30FF0000D7
:109FA0000082FF1FF188FF1F9988FF1FC588FF1FD0
:109FB0006D88FF1F4188FF1F2491FF1F4C90FF1FDA
:109FC0008490FF1FD490FF1F0491FF1F1A4B03EBD7
:109FD000C00010B4426802F14043A3F592217C29ED
:109FE00023D9A3F594217C290DD9A3F596217C29A9
:109FF0001FD9A3F598217C2919D9A3F59A237C2B85
:10A0000011D80E4C00E00E4C72B613680D4823F0C8
:10A010008773C2F3840123F4803343F080731360A9
:10A0200044F8210062B610BC7047074CECE7074CBF
:10A03000EAE7074CE8E700BF30FF00002491FF1F6C
:10A040008490FF1F159E00004C90FF1F0491FF1F7E
:10A05000D490FF1F30B4054B054D064C0022102153
:10A060001A602A602060196030BC704714D0034029
:10A0700004D0034000D00340282838B52ED0002952
:10A0800004464FDD5F4B1B78012505FA03F28A4237
:10A0900002D8212837D938BD0338C2B2012A3AD9AB
:10A0A000202C4AD0192C48D0574A126802FB0112C2
:10A0B00022FA03F31D2800F29B80DFE800F0928B68
:10A0C000847D9999766F99999999999999999968AF
:10A0D000615A53994C99999999999945494B1B788B
:10A0E0000B2B08D90C2B1CBF0C3B19410846BDE8B3
:10A0F0003840FFF7B9BCC3F10C0399400846BDE8EE
:10A100003840FFF7B1BC2946FFF786FE2946BDE877
:10A110003840FFF7A3BE3D4A126802FB011222FA43
:10A1200003F3C7E72128B6D80021FFF775FE2046C4
:10A130000121BDE83840FFF791BE354A126802FBA5
:10A14000011222FA03F3B5E73249334A0B604FF4A8
:10A150005173136038BD3149314A0B604FF451736C
:10A16000136038BD2F49304A0B6040F244431360FE
:10A1700038BD2E492E4A0B6040F24443136038BD6F
:10A180002C492D4A0B6040F24443136038BD2B49E3
:10A190002B4A0B6040F24443136038BD29492A4AD8
:10A1A0000B6040F24443136038BD2849284A0B60D5
:10A1B00040F24443136038BD2649274A0B6040F201
:10A1C0004443136038BD2549254A0B6040F244439F
:10A1D000136038BD2349244A0B604FF45173136058
:10A1E00038BD2249224A0B604FF45173136038BDC9
:10A1F000212C3FF650AF7F29D4BF002101212046FA
:10A2000093E700BF2C91FF1F088003400890034094
:10A2100008800B4010800B4048A0044018800B4081
:10A220004CA004401880034008B004401080034054
:10A2300004B004404080034018C00440388003400C
:10A2400014C004402880034010B004402080034024
:10A250000CB004403080034010C0044048800340EC
:10A260001CC00440189003403490044010900340F8
:10A270003090044038B1102828BF1020044AC3B2DF
:10A28000107813707047024A0123107813707047DA
:10A290002C91FF1F2DE9F8430E4680463249334D7D
:10A2A000304603F055F847F6122300281ABF1D4622
:10A2B0004FF002094FF00109002425FA04F002F0E2
:10A2C00051FE4FF05E51074602F0A4FE01463046B3
:10A2D00003F052F830B90134072CEED1E80902F04E
:10A2E00041FE07463146384602F048FF4FF07C51A8
:10A2F00002F086FD03F07AF84FF6FF729042A8F163
:10A30000030328BF1046012B29D9B8F1170F17D81E
:10A31000174B23FA08F303F0010383F0010223B97A
:10A32000B8F1190F0FD0BDE8F883124B124D134945
:10A330001A6044EAC9042A6008601C60BDE8F8831A
:10A34000B8F1200FECD10E4B0E4D0F49002244EA1C
:10A35000C9041A602A6008601C60BDE8F8830B4BD2
:10A360000B4D0C49F2E700BF001BB740006CDC024C
:10A370006006F00000800340048003400880034032
:10A3800000800B4004800B4008800B40009003408D
:10A390000490034008900340212801D8FFF73CBDFA
:10A3A000704700BF212806D8044B53F8303093F88B
:10A3B0000002C0B270470020704700BF30FF0000AD
:10A3C000212801D8FFF74ABD704700BF72B60C497B
:10A3D0000C4B0D4A1B680868126862B6520102D520
:10A3E000322B88BF01300949C3F5BB334FF47A7271
:10A3F000FF33A1FB031302FB00F000EB9310704747
:10A40000F09CFF1F18E000E004ED00E0ABAAAAAA50
:10A410002DE9F843054672B6204F214B214A1B68AF
:10A420003C68126862B6520102D5322B88BF0134F3
:10A4300095B3C3F5BB331C4EDFF86490DFF864803E
:10A44000FF334FF47A72A6FB031302FB04F404EB10
:10A45000931472B6D9F800103A68D8F800E062B6E2
:10A46000C1F5BB33FF33A6FB03031EF0806FC4EBC3
:10A4700093134FF47A7002D0322988BF013200FB67
:10A480000233B3F57A7F04D3013D05D004F57A7425
:10A49000DFE701F029FCDCE7BDE8F883F09CFF1F53
:10A4A00018E000E004ED00E0ABAAAAAAF8B52D4B35
:10A4B0002D49DFF8D0E0DFF8D0C02C4E2C4D2D4CCC
:10A4C0002D4A2E4F4FF4000018604FF08070186036
:10A4D0004FF0007018604FF0806018604FF000601F
:10A4E00018600020086028234BF6FF71CCF800109C
:10A4F000CEF80030336013602B6023603B60B362A2
:10A500009362092245F8242CC4F8D80F05F57F651D
:10A51000C7F8D41F07F5FF2707F5FA67C6F8F83F15
:10A520002B6006F5FF26C4F8D42F05F5FD2504F5AC
:10A53000FF24386006F2F4761148316005F5FF65B6
:10A5400004F5FD642B6023600260FFF76BF91920AE
:10A55000FFF75EFF00F0B6FF40F21310BDE8F840D1
:10A56000FFF756BF08E100E0048003401480034079
:10A57000248003402C8003401C800340348003402F
:10A5800000800B400C800340088003402DE9F84F09
:10A59000214B1B6807460BB101221A70DFF8889027
:10A5A0001E4D99F80040DFF884801D4E0134272CA1
:10A5B0008ABF4FF0000A5FFA84FA5446AB462B7804
:10A5C000A34216D1FFF7E2FB40281FDC33791B06BC
:10A5D000F5D59BF800300133272B86BF00221346A8
:10A5E000DAB218F80330DBB2F3712A702B78A34289
:10A5F000E8D00C490A4BFFB208F804700120AC22E5
:10A60000087089F800A0DA70BDE8F88FFF28D6DD61
:10A6100001F06AFBD3E700BF689DFF1F659DFF1F28
:10A6200000C00640649DFF1F6C9DFF1FFC9CFF1F28
:10A630001C4BDFF894C01A681B49F0B542F48052F5
:10A640001A4D1A60DFF884E0194F1A4E1A4C002395
:10A650008CF800304FF451722B701F2840F21335E4
:10A660008EF800303B70337025600A6012D81946AE
:10A670000124124A124D11701248547000212C27E7
:10A68000402693724FF4003491701174D7702E707D
:10A690000460F0BDC0F34431C0F3471400F01F0361
:10A6A000E7E700BF348004400CC00440F99CFF1F62
:10A6B000659DFF1F649DFF1F08C0044000C0064049
:10A6C00031E400E004E100E0F89CFF1F6C9DFF1FF7
:10A6D000034B1B68DB0401D5FFF758BF704700BF71
:10A6E0003480044010B5044C237823B101F0FCFA07
:10A6F0002378002BFAD110BD649DFF1F054A064B3D
:10A7000010781B78C0B2DBB2984238BF4030C01A14
:10A71000704700BFF89CFF1FF99CFF1F30B42B4B04
:10A720001A7994061FD52A48DA7903782949013322
:10A730003F2B0978C8BF00238B42D2B203D0264CEE
:10A74000D9B2E2540170254A116861B1244A1278E5
:10A75000D2B2934236BFC2F140029B1A9B18272BFC
:10A76000C4BF01230B70194AD378DBB2180611D489
:10A770005A060DD5154B1B795B0609D5194B1A499D
:10A780001B6800220A7003B11A70104B2C22DA7079
:10A7900030BC704711790906EAD5144910480C7885
:10A7A0000178C9B28C420DD04A1C272A84BF0021EF
:10A7B0000A460F4D054C98BFD1B2AA5CD2B2E271E5
:10A7C0000170D5E76C21D170D2E700BF00C0064010
:10A7D000F89CFF1FF99CFF1F249DFF1FF49CFF1F87
:10A7E000659DFF1F689DFF1F649DFF1F6C9DFF1FE0
:10A7F000FC9CFF1F21282FD8184B195CFF292BD058
:10A80000174B184ADFF870C003EBC000F0B543687F
:10A81000DFF868E0144F154D154E00241C60DEF87B
:10A820000030012043F020038840CEF8003014604F
:10A830004FF4A07338602E60C2F800C0013BFDD118
:10A8400013689B05FCD42023013BFDD1094B09B2C1
:10A8500033F8110080B2F0BD0020704740000100C5
:10A8600030FF0000005004400850044004500440F1
:10A87000000002030051044080014A003880044077
:10A88000431E032B14D872B60A4951F8230068B14D
:10A8900070B4094C058834F81320466841F82360E9
:10A8A000521B24F8132062B670BC704762B6704722
:10A8B00000207047C89DFF1F0CA0FF1F0138032810
:10A8C0000BD872B6074B53F8203043B100205B68B9
:10A8D0000130002BFBD162B670470020704718464C
:10A8E000F9E700BF1C9EFF1F30B472B62B4A1378E5
:10A8F0001D0706D52A4B196A002936D0996A002906
:10A9000041D053781C0706D5254B196C00293ED041
:10A91000996C002939D09378190705D5204B196E09
:10A92000002936D0996E89B1D3781B0707D51C4B07
:10A93000D3F880207AB3D3F8882011213AB162B6D7
:10A94000184B00221A7030BC00F04ABE0D21154C85
:10A95000154D227843F8315003EBC1030830013A1A
:10A960005860227062B630BC704704220D4C0F4D07
:10A97000217843F8325003EBC20308304A1E586076
:10A98000227062B6EFE70521E1E70921DFE708223F
:10A99000ECE70C22EAE71022E8E700BF64000100C0
:10A9A0000080FF1F459EFF1FC80040008800400038
:10A9B000431E032B1DD81B4A400140F0100030B449
:10A9C000104472B6184CE25C032A1BD8DFE802F090
:10A9D0000212151703220D88E25410F0080F14BF5D
:10A9E000C823882343EA054308310360416062B607
:10A9F00030BC704708300222EDE70522EBE7083053
:10AA00000422E8E7094A52F8230038B1084A52F80C
:10AA10002300416042F8231062B6E9E742F82310B0
:10AA2000034AF7E70080FF1F549EFF1F1C9EFF1F75
:10AA30002C9EFF1F00BE70472DE9F04FDFF818B3C2
:10AA4000DFF818A387B044E0AD4F4FEA930807EB57
:10AA5000C809013ED9F8042003F00803F6B2A2F1B8
:10AA6000080003F0FF04002B40F0018157F8383054
:10AA70001B0C99B222F8081C002B00F0EF80A14BB0
:10AA800022F8064C42F8044C53F82620002A00F025
:10AA9000CF819D4D55F8263058609C4C45F82600D6
:10AAA00034F81630194424F8161000F079FD002807
:10AAB00000F0C281964A974B19F0080F00F1080088
:10AAC00018BF1346C9F8040047F8383008238BF83C
:10AAD00000309BF80040E4B265071CD58E4B1B7814
:10AAE000B3B18E490A7802F0FF0322B1013BDBB219
:10AAF0000B7003B900BE8A490A7802F0FF032AB13D
:10AB0000013BDBB20B70002B00F0688100F066FEA9
:10AB100004238BF8003004F0080303F0FF02002B3D
:10AB200000F0C9809AF80030DBB21E098CD19A0877
:10AB3000DFF8CC9159F8321009EBC200C1F3830160
:10AB4000013940680C2900F28580DFE801F07A7A4B
:10AB50008383838383834683838307000168714DE6
:10AB60004068714F714E6860296088B240F281611F
:10AB70000024674B49F832304FF0010E88423C60A8
:10AB8000C9F81040C9F8184086F800E05C4A00F2A5
:10AB9000E780B0F5D06F80F01B82B0F5817F00F0C8
:10ABA000D98100F26981802800F02A82822840F051
:10ABB000D781A98801F07F01042900F2D1815C4886
:10ABC0005C4A890008441470547001788C0740F185
:10ABD000608382F800E0022173E1534F3A682AB3A0
:10ABE000554B524E554819883478057840298E4681
:10ABF00045F0020828BF4FF0400E002C84F00104FD
:10AC00003470CEEB01010CBF8824C82409EBC806C0
:10AC100089B285F0010544EA0E447260198049F852
:10AC2000384072440570002965D03A603D4B1A885F
:10AC3000B2F5A06F0ED100219A785970404B1A706E
:10AC400008E038493F4C0D68A54200F09880304933
:10AC500049F832103C4A0123137037E72C4A2D4B38
:10AC600019F0080F18BF134647F838302EE700F0E8
:10AC7000B7FC364A364952F82630002B00F0E38004
:10AC800058688C5D42F8260003F10802C9F80420D8
:10AC9000032C05D8DFE804F02C02292602228A556D
:10ACA0001A8819F0080F0CBF8823C82343EA02430F
:10ACB00047F838300AE7E00700F19380210600F1F9
:10ACC000D180A20706D5234A234913780220DBB29C
:10ACD00013700870E30602D51F4B10221A7007B0DC
:10ACE000BDE8F08F04228A55DAE705228A55D7E7B6
:10ACF00003228A55D4E7BEF1400F18BF002294E723
:10AD00000080FF1FC89DFF1F749DFF1F0CA0FF1F29
:10AD1000C800400088004000509EFF1FD99DFF1FC3
:10AD2000C49EFF1F3C9EFF1F709DFF1FD89DFF1FED
:10AD3000C0200740489EFF1F849DFF1F449EFF1FA9
:10AD40009820074021090003942007401C9EFF1F04
:10AD5000549EFF1F88200740802007409020074016
:10AD6000B0F5106F00F07C8140F2A38040F6211214
:10AD7000904240F07B82A54A012313706AE74C6839
:10AD8000A3498C427FF463AF0178A9297FF45FAFB8
:10AD9000417845297FF45BAF8178C2297FF457AFB2
:10ADA000C1786B297FF453AF9A489B4E0178347871
:10ADB00081F00105002C41F0020105700CBF8820D4
:10ADC000C82084F0010449F8310009EBC10193481F
:10ADD0003470002505244D60047038E700F064FFEE
:10ADE00094E68F4B89488B491A614FF0020E80F828
:10ADF00000E08C4F0A708C49196099608B4E8C4D25
:10AE00008C4C9A610D213970FF213170DFF84CE2D2
:10AE100029702270884D894A8EF800109F270124DE
:10AE200006F8047C5D600470DA6007B0BDE8F08F5E
:10AE300043F82600824D30E6824A47F838001378FE
:10AE40000133137042E68B5D032B00F2BA8001A23E
:10AE500052F823F0CDAA0000CDAA0000ADAE00004C
:10AE6000A7AE00006F49724B80220D2008701A7047
:10AE7000A2077FF52FAF26E740F20232904240F062
:10AE8000ED81AA8802F07F02042A69D86D88002D1E
:10AE900066D16449CDF804E0920011440A7842F08A
:10AEA00002020A70C1E101238B550FE600238B5586
:10AEB0000CE6B0F5086F53D16349644A0978117004
:10AEC0007146ED888D4280F0E88252480478402D2A
:10AED000AE4644F0020C28BF4FF0400E02EB0E03CA
:10AEE00009EBCC01029301234A604FEA0E48CEEBF6
:10AEF000050101930025C82242EA080384F00102FB
:10AF000049F83C3035700270DFF814C1424BDFF86D
:10AF1000048149BBBEF1400F7FF42DAF42F0020C1B
:10AF200009EBCC03029ADFF8F8E05A608DBB0D0400
:10AF300045F088059DF804304EF83C500A443370C3
:10AF40000470134640297FF416AF0021404A3B604D
:10AF5000118010E7AA8802F07F02042A40F28B8158
:10AF6000304A0F23137006E74029D7D942F0020276
:10AF70000CEBC200029E4660BDB19DF804503548FE
:10AF80001D703346403988F8004040334CF8320099
:10AF9000DCE79DF8043033700D04029B047045F02B
:10AFA000C8050B444EF83C50CCE79DF804501D708A
:10AFB000029B1D4888F80040403940334CF832006D
:10AFC000C4E719F0080F0CBF022303238B557DE55E
:10AFD00021494A68002AC3D06C88B5F804E003E030
:10AFE0000C314A68002ABBD00B88A342F8D14B88A9
:10AFF0007345F5D1240A032C0CBF1178098960E749
:10B00000124A0221147054705BE700BF942007407D
:10B0100001000400449EFF1FD89DFF1FD99DFF1F04
:10B020000080FF1FC02007408800400088200740A4
:10B030008020074098200740889DFF1FDC9DFF1F50
:10B04000749DFF1F459EFF1F509EFF1F489EFF1FC0
:10B05000849DFF1FC8004000680001008C2007404D
:10B06000B248116AAC7804700C0600F19881D9F8E6
:10B070002820AF49100600F1DB81D9F83020AC4917
:10B08000120600F1D081D9F83820A949130600F141
:10B09000C581D9F84020A649150600F1BA81D9F832
:10B0A0004820A349140600F1AF81D9F85020A049E7
:10B0B000100600F1A481D9F858209D49120600F12C
:10B0C0009981D9F860209A49130600F18E81D9F848
:10B0D00068209749150600F18381D9F870209449BA
:10B0E000140600F17881D9F878209149100600F112
:10B0F0006D81D9F880208E49120600F16181D9F85E
:10B1000088208B49130600F15581D9F89020884991
:10B11000150600F14981D9F898208549140600F1F7
:10B12000FF808448844A854901908548854D864C36
:10B13000049700230596029580460F4616461D4645
:10B140000394306828B1446800F04AFA2046002C85
:10B15000F9D100233360029B38681A46002342F875
:10B16000253028B1446800F03BFA2046002CF9D184
:10B1700000223A60019A98F800301146002241F806
:10B18000042B039A0191023B4FF0000122F81510A5
:10B19000032B07D8DFE803F05D025D024FF00103E7
:10B1A00088F800300135042D06F1040607F1040784
:10B1B00008F10108C5D1654C654D2278654B049FA7
:10B1C000059E0021100729701A7000F192806249D3
:10B1D00062780A700021C9F83010C9F838101107D8
:10B1E000DFF84C816ED4A2785C49DFF844810A70A4
:10B1F00000211207C9F85010C9F858104BD4E27852
:10B2000057494B4C0A7013074FF00001C9F87010F2
:10B21000C9F8781000F1AE8033780193002283F0F2
:10B220000105C9F89020C9F89820002102918846AC
:10B230008E460A464B48047844F0020C09EBCC03D6
:10B240000393019B002B039B5A600CBF8822C822EA
:10B2500052E64FF0000388F80030A3E7B0F5A06F86
:10B260007FF47EAE012300250193DEE740F6212224
:10B270009042F7D074E66D88002D7FF471AE3A49A4
:10B28000CDF804E0920011440A7822F002020A701C
:10B29000CBE7022115E600F083F9002800F0EB80EF
:10B2A0000830324AC8F86400C8F8602000F078F925
:10B2B000002800F0DA8008302D4AC9F86C00C9F87F
:10B2C00068209CE700F06CF9002800F0E08008306E
:10B2D000264AC8F84400C8F8402000F061F9002868
:10B2E00000F0CF800830224AC9F84C00C9F8482045
:10B2F00079E700F055F9002800F0A58008301B4AD6
:10B30000C9F82400C9F8202000F04AF9002800F00C
:10B3100094800830164AC9F82C00C9F8282056E74E
:10B32000D1F89C00083800F05BF9FAE6509EFF1F48
:10B330000080FF1F2C9EFF1FC89DFF1F1C9EFF1F2C
:10B34000549EFF1F749DFF1F0CA0FF1F640001008F
:10B35000459EFF1FC4200740C8200740CC2007405F
:10B36000D0200740449EFF1FC020074088004000B7
:10B37000C800400000F014F9002870D008304F4A8F
:10B38000C4F88400C4F8802000F00AF9002860D0D6
:10B3900008304B4AC9F88C00C9F888203CE7506A4D
:10B3A000083800F01DF962E6D1F89400083800F082
:10B3B00017F9B0E6D1F88C00083800F011F9A4E6CE
:10B3C000D1F88400083800F00BF998E6C86F083807
:10B3D00000F006F98DE6486F083800F001F982E6C2
:10B3E000C86E083800F0FCF877E6486E083800F0C0
:10B3F000F7F86CE6C86D083800F0F2F861E6486DC1
:10B40000083800F0EDF856E6C86C083800F0E8F8A7
:10B410004BE6486C083800F0E3F840E6C86B0838A3
:10B4200000F0DEF835E6486B083800F0D9F82AE677
:10B43000C86A083800F0D4F81FE62A78C9F828004E
:10B4400001322A70C3E62A78C9F8200001322A7036
:10B450005AE72A78C9F8880001322A70DCE62A788F
:10B46000C4F8800001322A708EE72A78C9F8680093
:10B4700001322A70C3E62A78C8F8600001322A70C7
:10B4800014E72A78C9F8480001322A70ABE62A7816
:10B49000C8F8400001322A701FE740298E4628BFB5
:10B4A0004FF0400E02EB0E0302930123CEEB01019D
:10B4B0004FEA0E4800250193BCE600BF880040001B
:10B4C000C8004000F8B500F08FFD294B29482A4CF0
:10B4D0002A4F2B4DDFF8BCC0DFF8BCE0294E00221C
:10B4E0001A605A609A60DA601A615A619A61DA6188
:10B4F0001A625A629A62DA621A635A639A63DA6368
:10B500001A645A649A64DA641A655A659A65DA6547
:10B510001A665A669A66DA661A675A679A67DA6727
:10B52000C3F880200168C3F8842041F480210160C1
:10B53000C3F307212170C3F30740134938701B0E72
:10B540002B70FF238CF80030104D8EF8003010481F
:10B550000B700123337084F8642070264FF400745C
:10B56000102207F82C3C2E70046081F8F820F8BDFA
:10B570000080FF1F348004409C200740B02007401B
:10B58000B4200740942007401020074049E400E021
:10B5900008E100E08020074088200740704700BF96
:10B5A00072B60D480268B2FA82F30F2B10DC4FF02E
:10B5B0000041D94022EA0102026062B6074803EB6B
:10B5C000C303DB00C2180021C15010465160704710
:10B5D00062B60020704700BF3091FF1FBC83FF1F81
:10B5E0000D4B0E4AC31AA2FB03231B090F2B0CD8C9
:10B5F0000B4A127852B972B60A484FF000410268FD
:10B6000021FA03F31A43026062B67047064A1278C1
:10B61000002AF0D0FFF768B9BC83FF1F398EE338EA
:10B62000459EFF1F3091FF1F509EFF1F38B50E4BE8
:10B630000E4C1B68218805468BB1B1F5917F05D270
:10B640000B4A4B1C55549BB2238038BD002208483E
:10B6500098470021064A55540123238038BDB1F58F
:10B66000917FEDD338BD00BF7C9EFF1F16A0FF1F4A
:10B670001CA0FF1F2DE9F843214E224F3168012302
:10B6800080463B70B1B1204D4B8801EB8302013302
:10B6900000240F2BC2F808802C7004D84B800023A4
:10B6A0003B70BDE8F88340230B800320FFF780F94F
:10B6B0003460F4E7DFF8549099F80030002BF0D0B4
:10B6C000114D45F6215408E0013C12D02B7883B986
:10B6D00000F00AFB99F800307BB10320FFF7EEF889
:10B6E0000528F1D8FFF75CFF014630600028EBD059
:10B6F000CAE701232B70BDE8F883BDE8F88300BFDB
:10B70000989EFF1F6C9EFF1F9C9EFF1F509EFF1F59
:10B710001201F8B5D5B2A1B3012943D0437804464C
:10B7200000781B0643EA004040F4704045F00406F0
:10B730008F1E3043FFF79EFF022F04F1020314D93E
:10B74000053414F8023C14F8032C14F8010C1B0403
:10B7500043EA0223334343EA0060033FFFF78AFFD3
:10B76000022F234604F10304EBD8022F23D0012F2C
:10B770000DD045F4774040F00500BDE8F840FFF7F4
:10B7800079BF14482843BDE8F840FFF773BF187825
:10B7900045F4770545F0060545EA0020BDE8F84088
:10B7A000FFF768BF03780C4845EA03452843BDE826
:10B7B000F840FFF75FBF1A78587845F0774545F0B5
:10B7C000070545EA022545EA0040BDE8F840FFF7D5
:10B7D00051BF00BF06F0F70007F000F738B5084B7F
:10B7E0001C7824B9074D296809B14B8803B938BDC5
:10B7F0009B000B800320FFF7DBF82C6038BD00BFF7
:10B800006C9EFF1F989EFF1F2DE9F041AD4E3368DF
:10B810000746002B00F092801D885A88910803EBA0
:10B8200081010432AA428C6842D25A8004F00F0689
:10B830004FEA1428A449A6F1080208F00F00C4F347
:10B840000313062A00F101050B701AD9B31E012B50
:10B850005FFA88F04ED9052E48D0042E00F0A4815E
:10B86000731F022B7FD90F2E0ED1F72842D8F02854
:10B8700002D0964B1B883BB1FFF7D8FE0020BDE8F5
:10B88000F08127B1BD4202D00020BDE8F081082E32
:10B89000C4F3033300F08780092E11D00A2E40F044
:10B8A00094800A2BF0D18A4B8A4A1B68A02181E040
:10B8B0001846FFF795FE0420FEF7E2FF3060B5E77B
:10B8C000092BE1D1270E00F07B81834B814A1B6855
:10B8D0009021C4F307461170EDB2FCB2002B00F0CA
:10B8E0009D80224631462846984797E0F02843D964
:10B8F000F72841D0F1380E28C6D801A353F820F01C
:10B90000B7BA00009BBA000089BA000089B80000ED
:10B9100089B800007BBA000089B800005BBB00005A
:10B9200089B8000025BB00003FBB000063BA0000DF
:10B9300089B800004BBA00002FBA0000674B1B7893
:10B94000002BA1D00420FEF79BFF034630600028A7
:10B950009AD00588002D7FF460AFFFF741FE356077
:10B960002846BDE8F081FFF761FEC4F30740FFF70A
:10B970005DFE072E02D1200EFFF758FE534B584AAA
:10B98000198858481468584D524A017000270E0A09
:10B99000F0201F802E7010700CB301225348A04776
:10B9A0000120BDE8F081082B7FF46EAF504B494A6F
:10B9B0001B688021C4F307461170EDB2240E6BB3EF
:10B9C000284622463146984728E00B2E11D10B2BF2
:10B9D0007FF45AAF474B3F4A1B68B021EAE7464B1A
:10B9E0001B68002B00F0FB80404898470120BDE811
:10B9F000F0810C2E40F000810C2B7FF445AF3F4BC3
:10BA0000344A1B68C0211170EDB2C4F30746002B05
:10BA100000F0C88028463146240E98473849314AFC
:10BA2000314B0D7016701C700120BDE8F081354B54
:10BA30001B68002B00F0D6809847C4F30746254BBF
:10BA4000EDB2240E83F80080E8E72F4B1B68002B33
:10BA5000F2D12E4B1B68A3B1FE209847C4F30746D2
:10BA6000EDE72B4B1B68002BE6D1284B1B6843B13D
:10BA7000FC209847C4F30746E1E7264B1B68002BE0
:10BA8000DAD1C4F30746DAE7234B1B68C4F3074651
:10BA9000002BD4D030469847D1E7204B1A68002AB3
:10BAA000EFD0260C630C06F07F0003F47E5318439E
:10BAB000F6B29047C3E71A4B1B68C4F30746002B46
:10BAC000E8D1BCE7A49EFF1F1AA0FF1F16A0FF1F0E
:10BAD000809EFF1F14A0FF1FB49EFF1F509EFF1FDC
:10BAE0007C9EFF1F18A0FF1F19A0FF1F1CA0FF1F97
:10BAF000AC9EFF1FB09EFF1F949EFF1F709EFF1FF6
:10BB00001BA0FF1F5C9EFF1F609EFF1F649EFF1F08
:10BB1000A09EFF1F909EFF1FA89EFF1F789EFF1FE5
:10BB20008C9EFF1F3F4B1B68002B85D13E4B1B6833
:10BB3000002BA6D0FA209847C4F307467FE73B4B7B
:10BB40001B68002B7FF478AF374B1B68002B98D015
:10BB5000FB209847C4F3074671E7354B1B68002B61
:10BB60007FF46AAF304B1B68002B8AD0F8209847CF
:10BB7000C4F3074663E70E2B7FF486AE2D4A2E4BA7
:10BB80001268E0211970002A47D0260C610C06F0DB
:10BB90007F0301F47E511943EDB2A1F5005128460F
:10BBA0009047F6B2240E39E7FFF740FDC4F3074093
:10BBB000FFF73CFD200EFFF739FD0020BDE8F081C6
:10BBC0001E4B1D4A1B6880211170EDB2C4F307465D
:10BBD00083B1314628463A4698473C461EE7012045
:10BBE000BDE8F081104B1B68002B3FF44AAFFF20EB
:10BBF000984746E71C4611E70D2EBCD10D2B7FF46C
:10BC000043AE0F4B0C4A1B68D0211170EDB2C4F348
:10BC10000746002B7FF4FEAEC4E7C4F30746EDB23F
:10BC2000240EFBE6889EFF1F649EFF1F689EFF1F79
:10BC3000589EFF1F749EFF1F14A0FF1FAC9EFF1F86
:10BC4000849EFF1F38B5164D2868E0B101884488EE
:10BC5000A14213DD03191B7A83B104F10803C21852
:10BC60000C1B002302E012F8011F21B10133A34293
:10BC7000F9D1204638BD1C46204638BDFFF7B0FC40
:10BC80000020286038BD074B1B780BB9002038BD59
:10BC90000220FEF7F5FD28600028D7D1F6E700BFA7
:10BCA000C09EFF1F509EFF1F0D4B1B78BBB910B5E8
:10BCB0000C4C216803F0FF024B883F2B07DC073355
:10BCC0000B4401F1470003F8012F8342FBD14023CD
:10BCD0000B800120FEF76CFE0023236010BD70472F
:10BCE000B89EFF1FBC9EFF1F38B5224C237803B1BE
:10BCF00038BD01232370FFF7A5FF70BB00F048F8A3
:10BD000040BB00F0DBF810BBFEF7F8FCE0B9002305
:10BD10002370EFF30583002BEAD1EFF3108172B6A5
:10BD2000154B1868E0B1154C2278CAB945691D60F9
:10BD300001232370C5B1AA6101B962B60025457718
:10BD4000836898472570D3E700F020F8DFE700F01C
:10BD50001BF8D9E700F016F8D3E7FFF71FFCCDE793
:10BD60000029C5D162B638BD054B1D600029E5D15B
:10BD7000E3E700BFC59EFF1FDC9CFF1FE09CFF1F89
:10BD8000D89CFF1F704700BF704700BF704700BFBF
:10BD9000054A064B10781B78C0B2DBB2984238BF18
:10BDA0004030C01A704700BFCC9EFF1FCD9EFF1FC2
:10BDB000F0B4384B1A7912F0300F2CD072B6997D4E
:10BDC00001F0FF0200293DD062B6334F3349387885
:10BDD0000D78334E1C46C0B2EDB2431C402BE179C6
:10BDE00028BF0023AB4202F1FF32C9B21CBFF1549D
:10BDF000184612F0FF02F0D12A4B1B68C2B23A700B
:10BE00004BB1A84236BFC5F14005401B4019272859
:10BE1000C4BF01221A701F49CA78D2B2150616D4BF
:10BE200052060DD51B4B1B795B0609D51E4B1F49CE
:10BE30001B6800220A7003B11A70164B3C22DA709C
:10BE4000F0BC70474022D9795A7462B6E3E70B79A7
:10BE50001C06E5D5164B174E1C783378E4B2DBB2DE
:10BE60009C420ED0144D01E0A3420AD00133402B76
:10BE700028BF00230879E85CC0B2C871087D072894
:10BE8000F2D9DBB2034933700B79180644BF7C2327
:10BE9000CB70C5E700A00640CC9EFF1FCD9EFF1FC4
:10BEA000109FFF1FC89EFF1F549FFF1F509FFF1F23
:10BEB000589FFF1F519FFF1FD09EFF1F054A064B33
:10BEC00010781B78C0B2DBB2984238BF4030C01A3D
:10BED000704700BFCC9FFF1F619FFF1FF0B4384B1E
:10BEE0001A7912F0300F2CD072B6997D01F0FF0252
:10BEF00000293DD062B6334F334938780D78334E40
:10BF00001C46C0B2EDB2431C402BE17928BF002390
:10BF1000AB4202F1FF32C9B21CBFF154184612F015
:10BF2000FF02F0D12A4B1B68C2B23A704BB1A84253
:10BF300036BFC5F14005401B40192728C4BF012268
:10BF40001A701F49CA78D2B2150616D452060DD5FA
:10BF50001B4B1B795B0609D51E4B1F491B68002232
:10BF60000A7003B11A70164B3C22DA70F0BC7047AD
:10BF70004022D9795A7462B6E3E70B791C06E5D5FD
:10BF8000164B174E1C783378E4B2DBB29C420ED0CD
:10BF9000144D01E0A3420AD00133282B28BF00230F
:10BFA0000879E85CC0B2C871087D0728F2D9DBB215
:10BFB000034933700B79180644BF7C23CB70C5E767
:10BFC00000B00640CC9FFF1F619FFF1F8C9FFF1F8B
:10BFD0005C9FFF1FD09FFF1F609FFF1FD49FFF1F0D
:10BFE000CD9FFF1F649FFF1F70B584B072B6194BC1
:10BFF000194D1A48702241260F2480211A702E7084
:10C000001A460470197013781B06FCD5144B186877
:10C0100062B6144B144C984298BF00EB800001A903
:10C0200098BF40000A22FDF7CFFE01A92046002359
:10C0300011F8012B01333AB10A2B20F8022FF7D166
:10C040001623237004B070BD5B00DBB2237004B014
:10C0500070BD00BF00000240070002400600024021
:10C06000080002407F969800FC91FF1FFFFFFFFF32
:10C070002DE9F043DFF8EC808BB006460F4600F068
:10C0800073F898F90030013304460D4637D0304636
:10C09000394600F0DFF9002831D02BA3D3E9002383
:10C0A0003046394600F026FE814668BB28A3D3E916
:10C0B00000233046394600F0FFFD00B398F9003008
:10C0C000254ACDF82090042400200021022BCDE940
:10C0D0000467CDE9026700940192CDE906012CD0F6
:10C0E000684600F0BDF940B3089B1BB101F0AAF906
:10C0F000089B0360DDE906010BB0BDE8F083204634
:10C1000029460BB0BDE8F083134A98F9003001923C
:10C1100003210022CDE90467CDE90267009108926E
:10C120002BB90E4B4FF06042CDE90623D8E70C49FE
:10C130000020022BCDE90601D2D101F083F92223A0
:10C140000360D1E7AFF30080EF39FAFE422E86405C
:10C1500051302DD5104987C0D4000100FFFFEF47B3
:10C160000000F07F1292FF1F2DE9F04FB04F21F039
:10C170000042BA4283B00C464FEAD17605460DD94B
:10C18000AC4FBA4225D9C1F31303034340F0EF800B
:10C190000EB10020014603B0BDE8F08FA64B9A42D5
:10C1A00000F2CC80A54B9A4200F2DE808AA3D3E94C
:10C1B000002300F05DF90022A14B00F09BFD002858
:10C1C00000F005812846214600229D4B00F050F9E1
:10C1D000E1E783A3D3E9002300F08CFD002840F0C1
:10C1E000CB802846214680A3D3E9002300F064FDDC
:10C1F0000028CED1934B284603EBC60821467CA3EA
:10C20000D3E9002300F0E6FAD8E9002300F030F982
:10C2100000F07AFD804600F077FA77A3D3E9002397
:10C2200006460F4600F0D6FA02460B46284621463F
:10C2300000F01CF972A3D3E90023CDE900013046D8
:10C24000394600F0C7FA82468B4652465B46DDE926
:10C25000000100F00BF905460C462A462346284605
:10C26000214600F0B7FA68A3D3E9002306460F463B
:10C2700000F0B0FA66A3D3E9002300F0F7F83246E5
:10C280003B4600F0A7FA64A3D3E9002300F0F0F8DE
:10C2900032463B4600F09EFA61A3D3E9002300F04A
:10C2A000E5F832463B4600F095FA5FA3D3E9002358
:10C2B00000F0DEF832463B4600F08CFA02460B46B0
:10C2C0002846214600F0D2F806460F462846214669
:10C2D00032463B46B8F1000F56D000F07BFA3246AA
:10C2E00004460D463B4600204FF0804100F0BEF86A
:10C2F00002460B462046294600F096FB02460B46B6
:10C300005046594600F0B2F8DDE9002300F0AEF8DF
:10C310000B4602464A49002000F0A8F86FF47F73EC
:10C3200098454FDA08F57A7801EB085100224FF072
:10C33000B87300F04FFA03B0BDE8F08F424B9A4259
:10C340003FF658AF414BF4002344D3E9002300F0FB
:10C350008DF83F4BC6F101081C44CDE90001D4E93A
:10C3600000ABC6EB080870E74FF0000875E702461F
:10C370000B4600F07DF80EE717A3D3E90023104623
:10C38000194600F027FA06E700F024FA002280465A
:10C3900089464FF080433046394600F067F8024640
:10C3A0000B464046494600F03FFB2A46234600F034
:10C3B0005DF802460B460020214900F057F803B013
:10C3C000BDE8F08F01EB085103B0BDE8F08F804667
:10C3D00043E700BFAFF300809C7500883CE4377EE4
:10C3E000EF39FAFE422E864051302DD5104987C0D4
:10C3F000FE822B654715F73F0000E0FE422EE63F28
:10C40000763C7935EF39EA3DD0A4BE726937663E95
:10C41000F16BD2C541BDBB3E2CDE25AF6A56113F44
:10C4200093BDBE166CC1663F3E5555555555C53F2B
:10C43000412E8640FFFFEF7F422ED63FFFFF2F3E6B
:10C440000000F03FD8000100B1A2F03FF800010069
:10C45000E800010041F0004101F58010C00F704775
:10C460000020704781F0004102E000BF83F00043EC
:10C4700030B54FEA41044FEA430594EA050F08BF7F
:10C4800090EA020F1FBF54EA000C55EA020C7FEA43
:10C49000645C7FEA655C00F0E2804FEA5454D4EBC0
:10C4A0005555B8BF6D420CDD2C4480EA020281EA8A
:10C4B000030382EA000083EA010180EA020281EAC2
:10C4C0000303362D88BF30BD11F0004F4FEA013114
:10C4D0004FF4801C4CEA113102D0404261EB410123
:10C4E00013F0004F4FEA03334CEA133302D05242A9
:10C4F00063EB430394EA050F00F0A780A4F1010465
:10C50000D5F1200E0DDB02FA0EFC22FA05F280189E
:10C5100041F1000103FA0EF2801843FA05F3594184
:10C520000EE0A5F120050EF1200E012A03FA0EFC03
:10C5300028BF4CF0020C43FA05F3C01851EBE3712D
:10C5400001F0004507D54FF0000EDCF1000C7EEB4A
:10C5500000006EEB0101B1F5801F1BD3B1F5001F88
:10C560000CD349085FEA30004FEA3C0C04F10104A7
:10C570004FEA445212F5800F80F09A80BCF1004FD0
:10C5800008BF5FEA500C50F1000041EB045141EA52
:10C59000050130BD5FEA4C0C404141EB010111F453
:10C5A000801FA4F10104E9D191F0000F04BF0146FE
:10C5B0000020B1FA81F308BF2033A3F10B03B3F1DC
:10C5C00020020CDA0C3208DD02F1140CC2F10C026C
:10C5D00001FA0CF021FA02F10CE002F11402D8BFCA
:10C5E000C2F1200C01FA02F120FA0CFCDCBF41EA96
:10C5F0000C019040E41AA2BF01EB0451294330BD65
:10C600006FEA04041F3C1CDA0C340EDC04F1140441
:10C61000C4F1200220FA04F001FA02F340EA030018
:10C6200021FA04F345EA030130BDC4F10C04C4F15E
:10C63000200220FA02F001FA04F340EA030029463E
:10C6400030BD21FA04F0294630BD94F0000F83F488
:10C65000801306BF81F480110134013D4EE77FEA6B
:10C66000645C18BF7FEA655C29D094EA050F08BFB7
:10C6700090EA020F05D054EA000C04BF1946104698
:10C6800030BD91EA030F1EBF0021002030BD5FEADC
:10C69000545C05D14000494128BF41F0004130BD04
:10C6A00014F580043CBF01F5801130BD01F0004558
:10C6B00045F0FE4141F470014FF0000030BD7FEACB
:10C6C000645C1ABF194610467FEA655C1CBF0B46C6
:10C6D000024650EA013406BF52EA033591EA030FDD
:10C6E00041F4002130BD00BF90F0000F04BF0021D5
:10C6F000704730B54FF4806404F132044FF0000508
:10C700004FF0000150E700BF90F0000F04BF002180
:10C71000704730B54FF4806404F1320410F00045E6
:10C7200048BF40424FF000013EE700BF42004FEAE1
:10C73000E2014FEA31014FEA02701FBF12F07F435E
:10C7400093F07F4F81F06051704792F0000F14BF5B
:10C7500093F07F4F704730B54FF4607401F000459F
:10C7600021F0004120E700BF50EA010208BF7047F6
:10C7700030B54FF000050AE050EA010208BF7047EB
:10C7800030B511F0004502D5404261EB41014FF454
:10C79000806404F132045FEA915C3FF4DCAE4FF058
:10C7A00003025FEADC0C18BF03325FEADC0C18BF3F
:10C7B000033202EBDC02C2F1200300FA03FC20FA90
:10C7C00002F001FA03FE40EA0E0021FA02F11444DD
:10C7D000C1E600BF70B54FF0FF0C4CF4E06C1CEAF2
:10C7E00011541DBF1CEA135594EA0C0F95EA0C0F67
:10C7F00000F0DEF82C4481EA030621EA4C5123EADA
:10C800004C5350EA013518BF52EA033541F4801108
:10C8100043F4801338D0A0FB02CE4FF00005E1FBBB
:10C8200002E506F00042E0FB03E54FF00006E1FB05
:10C8300003569CF0000F18BF4EF0010EA4F1FF0448
:10C84000B6F5007F64F5407404D25FEA4E0E6D4188
:10C8500046EB060642EAC62141EA55514FEAC52099
:10C8600040EA5E504FEACE2EB4F1FD0C88BFBCF515
:10C87000E06F1ED8BEF1004F08BF5FEA500E50F1C6
:10C88000000041EB045170BD06F0004646EA01018C
:10C8900040EA020081EA0301B4EB5C04C2BFD4EBBE
:10C8A0000C0541EA045170BD41F480114FF0000EB7
:10C8B000013C00F3AB8014F1360FDEBF002001F025
:10C8C000004170BDC4F10004203C35DA0C341BDC9F
:10C8D00004F11404C4F1200500FA05F320FA04F071
:10C8E00001FA05F240EA020001F0004221F00041A5
:10C8F00010EBD37021FA04F642EB06015EEA430E18
:10C9000008BF20EAD37070BDC4F10C04C4F1200547
:10C9100000FA04F320FA05F001FA04F240EA0200FA
:10C9200001F0004110EBD37041F100015EEA430ECB
:10C9300008BF20EAD37070BDC4F1200500FA05F2EB
:10C940004EEA020E20FA04F301FA05F243EA02036A
:10C9500021FA04F001F0004121FA04F220EA020079
:10C9600000EBD3705EEA430E08BF20EAD37070BDBF
:10C9700094F0000F0FD101F00046400041EB01019F
:10C9800011F4801F08BF013CF7D041EA060195F081
:10C99000000F18BF704703F00046520043EB03033B
:10C9A00013F4801F08BF013DF7D043EA0603704728
:10C9B00094EA0C0F0CEA135518BF95EA0C0F0CD033
:10C9C00050EA410618BF52EA4306D1D181EA030179
:10C9D00001F000414FF0000070BD50EA410606BF73
:10C9E0001046194652EA430619D094EA0C0F02D1B8
:10C9F00050EA013613D195EA0C0F05D152EA0336FD
:10CA00001CBF104619460AD181EA030101F000411A
:10CA100041F0FE4141F470014FF0000070BD41F063
:10CA2000FE4141F4780170BD70B54FF0FF0C4CF43D
:10CA3000E06C1CEA11541DBF1CEA135594EA0C0F5C
:10CA400095EA0C0F00F0A7F8A4EB050481EA030EA9
:10CA500052EA03354FEA013100F088804FEA033390
:10CA60004FF0805545EA131343EA12634FEA02225E
:10CA700045EA111545EA10654FEA00260EF000411F
:10CA80009D4208BF964244F1FD0404F5407402D271
:10CA90005B084FEA3202B61A65EB03055B084FEA02
:10CAA00032024FF480104FF4002CB6EB020E75EBFF
:10CAB000030E22BFB61A754640EA0C005B084FEA27
:10CAC0003202B6EB020E75EB030E22BFB61A7546A4
:10CAD00040EA5C005B084FEA3202B6EB020E75EBEF
:10CAE000030E22BFB61A754640EA9C005B084FEA67
:10CAF0003202B6EB020E75EB030E22BFB61A754674
:10CB000040EADC0055EA060E18D04FEA051545EA62
:10CB100016754FEA06164FEAC30343EA52734FEA0B
:10CB2000C2025FEA1C1CC0D111F4801F0BD141EA84
:10CB300000014FF000004FF0004CB6E711F4801FE9
:10CB400004BF01430020B4F1FD0C88BFBCF5E06FC9
:10CB50003FF6AFAEB5EB030C04BFB6EB020C5FEAD9
:10CB6000500C50F1000041EB045170BD0EF0004E2E
:10CB70004EEA113114EB5C04C2BFD4EB0C0541EA60
:10CB8000045170BD41F480114FF0000E013C90E65D
:10CB900045EA060E8DE60CEA135594EA0C0F08BF21
:10CBA00095EA0C0F3FF43BAF94EA0C0F0AD150EA20
:10CBB00001347FF434AF95EA0C0F7FF425AF1046B3
:10CBC00019462CE795EA0C0F06D152EA03353FF4DB
:10CBD000FDAE1046194622E750EA410618BF52EA58
:10CBE00043067FF4C5AE50EA41047FF40DAF52EA2C
:10CBF00043057FF4EBAE12E74FF0FF3C06E000BFC9
:10CC00004FF0010C02E000BF4FF0010C4DF804CDD5
:10CC10004FEA410C7FEA6C5C4FEA430C18BF7FEA95
:10CC20006C5C1BD001B050EA410C0CBF52EA430CC3
:10CC300091EA030F02BF90EA020F0020704710F143
:10CC4000000F91EA030F58BF994208BF90422CBFD2
:10CC5000D8176FEAE37040F0010070474FEA410CCB
:10CC60007FEA6C5C02D150EA013C07D14FEA430CE9
:10CC70007FEA6C5CD6D152EA033CD3D05DF8040B5A
:10CC8000704700BF8446104662468C46194663468C
:10CC900000E000BF01B5FFF7B7FF002848BF10F163
:10CCA000000F01BD4DF808EDFFF7F4FF0CBF0120A8
:10CCB00000205DF808FB00BF4DF808EDFFF7EAFF24
:10CCC00034BF012000205DF808FB00BF4DF808EDDF
:10CCD000FFF7E0FF94BF012000205DF808FB00BFD4
:10CCE0004DF808EDFFF7CEFF94BF012000205DF85E
:10CCF00008FB00BF4DF808EDFFF7C4FF34BF01206B
:10CD000000205DF808FB00BF4FEA410212F5001257
:10CD100015D211D56FF47873B3EB625212D94FEA82
:10CD2000C12343F0004343EA505311F0004F23FA6C
:10CD300002F018BF404270474FF00000704750EAC1
:10CD4000013005D111F0004008BF6FF0004070477E
:10CD50004FF00000704700BF4FEA4102B2F1E043DC
:10CD600024BFB3F5001CDCF1FE5C0DD901F0004CD2
:10CD70004FEAC0024CEA5070B2F1004F40EB830022
:10CD800008BF20F00100704711F0804F21D113F14E
:10CD90003872BCBF01F00040704741F480114FEA87
:10CDA0005252C2F11802C2F1200C10FA0CF320FA10
:10CDB00002F018BF40F001004FEAC1234FEAD3232D
:10CDC00003FA0CFC40EA0C0023FA02F34FEA430397
:10CDD000CCE77FEA625307D150EA01331EBF4FF020
:10CDE000FE4040F44000704701F0004040F0FE403B
:10CDF00040F40000704700BF80F0004002E000BF38
:10CE000081F0004142001FBF5FEA410392EA030F35
:10CE10007FEA226C7FEA236C6AD04FEA1262D2EB7F
:10CE20001363C1BFD218414048404140B8BF5B4284
:10CE3000192B88BF704710F0004F40F4000020F01D
:10CE40007F4018BF404211F0004F41F4000121F033
:10CE50007F4118BF494292EA030F3FD0A2F101027D
:10CE600041FA03FC10EB0C00C3F1200301FA03F1BB
:10CE700000F0004302D5494260EB4000B0F5000FDE
:10CE800013D3B0F1807F06D340084FEA310102F19D
:10CE90000102FE2A51D2B1F1004F40EBC25008BF4F
:10CEA00020F0010040EA03007047490040EB000019
:10CEB00010F4000FA2F10102EDD1B0FA80FCACF148
:10CEC000080CB2EB0C0200FA0CF0AABF00EBC25047
:10CED00052421843BCBFD0401843704792F0000F35
:10CEE00081F4000106BF80F400000132013BB5E788
:10CEF0004FEA41037FEA226C18BF7FEA236C21D0FE
:10CF000092EA030F04D092F0000F08BF0846704762
:10CF100090EA010F1CBF0020704712F07F4F04D130
:10CF2000400028BF40F00040704712F100723CBF43
:10CF300000F50000704700F0004343F0FE4040F46D
:10CF4000000070477FEA226216BF08467FEA23632B
:10CF50000146420206BF5FEA412390EA010F40F416
:10CF6000800070474FF0000304E000BF10F0004362
:10CF700048BF40425FEA000C08BF704743F0964349
:10CF800001464FF000001CE050EA010208BF704764
:10CF90004FF000030AE000BF50EA010208BF7047EB
:10CFA00011F0004302D5404261EB41015FEA010C00
:10CFB00002BF84460146002043F0B64308BFA3F1F8
:10CFC0008053A3F50003BCFA8CF2083AA3EBC253DA
:10CFD00010DB01FA02FC634400FA02FCC2F12002F9
:10CFE000BCF1004F20FA02F243EB020008BF20F030
:10CFF0000100704702F1200201FA02FCC2F1200296
:10D0000050EA4C0021FA02F243EB020008BF20EA8A
:10D01000DC7070474FF0FF0C1CEAD0521EBF1CEAB8
:10D02000D15392EA0C0F93EA0C0F6FD01A4480EAA6
:10D03000010C400218BF5FEA41211ED04FF000638F
:10D0400043EA501043EA5111A0FB01310CF00040BB
:10D05000B1F5000F3EBF490041EAD3715B0040EAE1
:10D06000010062F17F02FD2A1DD8B3F1004F40EBB1
:10D07000C25008BF20F00100704790F0000F0CF084
:10D08000004C08BF49024CEA502040EA51207F3A48
:10D09000C2BFD2F1FF0340EAC250704740F4000023
:10D0A0004FF00003013A5DDC12F1190FDCBF00F014
:10D0B00000407047C2F10002410021FA02F1C2F1C2
:10D0C000200200FA02FC5FEA310040F1000053EA5E
:10D0D0004C0308BF20EADC70704792F0000F00F0AC
:10D0E000004C02BF400010F4000F013AF9D040EAB2
:10D0F0000C0093F0000F01F0004C02BF490011F446
:10D10000000F013BF9D041EA0C018FE70CEAD15343
:10D1100092EA0C0F18BF93EA0C0F0AD030F0004CC3
:10D1200018BF31F0004CD8D180EA010000F0004077
:10D13000704790F0000F17BF90F0004F084691F035
:10D14000000F91F0004F14D092EA0C0F01D142026F
:10D150000FD193EA0C0F03D14B0218BF084608D138
:10D1600080EA010000F0004040F0FE4040F4000082
:10D17000704740F0FE4040F4400070474FF0FF0C15
:10D180001CEAD0521EBF1CEAD15392EA0C0F93EA5C
:10D190000C0F69D0A2EB030280EA010C49024FEAAE
:10D1A000402037D04FF0805343EA111143EA101367
:10D1B0000CF000408B4238BF5B0042F17D024FF41F
:10D1C000000C8B4224BF5B1A40EA0C00B3EB510FFA
:10D1D00024BFA3EB510340EA5C00B3EB910F24BFE3
:10D1E000A3EB910340EA9C00B3EBD10F24BFA3EB68
:10D1F000D10340EADC001B0118BF5FEA1C1CE0D130
:10D20000FD2A3FF650AF8B4240EBC25008BF20F0E2
:10D21000010070470CF0004C4CEA50207F32C2BF36
:10D22000D2F1FF0340EAC250704740F400004FF0D3
:10D230000003013A37E792F0000F00F0004C02BF04
:10D24000400010F4000F013AF9D040EA0C0093F0CE
:10D25000000F01F0004C02BF490011F4000F013B28
:10D26000F9D041EA0C0195E70CEAD15392EA0C0F90
:10D2700008D142027FF47DAF93EA0C0F7FF470AFC8
:10D28000084676E793EA0C0F04D14B023FF44CAF0B
:10D2900008466EE730F0004C18BF31F0004CCAD1A0
:10D2A00030F000427FF45CAF31F000437FF43CAFDC
:10D2B0005FE700BF4FF0FF3C06E000BF4FF0010CFE
:10D2C00002E000BF4FF0010C4DF804CD4FEA4002E0
:10D2D0004FEA41037FEA226C18BF7FEA236C11D02A
:10D2E00001B052EA530C18BF90EA010F58BFB2EBDD
:10D2F000030088BFC81738BF6FEAE17018BF40F05D
:10D30000010070477FEA226C02D15FEA402C05D110
:10D310007FEA236CE4D15FEA412CE1D05DF8040B95
:10D32000704700BF844608466146FFE70FB5FFF728
:10D33000C9FF002848BF10F1000F0FBD4DF808EDE0
:10D34000FFF7F4FF0CBF012000205DF808FB00BFD1
:10D350004DF808EDFFF7EAFF34BF012000205DF82B
:10D3600008FB00BF4DF808EDFFF7E0FF94BF012078
:10D3700000205DF808FB00BF4DF808EDFFF7D2FF75
:10D3800094BF012000205DF808FB00BF4DF808EDB8
:10D39000FFF7C8FF34BF012000205DF808FB00BF85
:10D3A0004FEA4002B2F1FE4F0FD34FF09E03B3EBB2
:10D3B00012620DD94FEA002343F0004310F0004FF2
:10D3C00023FA02F018BF404270474FF00000704748
:10D3D00012F1610F01D1420205D110F0004008BFE7
:10D3E0006FF0004070474FF00000704742000ED2CF
:10D3F000B2F1FE4F0BD34FF09E03B3EB126209D490
:10D400004FEA002343F0004323FA02F070474FF045
:10D410000000704712F1610F01D1420202D14FF0BA
:10D42000FF3070474FF00000704700BF0B460146C9
:10D43000184600F001B800BF13460A460146022014
:10D4400000F0B0BE014B1868704700BF4096FF1F48
:10D4500070B50F4E0F4D761BB61018BF002405D0C7
:10D46000013455F8043B9847A642F9D10A4E0B4DBA
:10D47000761B02F04BFEB61018BF002406D0013414
:10D4800055F8043B9847A642F9D170BD70BD00BF66
:10D4900018010100180101002C0101001801010010
:10D4A000024B0146186800F00BB800BF4096FF1F02
:10D4B000024B0146186800F039BF00BF4096FF1FBD
:10D4C0002DE9F04F01F10B05162D83B0064640F211
:10D4D0009F8035F0070500F1BF80A94200F2BC80B3
:10D4E00000F058FBB5F5FC7FC0F09C826B0A00F0A1
:10D4F000BA80042B00F28381A80900F1390E4FEAAB
:10D500004E033830C44F07EB8303A3F108015C6876
:10D51000A14207D1ACE0002A80F2AC80E468A142CD
:10D5200000F0A680636823F003035A1B0F2AF2DD84
:10D53000B9493C6901F1080E744500F0B381636894
:10D5400023F003035A1B0F2A00F39981002AC1F824
:10D5500014E0C1F810E080F29E80B3F5007F80F007
:10D560006781DB0803F1010C01229B1002FA03F32F
:10D570004A6851F83C80C4F8088001EBCC091A4392
:10D58000A9F10803E3604A6041F83C40C8F80C4048
:10D59000831001249C40944200F28A80144206D1F8
:10D5A00020F003006400144200F10400FAD007EBFD
:10D5B000C009CC468046DCF80C108C4507D173E1DD
:10D5C000002A80F28181C9688C4500F06D814B682A
:10D5D00023F003035A1B0F2AF2DD0C46D1F80CC0CE
:10D5E00054F8088F4B1945F001054D6042F00101D8
:10D5F000C8F80CC03046CCF808807B613B61C3F8AA
:10D600000CE0C3F808E059609A5000F0C5FA1FE03A
:10D61000102921D800F0BEFA1025062302207E4FE3
:10D6200007EB8303A3F108025C68944200F0458194
:10D630006368E168A56823F00303234430465A6811
:10D64000E96042F001028D605A6000F0A5FA0834EA
:10D65000204603B0BDE8F08F00240C232046336041
:10D6600003B0BDE8F08F80234FF0400E3F2049E724
:10D6700070465DE72344E1685A68A56842F00102FC
:10D68000E96030468D605A6000F086FA0834204622
:10D6900003B0BDE8F08F234430465A6842F00102DF
:10D6A0005A6000F079FA0834204603B0BDE8F08FE4
:10D6B000BC68636823F00308A84504D3C5EB0803DE
:10D6C0000F2B00F38C80554BDFF860911A68D9F866
:10D6D000003001332A4404EB080A00F0608102F5AF
:10D6E00080520F3222F47F6222F00F021146304640
:10D6F000019200F04BFCB0F1FF3F8346019A00F02D
:10D700005881824500F2FC80454B1968DA45114486
:10D71000196000F05381D9F80000DFF810E1013002
:10D720001BBFCAEB0B0A5144CEF800B019601BF0C6
:10D73000070100F01781C1F10800C1F58051834451
:10D7400008315A44C2F30B02C2EB01094946304684
:10D75000019300F01BFC431C019B00F03F81CBEBCD
:10D7600000024A4442F001021968C7F808B049446F
:10D77000BC42CBF804201960DFF8A49016D0B8F1B1
:10D780000F0F40F2FD806268A8F10C0323F007033D
:10D79000E01802F001024FF0050E1A430F2B6260F1
:10D7A000C0F804E0C0F808E000F21C811D4BBC6822
:10D7B0001A68914288BF19601B4B1A6891426268CF
:10D7C00088BF196022F003029542A2EB050301D83D
:10D7D0000F2B04DC304600F0DFF9002438E7621933
:10D7E00043F0010345F0010565603046BA605360BF
:10D7F00000F0D2F90834204603B0BDE8F08F142BB6
:10D8000071D9542B00F2A480280B00F16F0E4FEA5F
:10D810004E036E3076E600BF4496FF1FE09FFF1F69
:10D82000E49FFF1FDC9FFF1FD89FFF1F509AFF1F21
:10D830005A0A042A5ED9142A00F2B38002F15C016C
:10D8400049005B3207EB810C57F82110DFF8DC81CF
:10D85000ACF1080C8C4500F088804A6822F0030285
:10D86000934202D289688C45F7D1D1F80CC07A680E
:10D87000C4F80CC0A160CCF80840CC6088E66319FD
:10D8800042F0010745F00105656030464B610B61D0
:10D89000C3F80CE0C3F808E05F609A50083400F069
:10D8A0007BF9D5E64A6873E608F1010818F0030F22
:10D8B0000CF1080C7FF47FAE30E0DC68A34208BFB7
:10D8C00002303FF435AEB3E60B440C465A68C968E3
:10D8D00054F8085F42F001025A603046E9608D60FA
:10D8E00000F05AF9B4E603F15C0E03F15B004FEA75
:10D8F0004E0307E69A0902F1390149003832A1E7DF
:10D90000BC424A4B3FF400AF9C68626822F00302BD
:10D910005AE759F80839994540F0828010F0030F12
:10D9200000F1FF30F5D17B6823EA04037B606400DB
:10D930009C423FF6BDAE002C3FF4BAAE1C424046BE
:10D940007FF435AE64001C4200F10400FAD02EE6EC
:10D95000B3F5AA7F18D8E80B00F1780E4FEA4E0312
:10D960007730CFE54FF48051EBE60121D8F8043051
:10D97000921001FA02F21A43C8F80420614677E7D0
:10D980000123CBF8043025E740F25452934220D8CB
:10D99000A80C00F17D0E4FEA4E037C30B2E5103248
:10D9A000A4E6542A26D81A0B02F16F0149006E3200
:10D9B00048E7BC68626822F0030205E7CAF30B007F
:10D9C00000287FF4A8AE4244BB6842F001025A60CE
:10D9D000ECE6FE234FF07F0E7E2093E501224FF010
:10D9E0000009C1E604F10801304600F09FFCD9F8B7
:10D9F0000010DBE6B2F5AA7F05D8DA0B02F1780158
:10DA0000490077321EE740F254518A4205D89A0CF9
:10DA100002F17D0149007C3214E7FE217E2211E7EC
:10DA20007B6884E7E808431C5B00F8E54496FF1F29
:10DA30008842F0B50DD98B1898420AD28118002A75
:10DA400051D09A1A13F8014D01F8014D9342F9D1C2
:10DA5000F0BD0F2A48D941EA00039B0746D100F1E7
:10DA6000100401F11003154653F8106C44F8106CC3
:10DA700053F80C6C44F80C6C53F8086C44F8086CC0
:10DA8000103D53F8046C44F8046C0F2D03F110039F
:10DA900004F11004E8D8A2F1100323F00F0302F000
:10DAA0000F0E1033BEF1030F1944034421D91E1F7A
:10DAB0000D467446043C55F8047B46F8047F032C5D
:10DAC000F8D8AEF1040424F00304043423442144C0
:10DAD00002F0030262B1013B0A4411F8014B03F862
:10DAE000014F8A42F9D1F0BD0346F3E70346F2E75E
:10DAF000F0BD7246EEE700BF70B4840746D0541EF6
:10DB0000002A41D0CDB2034602E0621EE4B31446BF
:10DB100003F8015B9A07F8D1032C2ED9CDB245EA60
:10DB200005250F2C45EA054519D903F110022646B3
:10DB3000103E0F2E42F8105C42F80C5C42F8085C74
:10DB400042F8045C02F11002F2D8A4F1100222F0B3
:10DB50000F0204F00F041032032C13440DD91E469B
:10DB60002246043A032A46F8045BFAD8221F22F020
:10DB700003020432134404F003042CB1C9B21C4460
:10DB800003F8011BA342FBD170BC70471446034647
:10DB9000C2E700BF704700BF704700BF024B0A4694
:10DBA0000146186800F002B84096FF1F2DE9F04FBB
:10DBB000174683B0002900F0C1800E46814607F168
:10DBC0000B05FFF7E7FF56F804EC162D2EF00304C3
:10DBD000A6F1080840D810221546AF4241D8944219
:10DBE00075DAC94B996808EB04008842416800F077
:10DBF000D98021F0010303445B68DB077DD51EF06B
:10DC0000010F35D039464846FFF75AFC0746E0B1C8
:10DC100056F8043C23F001034344A0F108029A4261
:10DC200000F04481221F242A00F23181132A00F2DD
:10DC30000481034632461168196051685960926840
:10DC40009A603146484600F071FB4846FFF7A4FF52
:10DC5000384603B0BDE8F08F25F00705002D2A46B1
:10DC6000BBDA0C230020C9F8003003B0BDE8F08F08
:10DC700056F8083CC3EB080ADAF8043023F0030C2A
:10DC800004EB0C039342BDDB5746DAF80C1057F84F
:10DC9000080F221F242AC160886000F21781132A0E
:10DCA00040F212813168CAF808107168CAF80C1085
:10DCB0001B2A00F22B8108360AF11002316811602C
:10DCC00071685160B16891603E461C46D046631B46
:10DCD0000F2B1DD8D8F8043003F00103234344442C
:10DCE000C8F80430636843F0010363604846FFF7F7
:10DCF00053FF304603B0BDE8F08F21F0030121440B
:10DD0000914221DBC36882680C46D3609A60DEE7EB
:10DD1000D8F8042008EB050102F00102154343F096
:10DD200001020B44C8F804504A605A6842F00102EC
:10DD300008315A60484600F0F9FAD7E7114603B0B7
:10DD4000BDE8F04FFFF7BCBB1EF0010F7FF45AAFE8
:10DD500056F8083CC3EB080ADAF8043023F0030C49
:10DD600001EB0C0E96458BDBC36882685746D36087
:10DD70009A6057F8081FDAF80C30CB60221F242A6B
:10DD8000996000F29980132A62D93368CAF8083082
:10DD90007368CAF80C301B2A00F2A08008360AF11A
:10DDA000100356E021F0030BA34405F11000834556
:10DDB00059DA1EF0010F7FF425AF56F8081CC1EBAD
:10DDC000080ADAF8041021F0030CE34458453FF741
:10DDD00057AF5746DAF80C1057F8080F221F242ABD
:10DDE000C160886000F2B480132A40F2A5803168D7
:10DDF000CAF808107168CAF80C101B2A00F2AF802C
:10DE000008360AF110023168116071685160B1681A
:10DE100091600AEB0501C5EB0B0242F0010299602B
:10DE20004A60DAF8043003F001031D434846CAF89B
:10DE30000450FFF7B1FE38465CE73368036073684F
:10DE400043601B2A27D800F1080306F10802F2E616
:10DE50003B4632681A6072685A60B2689A603E4601
:10DE60007446D04633E708EB0501C5EB0B0B4BF0CE
:10DE7000010299604A6056F8043C03F001031D4317
:10DE8000484646F8045CFFF787FE304632E73146E5
:10DE9000FFF7CEFDD5E6B3688360F368C360242A3C
:10DEA00028D000F1100306F11002C4E650F8043C3B
:10DEB00023F003031C440AE7314638467446D04633
:10DEC000FFF7B6FD3E4602E73A46F7E631463846EA
:10DED0001C46D046FFF7ACFD3E46F8E6B368CAF8EC
:10DEE0001030F368CAF81430242A1BD010360AF117
:10DEF0001803AEE7336903617369436106F11802E1
:10DF000000F1180397E600BF4496FF1FB168CAF8F6
:10DF10001010F168CAF81410242A0FD010360AF134
:10DF20001802CBE63369CAF818307369CAF81C3096
:10DF300018360AF120038CE73A4664E73269CAF8DA
:10DF400018207269CAF81C2018360AF12002B5E6BA
:10DF5000314638460193FFF76BFD019B59E7B168E5
:10DF6000CAF81010F168CAF81410242A03D0103629
:10DF70000AF1180247E73269CAF818207269CAF82C
:10DF80001C2018360AF120023DE700BF38B5074CC7
:10DF90000023054608462360FBF7E0FE431C00D043
:10DFA00038BD2368002BFBD02B6038BD40A1FF1F7C
:10DFB000FFFFFFFFFFFFFFFFFFFFFFFFFFFFFFFF71
:10DFC00090F800F06DE9024520F007016FF0000CB9
:10DFD00010F0070491F820F040F049804FF0000461
:10DFE0006FF00700D1E9002391F840F000F108003C
:10DFF00082FA4CF2A4FA8CF283FA4CF3A2FA8CF374
:10E000004BBBD1E9022382FA4CF200F10800A4FADA
:10E010008CF283FA4CF3A2FA8CF3E3B9D1E904232E
:10E0200082FA4CF200F10800A4FA8CF283FA4CF365
:10E03000A2FA8CF37BB9D1E9062301F1200182FA1F
:10E040004CF200F10800A4FA8CF283FA4CF3A2FA25
:10E050008CF3002BC6D0002A04BF04301A4612BA33
:10E06000B2FA82F2FDE8024500EBD2007047D1E936
:10E07000002304F00305C4F100004FEAC50514F0C5
:10E08000040F91F840F00CFA05F562EA05021CBF96
:10E0900063EA050362464FF00004A9E7002A41D075
:10E0A00040EA010313F00303F0B425D1032A23D976
:10E0B00004680D68AC421FD1043A35D0A4F1013593
:10E0C00025EA040414F0803F31D1071D0D1D0DE039
:10E0D00057F8043B0E68A3F10134B34224EA030469
:10E0E0000AD1043A20D014F0803F23D1032A2946D4
:10E0F000384605F10405EBD803780C789C4202F110
:10E10000FF320CD182B114B916E06AB17BB110F8BC
:10E11000013F11F8014FA34202F1FF32F5D0181B65
:10E12000F0BC7047104670471046F0BC7047184668
:10E13000F0BC70470020F3E72046F1E740EA010316
:10E140009B0770B42BD1032A29D90C4603462146DC
:10E1500054F8046BA6F1013525EA060515F0803F59
:10E1600006D1043A032A43F8046B2146EFD8A2B142
:10E170000C781C70013A013301313CB16AB111F8DD
:10E18000014B03F8014B013A002CF7D12AB11A4494
:10E19000002103F8011B9A42FBD170BC7047034673
:10E1A000E5E700BF2DE9F047254C2568D5F8484143
:10E1B0000646884692469946C4B360681F2817DC15
:10E1C000431C76B104EB80050122C5F888A0D4F881
:10E1D000881182401143022EC4F88811C5F80891B5
:10E1E0001ED00230636044F820800020BDE8F08734
:10E1F000144B03B34FF4C870FFF752F90446D0B183
:10E20000D5F84831002780E88800C5F848413846ED
:10E210000123C4F88871C4F88C71002EE1D0D1E7D5
:10E22000D4F88C110A43C4F88C21DAE705F5A674FA
:10E23000C5F84841C1E74FF0FF30BDE8F08700BFA7
:10E2400008010100A1D40000024B13B1024800F004
:10E2500005B870470000000069E200000023014695
:10E260001A461846FFF79EBF38B5074D074C2C1BC2
:10E27000A41005D0013C55F8043D9847002CF9D175
:10E28000BDE8384001F052BF00000000000000006F
:10E29000F8B5234F0C460646FFF77CFCBB685D686B
:10E2A00025F00305291B01F6EF7121F47F6121F0B0
:10E2B0000F01A1F58054B4F5805F07DB00213046E3
:10E2C000FFF764FEBB682B44984204D03046FFF74A
:10E2D00063FC0020F8BD61423046FFF757FE013075
:10E2E0000DD0104BBA6819682D1B45F0010530465A
:10E2F000091B55601960FFF74FFC0120F8BD002194
:10E300003046FFF743FEBA68831A0F2BDEDD064C5A
:10E310000449246843F00103001B53600860D5E7FB
:10E320004496FF1FE49FFF1F509AFF1F002945D00E
:10E330002DE9F0410D468046FFF72CFC55F8047C92
:10E340006A4927F00103A5F10804E2188E685068B5
:10E35000B24220F0030062D0FE0750600BD455F8A3
:10E36000087CE41B01F1080EA56875453B446FD09D
:10E37000E768EF60BD6015186D68ED0742D543F0A2
:10E3800001026260E350B3F5007F18D2DB085A1C2B
:10E390004D6851F83270A76001209B1000FA03F31A
:10E3A00001EBC2001D430838E0604D6041F8324087
:10E3B000FC604046BDE8F041FFF7EEBB70475A0AEB
:10E3C000042A53D89A0902F139077F0002F138056F
:10E3D00001EB870051F827204449083890424DD07E
:10E3E000516821F003018B4202D292689042F7D12A
:10E3F000D068E060A2608460D4604046BDE8F0412F
:10E40000FFF7CABB95683A4FBD4203443FD0D0687E
:10E41000E86043F0010285606260E350B3E7FF0704
:10E42000034407D455F8082CA41A1344A068E268E2
:10E43000C26090602F4A126843F00100934260600E
:10E440008C60B6D32C4B40461968FFF721FFB0E72C
:10E4500011184968C90744D49168D268CA60034456
:10E4600043F0010091606060E350A2E7142A17D8DE
:10E4700002F15C077F0002F15B05A9E7AA104B6877
:10E48000012505FA02F213434B600246B1E743F05F
:10E4900001024C610C61E560A5606260E35088E7B1
:10E4A000542A06D81A0B02F16F077F0002F16E059D
:10E4B0008EE7B2F5AA7F06D8DA0B02F178077F0063
:10E4C00002F1770584E740F25450824206D89A0C54
:10E4D00002F17D077F0002F17C0579E7FE277E25AA
:10E4E00076E743F001026260E35062E74496FF1F63
:10E4F0004C96FF1F4C9AFF1FE09FFF1F0000CC109F
:10E50000581BFC21AC26C62A7C2E3831F4334C36FD
:10E51000A438983A5A3C543D803E7A3FFF3FFFFF73
:10E520000000580246056608540BD80E5C1270179E
:10E53000FC21F82A70305834DC37663A8C3C803E37
:10E54000FF3FFFFF0000FF03FF07FF0BFF0FFF135D
:10E55000FF17FF1BFF1FFF23FF27FF2BFF2FFF339B
:10E56000FF37FF3BFF3FFFFF0000D007100E88136F
:10E570003219AA1E282374275C2B442F6432843559
:10E580004038663A8C3C803EFF3FFFFF0000900120
:10E5900020031405D0075A0AAC0DCC10B4146A1825
:10E5A000E81C342180252A2B70301437FF3FFFFFF1
:10E5B0000000580246056608540BD80E5C12E015A0
:10E5C000FA19141E6022AC265C2B0C30BC34023AC3
:10E5D000FF3FFFFF0000C800F40184031405080793
:10E5E0002E091C0CD80EF811AE159619401F1C25CB
:10E5F000F22B5834FF3FFFFF00006400C800900179
:10E60000BC021A04DC059E07F609800CA00F241337
:10E61000A2174C1D5424442FFF3FFFFF0000580257
:10E6200046056608540BA00FD4172823F82A442F58
:10E63000643284354038663A8C3C803EFF3FFFFFB1
:10E6400000007805220B0410B4143219B01DFC210F
:10E650004826FE29822D383126344637663A223D37
:10E66000FF3FFFFF0000540BEC13FA1908201C2594
:10E670003629EC2C0C302C33E8357238663AF63BF0
:10E68000863D163FFF3FFFFFFCE4000064E600000C
:10E6900068E5000040E6000044E50000B0E5000049
:10E6A0008CE50000D4E50000F8E5000020E500005E
:10E6B0001CE6000044E70000BCE600000000D007B4
:10E6C000800CD80E0010C012EC130C17FA19141E8F
:10E6D0006022AC265C2B0C30BC34023AFF3FFFFFBB
:10E6E00000000000CDCC4C3DCDCCCC3D9A99193EDC
:10E6F000CDCC4C3E0000803E9A99993E3333B33ED8
:10E70000CDCCCC3E6666E63E2C011301FA00E1005A
:10E71000C800AF0096007D0064004B003200190075
:10E7200040067805B004E80384032003BC025802C5
:10E73000F40190012C01FA00C80096006400320038
:10E740001900FFFF000078053408540B800C3C0FC3
:10E750005C12E015FA19141E6022AC265C2B0C30FA
:10E76000BC34023AFF3FFFFFD8E70000F69AFF1FD4
:10E770000000FF0F0A9CFF1F0000FF0F793400000C
:10E78000A4E70000689BFF1F32005E01000000004C
:10E79000000000001934000054485200534E53004A
:10E7A0004D415800544F5543482053454E53450062
:10E7B000455854524120434F4E54524F4C4C4552B1
:10E7C0000000000050495443482042454E44000098
:10E7D000424954450000000042524541544800FF60
:10E7E000B0E70000C09BFF1FF401A00F2E9BFF1F8E
:10E7F000F401A00F25340000D0E70000A09BFF1F0C
:10E80000BC025C12F29AFF1FBC025C125D34000075
:10E81000C4E70000F49BFF1FF401A00F649BFF1FDF
:10E82000F401A00F41340000C8EF0000D0EF000059
:10E83000CCEE00008CEF0000A8EF0000ACEF000071
:10E84000B0EF0000B4EF0000B8EF0000BCEF000034
:10E85000C0EF000094EF0000C4EF0000CCEE000019
:10E86000C8EE00009CEF0000A0EF0000A4EF000045
:10E87000CCEE00008CEF000090EF000094EF000061
:10E8800098EF00007CEF000080EF000084EF0000B4
:10E89000F0F3000088EF0000D8EF0000DCEF00008C
:10E8A000E0EF0000E4EF0000E8EF0000ECEF000014
:10E8B000F0EF0000F4EF0000F8EF0000FCEF0000C4
:10E8C00000F0000004F0000008F00000010000006B
:10E8D0004CF10000060000000000000000000000F5
:10E8E0000000000000000000000000000000000028
:10E8F0000000000000000000000000000000000018
:10E900000000000000000000000000000000000007
:10E9100000000000000000000000000000000000F7
:10E9200000000000000000000000000000000000E7
:10E9300000000000000000000000000000000000D7
:10E9400000000000000000000000000000000000C7
:10E9500000000000000000000000000000000000B7
:10E9600000000000000000000000000000000000A7
:10E970000000000000000000000000000000000097
:10E980000000000000000000000000000000000087
:10E990000000000000000000000000000000000077
:10E9A0000000000000000000000000000000000067
:10E9B0000000000000000000000000000000000057
:10E9C0000000000000000000000000000000000047
:10E9D0000000000000000000000000000000000037
:10E9E0000000000000000000000000000000000027
:10E9F0000000000000000000000000000001FFFF18
:10EA0000FFE3600007736000000000000001FFFFEB
:10EA1000FFE360000EE360000000000000018000E2
:10EA2000000360001DC36000000000000001BFFF84
:10EA3000FFE360003B836000000000000001BFFFB7
:10EA4000FFE3600077036000000000000001B000F9
:10EA500000036000EE036000000000000001B00051
:10EA600000036001DC036000000000000001B00052
:10EA700000036003B8036000000000200001B00044
:10EA80000003600770036000000000600001BFFF2A
:10EA9000FFE3600EE0036000000000600001BFFFC4
:10EAA000FFE3601DC0036000000300600001800000
:10EAB0000003603B80036000000300E00001BFFF33
:10EAC000FFE3607700036000000300C00001BFFFA8
:10EAD000FFE360EE00036000000380C00001B000AF
:10EAE000000361DC00036000000780C00001B0008B
:10EAF000000363B8000360000007C0C00001B0005D
:10EB000000036770000360000006C0C00001B00091
:10EB100000036EE000036000000660C10101B00068
:10EB200000037DC000036000000630C30301BFFF87
:10EB3000FFE37B8000036000000C30C30701BFFFD0
:10EB4000FFE3770000036000000C1CC30601800097
:10EB500000030E0000036000000C0CC20E01FFFF5A
:10EB6000FFE3FC0000036000000C0EC61E01FFFF67
:10EB7000FFE3F80000036000000C07C61E00000061
:10EB80000000000000000000000C03C6760000003A
:10EB90000000000000000000000C01C7E6000000BB
:10EBA0000000000000000000000C00C7C6000000CC
:10EBB0000000000000000000000C00030600000040
:10EBC0000000000000000000000C00000000000039
:10EBD0000000000000000000000C00000000000029
:10EBE0000000000000000000000000000000000025
:10EBF0000000000000000000000000000000000015
:10EC00000000000000000000000000000000000004
:10EC100000000000000000000000000000000000F4
:10EC200000000000000000000000000000000000E4
:10EC300000000000000000000000000000000000D4
:10EC400000000000000000000000000000000000C4
:10EC500000000000000000000000000000000000B4
:10EC600000000000000000000000000000000000A4
:10EC70000000000000000000000000000000000094
:10EC80000000000000000000000000000000000084
:10EC90000000000000000000000000000000000074
:10ECA0000000000000000000000000000000000064
:10ECB0000000000000000000000000000000000054
:10ECC0000000000000000000000000000000000044
:10ECD00000000000000000000000000070F20000D2
:10ECE00040F20000C29BFF1F000030000000000047
:10ECF000894D0000153E00000000000001000000EA
:10ED00006CF1000003000000010000000CF00000A6
:10ED100007000000000000004CF2000040F200007C
:10ED2000E49BFF1F0000300000000000994D000030
:10ED3000B13F0000000000000100000054F100009D
:10ED400005000000010000003CF100000800000088
:10ED500000000000F8F00000F8F000006A9BFF1FC0
:10ED600000000C00030000006D510000353E000063
:10ED7000000000000000000034F2000040F200003B
:10ED8000E69BFF1F0000300000000000994D0000CE
:10ED9000B13F000000000000000000000100000082
:10EDA000B54100000100000060F100000400000017
:10EDB0000000000074F100007CF10000429BFF1F86
:10EDC000010010000600000001540000253E000074
:10EDD000154800002C010000F5400000060000006E
:10EDE00009000000988DFF1F0CF2000000000301D5
:10EDF00006000000D48BFF1F00000000010000008F
:10EE0000A156000044F10000000005010A000000C6
:10EE1000648BFF1F0100000044F1000009000000A6
:10EE2000D0F0000000000101080000007C8CFF1FF2
:10EE30000000000064F2000040F20000E09BFF1FB1
:10EE40000000300000000000994D0000B13F0000BC
:10EE5000000000000CF000000000040508000000A5
:10EE6000788DFF1F000000001CF2000028F2000057
:10EE7000249BFF1F0000010001000000B5440000BA
:10EE8000053E0000000000000000000068F00000E7
:10EE900034F000003E9BFF1F00000900000000004E
:10EEA000D9440000453E00000000000000000000C2
:10EEB00001000000154A000070F00000000002018F
:10EEC000080000004C8EFF1F4F4E00004F464600CA
:10EED000424154004C4F572000000000555342005F
:10EEE0004D454E55202020202020202020585858C5
:10EEF00020592E595600000058000000524F54006F
:10EF00004D454C0044594E006D730000425448007A
:10EF1000424954004C5652004E524D005245560044
:10EF2000312F0000415400004D4F44005042440036
:10EF300045433200454353004C564C004C5650005C
:10EF4000474C4400762E0000312E342E3500000050
:10EF50004E754556490000006669726D77617265AD
:10EF600020762E0053455400434C5200444F4E2708
:10EF70005400000050414E494300000045574900ED
:10EF80004557580053415800455652004D57000010
:10EF90004650000043460000535000005357000005
:10EFA00053454C005345450042520000564C00006A
:10EFB000455800004D572B0042522B00564C2B0059
:10EFC00045582B00554E4F00425254480000000057
:10EFD00050544348000000002D3400002D33000041
:10EFE0002D3200002D3100004C494E002B31000025
:10EFF0002B3200002B3300002B3400005331000073
:10F00000533200005A3100005A3200005649425231
:10F0100041544F00444952454354494F4E0000006B
:10F02000434F4E54524F4C00535155454C4348208A
:10F03000420000004C4556454C00000053454E53DD
:10F040004520425445000000535155454C4348204B
:10F050004C00000053454E5345204C5652000000D2
:10F0600052455455524E000044455054480000004B
:10F070005345545550204354524C53004C4556452B
:10F080004C2043430000000050494E4B59204B4553
:10F09000590000004445474C4954434800000000D3
:10F0A00045584354522043433200000045585452BF
:10F0B0004120435452000000504954434842454EB9
:10F0C00044000000504F52542F474C4400000000B1
:10F0D00053455455502042524541544800000000C9
:10F0E00056454C20424F4F535400000056454C208B
:10F0F00044454C415900000043555256450000001C
:10F1000056454C4F43495459000000004252454176
:10F110005448204154000000434332205249534593
:10F1200000000000425254482043433200000000D7
:10F1300042525448204343310000000041424F55A1
:10F14000540000004558545241530000524F54415E
:10F15000544F520053455455502043544C00000026
:10F1600053455455502042520000000041444A5536
:10F17000535400004D494449204348004D494449F7
:10F180002043484E4C000000574C204348414E005D
:10F19000574C20504F5745520000000046415354F1
:10F1A00020424F4F54000000444143204F5554002B
:10F1B00042434153204D4F44450000003352442008
:10F1C0005452494C4C00000053504543204B455984
:10F1D000000000004741544520484F4C44000000C7
:10F1E0004C45474143592042520000004C4547419D
:10F1F00043592050420000004F43544156450000FF
:10F200005452414E53504F5345000000524F544109
:10F21000544F522053455455500000005052494F0E
:10F2200052495459000000004D4F4E4F2050524952
:10F230004F000000524F544154452034000000005C
:10F2400053454D49544F4E4553000000524F5441D1
:10F250005445203300000000524F544154452032A1
:10F2600000000000524F544154452031000000007E
:10F27000504152414C4C454C00FFFFFF0000000044
:10F2800058F2000040F20000E29BFF1F0000300037
:10F2900000000000994D0000B13F00000000000098
:10F2A0000021110202000000002111020504FFFFED
:10F2B000003E7FFF4E754556496330310000000027
:10F2C0007676764E75455649636363007676764E5C
:10F2D000754556496330346565767676767676760A
:10F2E00076000000496E76616C696420636F6E661B
:10F2F000696720666F726D6174000000496E766107
:10F300006C696420636865636B73756D0000000051
:10F31000496E76616C696420636F6E6669672073FD
:10F32000697A6500496E76616C696420636F6E6608
:10F3300069672076657273696F6E0000496E766149
:10F340006C6964206D6573736167652E0000000051
:10F35000653030006330300053656E64696E67203D
:10F36000636F6E6669672E2E2E000000436F6E6617
:10F3700069672073656E742E0000000063303300EF
:10F3800053656E64696E672076657273696F6E2E61
:10F390000000000063303200526563656976696E73
:10F3A0006720636F6E6669672E2E2E004E6577208C
:10F3B000636F6E6669672073617665642E00000076
:10F3C000556E6B6E6F776E206D6573736167652E1A
:10F3D0000000000065303100436F6E666967206D84
:10F3E000676D7400506F776572206F6666204E758A
:10F3F00045564900746F20657869740052656164F0
:10F40000792E00FF34800440400000001211FFFFFD
:10F41000FF02020000001310FFFFFF0202000000C5
:10F420001800000034800440800000001EFFFFFF31
:10F43000FF02000000001DFFFFFFFF0200000000B0
:10F4400019000000000000000000000051720000E0
:10F4500015720000C971000011720000CD7100002A
:10F46000D9710000F9710000000103070F1F3F7FF1
:10F470002200FF2100FFFFFF0080C0E0F0F8FCFE4B
:10F480000000000000000000A991000005960000A7
:10F49000C9710000D57B00006D7C0000518A00001E
:10F4A000058A0000398A0000118A0000258A0000C0
:10F4B00021890000518A0000798A0000697E0000DD
:10F4C000B18600004D860000498B0000558A00007F
:10F4D000AD8B00004D8C0000DA02818FDA1281FFC3
:10F4E00000006000000000000000000000000000BC
:10F4F00000E000000000000000000000000000012B
:10F50000E00000000000000000000000000001F02A
:10F510000000000000000000000000000003F000F8
:10F5200000000000000000000000000007F00000E4
:10F53000000000000000000000000007F8000000CC
:10F54000000000000000000000000FF800000003B1
:10F55000C0007E000001E0007F0FF800000003C043
:10F5600000FE000001E000FFEFF800000003C00013
:10F57000FE000001E000FFFFF800000003C000F003
:10F580000000000F007FFE7FC0000003C000F000FD
:10F5900000000F003FFE7FF83FF1FBCFFCFEF3BC05
:10F5A0003DEFE01FFE7FFF7FFBFFDFFEFEFFBC3D68
:10F5B000EFE01FC6FFFF7FFBFFDFFEFEFFBC3DEF5E
:10F5C000E00FE3C7FE787BC3DE1EF0FFBC3DEF001B
:10F5D00007FF87FC787BC3DE1EF0F83C3DEF00019F
:10F5E000FFFFF0007BC3C01EF0F03C3DEF0001F3D5
:10F5F0007FE03FFBC3CFFEF0F03C3DEF0003E33F75
:10F60000807FFBC3DFFEF0F03C3DEF0007E73C00EE
:10F61000787BC3DE1EF0F03C3DEF0007FFBE0078B4
:10F620007BC3DE1EF0F03C3DEF0007FFFE00787B61
:10F63000C3DE1EF0F03C3DEF000FFFFE007FFBFF3E
:10F64000DFFEF0F03FFDEFE00FFFFF007FFBFFDF8D
:10F65000FEF0F03FFDEFE00FF9FF003E79F9CF9E9D
:10F66000F0F01F3DE7E01FF1FF0000000000000088
:10F6700000000000001F80FF007FFFFFFFFFFFFF73
:10F68000FFFFFFE01C007F007FFFFFFFFEB46D88DF
:10F690008D18E000001F007FFFFFFFFE95AD7DB5D8
:10F6A00077E000000F007FFFFFFFFEA5AD9D8D19E5
:10F6B000E0000006007FFFFFFFFEB5ADEDB57EE088
:10F6C000AED580A8D300408D2000A1C8DB40A4A601
:10F6D0002EAFFFFF000000000001800000000000CE
:10F6E0000000000003800000000000000000000790
:10F6F000C000000000000000000007C00000000083
:10F7000000000000000FC00000000000000000002A
:10F710001FE00000000000000000001FE0000000EB
:10F720000000000000003FE00000000000000000BA
:10F73000003FF00000000000000000007FF000002B
:10F7400000000000001FF87FF00000000000000033
:10F750003FFE7FF0000000000000003FFF7FF00050
:10F760000000000000001FFFFBE0000000000000A0
:10F77000000FFFF9FFC00000000000000FFFF9FFBD
:10F78000F800000000000007FFF1FFFF000000008C
:10F79000000003FC73FFFF80000000000001FE3F3B
:10F7A000FFFF80000000000000FF1E0FFF000000B0
:10F7B000000000007FFE1FFC000000000000003F72
:10F7C000FFFFF8000000000000000FDFFFE0000076
:10F7D00000000000001F19FFC00000000000000032
:10F7E0003F3CFF00000000000000007E7CF80000AD
:10F7F0000000000000007FFE7C0000000000000010
:10F8000000FFFFFC0000000000000000FFFFFE0002
:10F8100000000000000000FFFFFE000000000000EC
:10F820000001FFEFFE0000000000000001FFCFFE1E
:10F830000000000000000003FF07FE0000000000C1
:10F84000000003FC07FE0000000000000003F003BE
:10F85000FE00000000000000018000FE000000002B
:10F860000000000000007E0000000000000000001A
:10F87000003E000000000000000000000C0000003E
:10F88000000000078000FC000003C00000000780AB
:10F8900001FC000003C0000000078001FC00000321
:10F8A000C0000000078001E00000001E000000070B
:10F8B0008001E00000001E007FE3F79FF9FDE7787C
:10F8C0007BDFC0FFF7FFBFFDFDFF787BDFC0FFF7E9
:10F8D000FFBFFDFDFF787BDFC0F0F787BC3DE1FF98
:10F8E000787BDE00F0F787BC3DE1F0787BDE00003E
:10F8F000F787803DE1E0787BDE007FF7879FFDE1C1
:10F90000E0787BDE00FFF787BFFDE1E0787BDE007B
:10F91000F0F787BC3DE1E0787BDE00F0F787BC3D87
:10F92000E1E0787BDE00F0F787BC3DE1E0787BDE4C
:10F9300000FFF7FFBFFDE1E07FFBDFC0FFF7FFBF88
:10F94000FDE1E07FFBDFC07CF3F39F3DE1E03E7B28
:10F95000CFC00000000000000000000000FFFFFF1B
:10F96000FFFFFFFFFFFFFFC0FFFFFFFFFD68DB1191
:10F970001A31C0FFFFFFFFFD2B5AFB6AEFC0FFFFEC
:10F98000FFFFFD4B5B3B1A33C0FFFFFFFFFD6B5BCF
:10F99000DB6AFDC0DA0281FF000000000000000009
:10F9A000A991000005960000C9710000D57B0000F8
:10F9B000899D0000518A0000058A0000398A0000F4
:10F9C000118A0000258A000021890000518A000068
:10F9D000798A0000758A00009D8A0000F58A00007F
:10F9E000498B0000558A0000AD8B00004D8C000053
:10F9F00000000000003E5B4F5B3E3E6B4F6B3E1CC9
:10FA00003E7C3E1C183C7E3C181C577D571C1C5EDF
:10FA10007F5E1C00183C1800FFE7C3E7FF001824B6
:10FA20001800FFE7DBE7FF30483A060E2629792960
:10FA300026407F050507407F05253F5A3CE73C5A95
:10FA40007F3E1C1C08081C1C3E7F14227F22145F72
:10FA50005F005F5F06097F017F006689956A6060CD
:10FA600060606094A2FFA29408047E040810207EC7
:10FA7000201008082A1C08081C2A08081E1010104C
:10FA8000100C1E0C1E0C30383E3830060E3E0E0692
:10FA9000000000000000005F0000000700070014E5
:10FAA0007F147F14242A7F2A1223130864623649A4
:10FAB0005620500008070300001C2241000041228C
:10FAC0001C002A1C7F1C2A08083E08080080703091
:10FAD0000008080808080000606000201008040200
:10FAE0003E5149453E00427F400072494949462106
:10FAF00041494D331814127F1027454545393C4A7A
:10FB00004949314121110907364949493646494990
:10FB1000291E0000140000004034000000081422D8
:10FB20004114141414140041221408020159090646
:10FB30003E415D594E7C1211127C7F494949363E47
:10FB4000414141227F4141413E7F494949417F092D
:10FB50000909013E414151737F0808087F00417F38
:10FB600041002040413F017F081422417F40404036
:10FB7000407F021C027F7F0408107F3E4141413ECE
:10FB80007F090909063E4151215E7F091929462650
:10FB90004949493203017F01033F4040403F1F2054
:10FBA00040201F3F4038403F63140814630304782B
:10FBB00004036159494D43007F414141020408104B
:10FBC00020004141417F0402010204404040404086
:10FBD000000307080020545478407F2844443838F4
:10FBE00044444428384444287F3854545418000866
:10FBF0007E090218A4A49C787F0804047800447D40
:10FC000040002040403D007F1028440000417F40DC
:10FC1000007C047804787C08040478384444443830
:10FC2000FC1824241818242418FC7C080404084810
:10FC30005454542404043F44243C4040207C1C2061
:10FC400040201C3C4030403C44281028444C9090BC
:10FC5000907C4464544C4400083641000000770016
:10FC600000004136080002010204023C2623263C23
:10FC70001EA1A161123A4040207A385454555921AE
:10FC80005555794122545478422155547840205496
:10FC90005579400C1E5272123955555559395454E4
:10FCA000545939555454580000457C410002457D53
:10FCB000420001457C407D1211127DF0282528F07C
:10FCC0007C545545002054547C547C0A097F4932A9
:10FCD000494949323A4444443A324A4848303A4120
:10FCE00041217A3A42402078009DA0A07D3D4242C9
:10FCF000423D3D4040403D3C24FF2424487E494352
:10FD0000662B2FFC2F2BFF0929F620C0887E0903C4
:10FD100020545479410000447D413048484A3238EB
:10FD20004040227A007A0A0A727D0D19317D262917
:10FD3000292F28262929292630484D40203808080F
:10FD4000080808080808382F10C8ACBA2F10283443
:10FD5000FA00007B000008142A142222142A140836
:10FD60005500550055AA55AA55AAFF55FF55FF0045
:10FD70000000FF00101010FF00141414FF001010FA
:10FD8000FF00FF1010F010F0141414FC001414F70E
:10FD900000FF0000FF00FF1414F404FC14141710FB
:10FDA0001F10101F101F1414141F00101010F0004B
:10FDB0000000001F101010101F10101010F0100085
:10FDC0000000FF101010101010101010FF10000095
:10FDD00000FF140000FF00FF00001F10170000FCD0
:10FDE00004F414141710171414F404F40000FF00A2
:10FDF000F714141414141414F700F714141417142B
:10FE000010101F101F141414F4141010F010F00030
:10FE1000001F101F0000001F14000000FC14000051
:10FE2000F010F01010FF10FF141414FF1410101035
:10FE30001F00000000F010FFFFFFFFFFF0F0F0F0E8
:10FE4000F0FFFFFF0000000000FFFF0F0F0F0F0F7C
:10FE50003844443844FC4A4A4A347E0202060602C8
:10FE60007E027E0263554941633844443C04407E2F
:10FE7000201E2006027E020299A5E7A5991C2A49A8
:10FE80002A1C4C7201724C304A4D4D303048784833
:10FE900030BC625A463D3E494949007E0101017E1F
:10FEA0002A2A2A2A2A44445F444440514A44404072
:10FEB000444A51400000FF0103E080FF00000808B1
:10FEC0006B6B083612362436060F090F0600001831
:10FED000180000001010003040FF0101001F010158
:10FEE0001E00191D1712003C3C3C3C0000000000A5
:10FEF0000D0AFFFF050E08090D0C06070F0400137D
:10FF00000393050E08090D0C06070F04FFFFC585B6
:10FF1000848687C4FFFF001303931A9217FFFFFF25
:10FF20006FF07F030370037813F0800FFBD07047EE
:10FF30004008FE4340A004404408FE4344A004405F
:10FF40000018FE4300C004403000FE4330900440DF
:10FF50003400FE43349004401C18FE431CC004408F
:10FF60001018FE4310C004400818FE4308C00440A7
:10FF70000C18FE430CC004400C10FE430CB00440AF
:10FF80001010FE4310B004401810FE4318B0044097
:10FF90001C10FE431CB004401410FE4314B0044077
:10FFA0000418FE4304C004400010FE4300B00440A7
:10FFB0000008FE4300A004400408FE4304A00440DF
:10FFC0000C08FE430CA004400808FE4308A00440AF
:10FFD0001418FE4314C004401818FE4318C004400F
:10FFE0000410FE4304B004400810FE4308B004406F
:10FFF0001400FE43149004404C08FE434CA00440FF
:020000021000EC
:100000000420FE4304D004402410FE4324B00440E6
:100010002010FE4320B004402810FE4328B00440C6
:100020002C10FE432CB004400020FE4300D00440BE
:100030004808FE4348A004401000FE4310900440CE
:10004000090AFFFFFFFFFFFFFFFFFFFFFFFFFF0D9D
:1000500000060807FFFF0E0FFF0CFFFFFFFFFFFF6B
:100060000B05FFFF15191519000100003491FF1F42
:1000700012000000000200006091FF1F73000000EA
:1000800000220100D491FF1F210000000021010087
:10009000BC91FF1F0900000000030000F891FF1F42
:1000A00000000000010309044891FF1F0000000048
:1000B00002030904448FFF1F00000000030309042A
:1000C000FC91FF1F00000000000000000000000085
:1000D0000000000065787000000000000000E03FB4
:1000E000000000000000E0BF763C7935EF39EA3DC2
:1000F000763C7935EF39EABD0000E0FE422EE63F5E
:100100000000E0FE422EE6BF1892FF1FF8B500BFC8
:10011000F8BC08BC9E46704749E200003504000068
:0C012000D1330000414E0000456E00008D
:04012C00F8B500BF63
:1001300038B5084B1C681C6054B1074D94FAA4F301
:10014000B3FA83F355F823309847631E1C40F5D16A
:1001500038BD00BFA0D004402491FF1F38B5084B24
:100160001C681C6054B1074D94FAA4F3B3FA83F3EE
:1001700055F823309847631E1C40F5D138BD00BFA9
:10018000A0C004400491FF1F38B5084B1C681C60D8
:1001900054B1074D94FAA4F3B3FA83F355F823301E
:1001A0009847631E1C40F5D138BD00BFA0B0044085
:1001B000D490FF1F38B5084B1C681C6054B1074D24
:1001C00094FAA4F3B3FA83F355F823309847631EE7
:1001D0001C40F5D138BD00BFA0A004408490FF1F93
:1001E00038B5084B1C681C6054B1074D94FAA4F351
:1001F000B3FA83F355F823309847631E1C40F5D1BA
:1002000038BD00BFA09004404C90FF1F00000000CC
:1002100000200000000102070B0102070B4A140036
:10022000320000000100000000200000002000005B
:1002300000100000AB0A0000000800006606000085
:100240005505000092040000000400008E03000029
:1002500033030000E8020000AB02000024000000AD
:100260000020000002000200FBFFFFFF0000000072
:10027000000000000000000000000000000000007E
:100280000000000000000000000000000C00000062
:10029000140500000C0000000000F0410200FFFF08
:1002A000FFFF000068E70000F8E7000010E800002A
:1002B000E0E7000080E700000000000048F00000D8
:1002C00034F000009C89FF1F01001E0000000000A8
:1002D000000000000000000000000000000000001E
:1002E000ECF10000ECF10000BC9BFF1F00000100DE
:1002F00001000000000000000000000000000000FD
:100300000000000090F1000090F10000B09CFF1F81
:1003100000000300000000000000000000000000DA
:100320000000000000000000BCF10000BCF1000073
:100330005C9BFF1F030004000000000000000000A1
:1003400000000000000000000000000001000000AC
:1003500000000000000000000CF100000CF10000A3
:100360007C9BFF1F00000100010000000000000056
:10037000000000000000000000000000E0F00000AD
:10038000E0F00000889AFF1F000009000100000053
:10039000000000000000000000000000000000005D
:1003A00018F1000018F100009A9AFF1F01000A00DE
:1003B000010000000000000000000000000000003C
:1003C0000000000060F0000034F00000AC89FF1F66
:1003D0000000040000000000000000000000000019
:1003E0000000000000000000B0F10000B0F10000CB
:1003F000BE9BFF1F00000100000000000000000085
:10040000000000000000000000000000B8F0000044
:10041000B8F000008E9BFF1F00000C0000000000E1
:1004200000000000000000000000000000000000CC
:10043000F8F10000F8F10000209BFF1F000006000B
:1004400000000000000000000000000000000000AC
:1004500001000000EC89FF1F548DFF1F8C8BFF1FD4
:100460009C8CFF1F348AFF1FF48AFF1F6C8EFF1FB6
:10047000D88EFF1F108AFF1FE88CFF1F00000000AE
:10048000D4F10000D4F10000B09AFF1F0000010079
:10049000010000000000000000000000000000005B
:1004A00000000000C4F00000C4F000002C9BFF1FFF
:1004B0000000040001000000000000000000000037
:1004C00000000000D8EC000030EE00007CF20000DC
:1004D00014ED000074ED000064EE00000000000068
:1004E00024F1000024F10000889BFF1F00007F0022
:1004F00001000000000000000000000000000000FB
:1005000000000000ECF00000ECF00000809BFF1FFA
:1005100000001E00010000000000000000000000BC
:10052000000000000000000054F0000034F0000063
:100530007489FF1F01000C00000000000000000093
:1005400000000000000000000000000094F0000027
:1005500094F00000089CFF1F00004600000000000F
:10056000000000000000000000000000048EFF1FDB
:10057000EC8BFF1FAC8AFF1F648AFF1F208FFF1FB9
:1005800050ED0000108CFF1F888AFF1F0000000044
:10059000C8F10000C8F100008C9BFF1F00000100A3
:1005A000010000000000000000000000000000004A
:1005B0000000000000F2000000F20000CE9BFF1FD0
:1005C0000000180000000000000000000000000013
:1005D00000000000040000000000000088F100009E
:1005E00088F10000E48CFF1F0400500000000000B0
:1005F00000000000000000000000000000000000FB
:1006000014F0000014F00000069CFF1F0000010021
:1006100001000000000000000000000000000000D9
:1006200000000000ACF00000ACF00000BA9BFF1F1F
:1006300000000400010000000000000000000000B5
:100640000000000000000000E0F10000E0F1000008
:100650001C9BFF1F000001000100000000000000C3
:100660000000000000000000FC8EFF1F88EE00006C
:10067000D08AFF1F0C8DFF1F348CFF1FC889FF1FFE
:10068000BC8DFF1FE08DFF1FC08CFF1F3C8BFF1F29
:10069000B0ED0000FCEC0000A4ED000038ED00001F
:1006A000CCE8000014EE000044ED00000000000063
:1006B0003CF0000034F000007689FF1F01001100BB
:1006C000000000000000000000000000000000002A
:1006D0000000000028F0000034F00000A489FF1F93
:1006E00001001E00000000000000000000000000EB
:1006F000000000000000000030F1000030F10000B8
:100700008C9AFF1F00000A0001000000000000009A
:1007100000000000000000000000000088F0000061
:1007200088F00000F89AFF1F00001D000000000084
:10073000000000000000000000000000B08BFF1F60
:10074000308DFF1F908EFF1F08ED0000588CFF1F9B
:10075000288EFF1FB48EFF1F188BFF1F00000000A4
:10076000A8F10000A8F10000669BFF1F0000010037
:100770000000000000000000000000000000000079
:1007800000000000A0F00000A0F00000789AFF1F19
:1007900000007F00010000000000000000000000D9
:1007A00000000000000000007CF000007CF0000071
:1007B000A69AFF1F00007F0001000000000000005B
:1007C0000000000000000000000000009CF100009C
:1007D0009CF10000FC9BFF1F0000010000000000D6
:1007E0000000000000000000000000000000000009
:1007F00020F0000020F000008A9AFF1F0000020095
:1008000001000000000000000000000000000000E7
:100810000000000000F1000000F10000589BFF1FE5
:1008200000007F0001000000000000000000000048
:100830000000000016034E007500450056004900F8
:1008400020004D0049004400490000004CF4000025
:1008500000000000E8030000000000000060064007
:1008600004F4000000000000000000000000000090
:100870000000000000000000000000000000000078
:100880000000000000000000000000000000000068
:100890000000000000000000000000000000000058
:1008A0000000000000000000000000000000000048
:1008B00000000000000000004CF4000000000000F8
:1008C000E8030000000000000070064024F400006F
:1008D0000000000000000000000000000000000018
:1008E0000000000000000000000000000000000008
:1008F00000000000000000000000000000000000F8
:1009000000000000000000000000000000000000E7
:1009100000000000000000000000000000000000D7
:1009200000000000D9940000D9940000D994000080
:10093000D99400000A04000044A1FF1F159E000086
:10094000159E0000159E0000159E0000159E0000DB
:10095000159E0000159E0000159E0000159E0000CB
:10096000159E0000159E0000159E0000159E0000BB
:10097000159E0000159E0000159E0000159E0000AB
:10098000159E0000159E0000159E0000159E00009B
:10099000159E0000159E0000159E0000159E00008B
:1009A000159E0000159E0000159E0000159E00007B
:1009B000159E0000159E0000159E0000159E00006B
:1009C000159E0000159E0000159E0000159E00005B
:1009D000159E0000159E0000159E0000159E00004B
:1009E000159E0000159E0000159E0000159E00003B
:1009F000159E0000159E0000159E0000159E00002B
:100A0000159E0000159E0000159E0000159E00001A
:100A1000159E0000159E0000159E000008000000B5
:100A2000FFFFFFFF1201100100000040C016850407
:100A300075020102030100001803540065006500FF
:100A40006E00730079006400750069006E006F002D
:100A500009027300020100C0320904000002010310
:100A60000000072401000125000624020101000600
:100A700024020202000924030103010201000924E7
:100A80000302040101010009050402400000000006
:100A9000052501010109058302400000000005252C
:100AA00001010309040100020300000009211101F2
:100AB0000001222100070581034000010705020310
:100AC0002000020006C9FF0904A15C750815002674
:100AD000FF009540097581029520097691029504E1
:100AE0000976B102C0000000040309040C030000F1
:100AF00000000000000000000000000000000000F6
:100B00000000010000000000000000000495FF1F2D
:100B10006C95FF1FD495FF1F00000000000000002F
:100B200000000000000000000000000000000000C5
:100B300000000000000000000000000000000000B5
:100B400000000000000000000000000000000000A5
:100B50000000000000000000000000000000000095
:100B60000000000000000000000000000000000085
:100B70000000000000000000000000000000000075
:100B80000000000000000000000000000000000065
:100B90000000000000000000000000000000000055
:100BA0000000000000000000000000000000000045
:100BB00001000000000000000E33CDAB34126DE6E2
:100BC000ECDE05000B00000000000000000000004B
:100BD0000000000000000000000000000000000015
:100BE0000000000000000000000000000000000005
:100BF00000000000000000000000000000000000F5
:100C000000000000000000000000000000000000E4
:100F30001892FF1F00000000000000004496FF1FF1
:100F40004496FF1F4C96FF1F4C96FF1F5496FF1FA1
:100F50005496FF1F5C96FF1F5C96FF1F6496FF1F51
:100F60006496FF1F6C96FF1F6C96FF1F7496FF1F01
:100F70007496FF1F7C96FF1F7C96FF1F8496FF1FB1
:100F80008496FF1F8C96FF1F8C96FF1F9496FF1F61
:100F90009496FF1F9C96FF1F9C96FF1FA496FF1F11
:100FA000A496FF1FAC96FF1FAC96FF1FB496FF1FC1
:100FB000B496FF1FBC96FF1FBC96FF1FC496FF1F71
:100FC000C496FF1FCC96FF1FCC96FF1FD496FF1F21
:100FD000D496FF1FDC96FF1FDC96FF1FE496FF1FD1
:100FE000E496FF1FEC96FF1FEC96FF1FF496FF1F81
:100FF000F496FF1FFC96FF1FFC96FF1F0497FF1F30
:101000000497FF1F0C97FF1F0C97FF1F1497FF1FDC
:101010001497FF1F1C97FF1F1C97FF1F2497FF1F8C
:101020002497FF1F2C97FF1F2C97FF1F3497FF1F3C
:101030003497FF1F3C97FF1F3C97FF1F4497FF1FEC
:101040004497FF1F4C97FF1F4C97FF1F5497FF1F9C
:101050005497FF1F5C97FF1F5C97FF1F6497FF1F4C
:101060006497FF1F6C97FF1F6C97FF1F7497FF1FFC
:101070007497FF1F7C97FF1F7C97FF1F8497FF1FAC
:101080008497FF1F8C97FF1F8C97FF1F9497FF1F5C
:101090009497FF1F9C97FF1F9C97FF1FA497FF1F0C
:1010A000A497FF1FAC97FF1FAC97FF1FB497FF1FBC
:1010B000B497FF1FBC97FF1FBC97FF1FC497FF1F6C
:1010C000C497FF1FCC97FF1FCC97FF1FD497FF1F1C
:1010D000D497FF1FDC97FF1FDC97FF1FE497FF1FCC
:1010E000E497FF1FEC97FF1FEC97FF1FF497FF1F7C
:1010F000F497FF1FFC97FF1FFC97FF1F0498FF1F2B
:101100000498FF1F0C98FF1F0C98FF1F1498FF1FD7
:101110001498FF1F1C98FF1F1C98FF1F2498FF1F87
:101120002498FF1F2C98FF1F2C98FF1F3498FF1F37
:101130003498FF1F3C98FF1F3C98FF1F4498FF1FE7
:101140004498FF1F4C98FF1F4C98FF1F5498FF1F97
:101150005498FF1F5C98FF1F5C98FF1F6498FF1F47
:101160006498FF1F6C98FF1F6C98FF1F7498FF1FF7
:101170007498FF1F7C98FF1F7C98FF1F8498FF1FA7
:101180008498FF1F8C98FF1F8C98FF1F9498FF1F57
:101190009498FF1F9C98FF1F9C98FF1FA498FF1F07
:1011A000A498FF1FAC98FF1FAC98FF1FB498FF1FB7
:1011B000B498FF1FBC98FF1FBC98FF1FC498FF1F67
:1011C000C498FF1FCC98FF1FCC98FF1FD498FF1F17
:1011D000D498FF1FDC98FF1FDC98FF1FE498FF1FC7
:1011E000E498FF1FEC98FF1FEC98FF1FF498FF1F77
:1011F000F498FF1FFC98FF1FFC98FF1F0499FF1F26
:101200000499FF1F0C99FF1F0C99FF1F1499FF1FD2
:101210001499FF1F1C99FF1F1C99FF1F2499FF1F82
:101220002499FF1F2C99FF1F2C99FF1F3499FF1F32
:101230003499FF1F3C99FF1F3C99FF1F4499FF1FE2
:101240004499FF1F4C99FF1F4C99FF1F5499FF1F92
:101250005499FF1F5C99FF1F5C99FF1F6499FF1F42
:101260006499FF1F6C99FF1F6C99FF1F7499FF1FF2
:101270007499FF1F7C99FF1F7C99FF1F8499FF1FA2
:101280008499FF1F8C99FF1F8C99FF1F9499FF1F52
:101290009499FF1F9C99FF1F9C99FF1FA499FF1F02
:1012A000A499FF1FAC99FF1FAC99FF1FB499FF1FB2
:1012B000B499FF1FBC99FF1FBC99FF1FC499FF1F62
:1012C000C499FF1FCC99FF1FCC99FF1FD499FF1F12
:1012D000D499FF1FDC99FF1FDC99FF1FE499FF1FC2
:1012E000E499FF1FEC99FF1FEC99FF1FF499FF1F72
:1012F000F499FF1FFC99FF1FFC99FF1F049AFF1F21
:10130000049AFF1F0C9AFF1F0C9AFF1F149AFF1FCD
:10131000149AFF1F1C9AFF1F1C9AFF1F249AFF1F7D
:10132000249AFF1F2C9AFF1F2C9AFF1F349AFF1F2D
:10133000349AFF1F3C9AFF1F3C9AFF1F00000200D7
:04134000FFFFFFFFAD
:00000001FF
